:020000040000FA
:10000000000404000000000094CE000094CE000024
:1000100094CE000094CE000094CE000094CE000058
:1000200094CE000094CE000094CE000094CE000048
:1000300094CE00006AA3000094CE000094CE00008D
:1000400094CE000094CE000094CE000094CE000028
:1000500094CE000094CE000094CE000094CE000018
:1000600094CE000094CE000094CE000094CE000008
:1000700094CE000094CE000094CE000094CE0000F8
:1000800094CE000094CE000094CE000094CE0000E8
:1000900094CE000094CE000094CE000094CE0000D8
:1000A00094CE000094CE000094CE000094CE0000C8
:1000B00094CE000094CE000094CE000094CE0000B8
:1000C00094CE000094CE000094CE000094CE0000A8
:1000D00094CE000094CE000094CE000094CE000098
:1000E00094CE000094CE000094CE000094CE000088
:1000F00094CE000094CE000094CE000094CE000078
:1001000094CE000094CE000094CE000094CE000067
:1001100094CE000094CE000094CE000094CE000057
:1001200094CE000094CE000094CE000094CE000047
:1001300094CE000094CE000094CE000094CE000037
:1001400094CE000094CE000094CE000094CE000027
:1001500094CE000094CE000094CE000094CE000017
:1001600094CE000094CE000094CE000094CE000007
:1001700094CE000094CE000094CE000094CE0000F7
:1001800094CB000094CE000094CE000094CE0000EA
:1001900094CE000094CE000094CE000094CE0000D7
:1001A00094CE000094CE000094CE000094CE0000C7
:1001B00094CE000094CE000094CE000094CE0000B7
:1001C00094CE000094CE000094CE000094CE0000A7
:1001D00094CE000094CE000094CE000094CE000097
:1001E00094CE000094CE000094CE000094CE000087
:1001F00094CE000094CE000094CE000094CE000077
:10020000FFFFFF00FFFFFF0094CE000094CE000030
:1002100094CE000094CE000094CE000094CE000056
:1002200094CE000094CE000094CE000094CE000046
:1002300094CE00006AA3000094CE000094CE00008B
:1002400094CE000094CE000094CE000094CE000026
:1002500094CE000094CE000094CE000094CE000016
:1002600094CE000094CE000094CE000094CE000006
:1002700094CE000094CE000094CE000094CE0000F6
:1002800094CE000094CE000094CE000094CE0000E6
:1002900094CE000094CE000094CE000094CE0000D6
:1002A00094CE000094CE000094CE000094CE0000C6
:1002B00094CE000094CE000094CE000094CE0000B6
:1002C00094CE000094CE000094CE000094CE0000A6
:1002D00094CE000094CE000094CE000094CE000096
:1002E00094CE000094CE000094CE000094CE000086
:1002F00094CE000094CE000094CE000094CE000076
:1003000094CE000094CE000094CE000094CE000065
:1003100094CE000094CE000094CE000094CE000055
:1003200094CE000094CE000094CE000094CE000045
:1003300094CE000094CE000094CE000094CE000035
:1003400094CE000094CE000094CE000094CE000025
:1003500094CE000094CE000094CE000094CE000015
:1003600094CE000094CE000094CE000094CE000005
:1003700094CE000094CE000094CE000094CE0000F5
:1003800094CB000094CE000094CE000094CE0000E8
:1003900094CE000094CE000094CE000094CE0000D5
:1003A00094CE000094CE000094CE000094CE0000C5
:1003B00094CE000094CE000094CE000094CE0000B5
:1003C00094CE000094CE000094CE000094CE0000A5
:100800002F002200007F240000018800000000006B
:100810000C000700C0622100010020001100070049
:10082000000020000000E000020032000000020092
:10083000000000007C150200000000000040DA000B
:100840000000FE004440A900C00520000000E000B8
:100850000300320000002000A00188004440A800EE
:100860000000060091018800800078000000EB0085
:1008700015003700E280400032A0B4009101BA00B8
:10088000E280400032A0B4009102BA00E280400051
:1008900032A0B4000002EB00472BDE00F507B200E7
:1008A000602CE10004003A000059EB008301E900EC
:1008B000FDFF3E00040037006128E1000100320026
:1008C0000082EB00040007001101BA000200E00002
:1008D000E8FF3A00000006003159BA008301E90040
:1008E0000C0032002159BA008301E90008003200EF
:1008F0000400E00003003A00E280400032A0B400AF
:10090000F5FF370011D9BA008301E900FAFF3A0078
:100910008100E800E180400032A0B4000000060041
:100920007C0F0400000000006410040000000000C0
:10093000A01004000000000094100400000000005B
:100940001C0E040000000000380E0400000000002F
:100950008001EB000200370061F079008301E800BC
:10096000828F5100FCFF3A000000060012010000D7
:10097000100100000200000000080000D804000080
:100980000A00000002000000010200000301000054
:100990000902000043000000020100000080000086
:1009A00064090000040000000001000002020000D1
:1009B00001000000052400000010000001040000F8
:1009C00024020000020500002406000000010000CF
:1009D000052400000101000001070000058100005E
:1009E000030A0000004000000904000001000000AC
:1009F000020A0000000000000007000005020000DD
:100A000002400000004000000705000082020000D4
:100A100040000000400000004E4F0000454D000027
:100A2000530000000A00FA00100798002107980000
:100A300032079800430798001E009000005E88006F
:100A40002E009000105E88003E009000205E88001E
:100A50004E009000305E88000000EB00B02488005B
:100A60009424A8009424A9009EC0A9000000EB00D3
:100A700060248800F00F200070248800F00F200010
:100A8000502488000000EB00302588000000EB00B7
:100A900040258800008020004800DE00C024880037
:100AA00000082000302488008804A8000000EB0023
:100AB000405E88000000EB00505E88000000EB0004
:100AC000605E88000000EB00000F78000E00370029
:100AD0001E0078004200DD008080E800E0BC2000BD
:100AE000808040000000EB00800878001E00780045
:100AF000C200DD00E0BC2000808040000000EB0070
:100B0000800878001E0FE8001E007800EF0F5000EC
:100B1000EFFF36008000EB000000EB00F103070060
:100B20008000EB000000EB00F9030700D00020007C
:100B3000502588000000EB00706088000040EB004A
:100B400012ECB7000000EB00806088000040EB0072
:100B500013ECB70080C0B30000E8B700808120002C
:100B60001040880080C8B30001E8B7000040EB00E7
:100B700004E8B700008220003040880000C4B300C1
:100B800005E8B7000080FA00000006000000FA0047
:100B9000010037009404A80094C4BF0061406000C5
:100BA0000004E000FBFF320094C4BF000044B20028
:100BB0000004E000FCFF3A00CD42A9000080FA00EA
:100BC000000006000000FA008AC4BF006140600017
:100BD0000004E0000400320036000700100020008E
:100BE000502488002C0037008AC4BF006240600097
:100BF0000004E0000400320029000700200020006B
:100C000050248800240037008AC4BF000042B2008C
:100C10000004E0000300320000022000502488009D
:100C20001D0037008AC4BF00704060000004E0006F
:100C30000300320000012000502488001600370015
:100C40008AC4BF0001C8B300014060000004E00096
:100C50000300320000082000502488000E003700F6
:100C60008AC4BF00644060000004E0000600320057
:100C70004000200050248800070037006F00070064
:100C800080002000502488008AC4BF0068406000B3
:100C90000004E000F9FF3A000080FA0000000600BE
:100CA0000000FA00F00F2000702488000080FA0095
:100CB000000006000200FA00CDC2BF0061406000E3
:100CC00080407800CDC2BF006140600000C0680075
:100CD0006140600061416000D12C200091407800AB
:100CE000E0CFB30000C0600002407000CDE2B7006A
:100CF0000000EB0070608800800020005024880015
:100D00000000EB00806088000040EB0012ECB700B0
:100D10000040EB0013ECB7008AC4BF0068406000DD
:100D20000004E000F4FF3A000000EB0050258800CA
:100D30000000EB00602588000000EB0070258800B3
:100D40000000EB00802588000000EB009025880063
:100D50000000EB00A02588000000EB00B025880013
:100D60000000EB00C02588000000EB00D0258800C3
:100D70000000EB00E02588000000EB00F025880073
:100D80000000EB00002688000000EB001026880021
:100D90000000EB00202688000000EB0030268800D1
:100DA0000000EB00402688000000EB00B024880023
:100DB000F00F200050248800F00F200070248800DD
:100DC0000000EB00000F7800080037001E007800DC
:100DD000C200DD0000802000808040000040EB0069
:100DE000904098001E007800640F40001E007800BC
:100DF000E50F5000F5FF3600D00020005025880098
:100E000080C0B30000E8B700808120001040880057
:100E100080C8B30001E8B7000040EB0004E8B70069
:100E2000008220003040880000C4B30005E8B7000D
:100E300094A4A9000080FA00000006000200FA0055
:100E4000CDC2BF000080FB004200DE0061406000B8
:100E500080407800CDC2BF000080FB004200DE0071
:100E60006140600000C06800614060006140600057
:100E70004201DD00D12C200091407800B0CFB300BA
:100E800000C0600002407000CDE2B70090248000F6
:100E9000BAEBB700BACBBF000080FB004300DE0016
:100EA0000080FB004200DD00800078000080200010
:100EB00000804000E05D8800BACBBF000034A00095
:100EC0000080FB004300DE000080FB004200DD00EC
:100ED000800078000080200000804000F05D8800E5
:100EE000E05D8000104090008080FB00C003200087
:100EF00080806000010F7800400220009E00780092
:100F0000808F50000C003200400320009E007800CB
:100F1000808F5000040032001E007800E40F500063
:100F20000300320005003700060007000300370009
:100F3000C002070001003700A60207000080FA0087
:100F4000000006000800FA00F15D800080C0B300D8
:100F500090409800E05D8000100090001040780004
:100F60008080FB0000062000808060003107980030
:100F700000022000BE009000808F5000230032004D
:100F800000042000BE009000808F50002500320039
:100F90003E0090000000E000010032002700370012
:100FA000E05D800010009000104078000080FB00A1
:100FB0006300600020079800AE009000E18F5000B1
:100FC0000A0032002E009000E20F50000A003200AA
:100FD000AE0090000100E00001003200090037007F
:100FE000E05D80003700070015003700E05D8000FD
:100FF0007001070012003700E05D8000B1010700BA
:101000000F003700FD0207000D003700505E800022
:101010000000E0000A003200505E80000000010085
:1010200007003700605E80000000E000040032002E
:10103000505E80000000010001003700EF02070051
:10104000E15D800080C0B30080487800E05D8000F2
:1010500010079800E05D80001000900010407800BC
:101060000004E0000F003500E05D800010009000FB
:1010700066004000104078000004E00006003A00DE
:10108000E05D800010009000670040001040780094
:101090000004E0000300320081CCB300014F78006F
:1010A0000200370080C8B300004F78001E4078006F
:1010B0009E0090009040980094A4A9000080FA003F
:1010C000000006000A00FA00200798002E00900099
:1010D00090009000110798001E0090000000E800AA
:1010E000104078000080FB00400798004E00900000
:1010F000E50F500042003200CE009000E58F500016
:101100000A003C004E009000E10F50001F0032002A
:10111000CE009000E38F50002B0032004E00900074
:101120000000E0000B0032001F013700CE009000ED
:10113000E88F5000FB0032004E009000E90F500095
:1011400000013200CE009000E68F500043003200D4
:1011500015013700F05D8000900090007060800005
:1011600080487800F05D8000100090008000E8006A
:10117000706080004800DE0080487800F05D8000EC
:10118000210020008F020700080137001E00900098
:101190000080E80010407800E14F500008003A005D
:1011A00071608000D0FF2F000080600070608800B8
:1011B000F05D80008000EB0082020700FB0037003A
:1011C0008E020700F90037001E0090000080E80042
:1011D00010407800E14F500007003A007060800036
:1011E0000010A00070608800F05D80008000EB00BF
:1011F00074020700ED00370080020700EB003700A3
:101200001E00900063004000104078000004E000E1
:1012100010003A001E0090000080E80010407800A6
:101220000004E0000B0035001E0090000080E80084
:101230001040780013ECB700F05D80008000EB00F8
:1012400060020700C1E120000000EB00250207005A
:10125000D600370069020700D40037001E00900056
:1012600063004000104078000080FB0030079800C9
:101270003E009000E20F50001F003200BE009000C0
:10128000E38F50006F0032003E009000E10F5000ED
:10129000010032009D003700005E8000A0608800E1
:1012A000005E8000104078000080FB00B060880085
:1012B0001E00900067004000104078000004E0002D
:1012C00093003A001E0090006600400090407800B5
:1012D000A06080001040780080CF50008C0031006A
:1012E0001E00900066004000104078000080FB0067
:1012F000B0608800860037001E0090000080E80083
:1013000090407800005E800071004000104078003E
:1013100080CF50000100390038020700105E8000C5
:10132000A0608800A06080000080E8001040780085
:101330008080FB00A06080006300400010407800C7
:101340000080FB004800DD0000804000B0608800A5
:101350000000EB00000F780010003700A160800053
:10136000B060800000804000A0608800A060800025
:101370000080E800104078008080FB00A0608000C2
:1013800063004000104078000080FB004800DD0052
:1013900000804000B06088001E0FE8001E00900032
:1013A0000080E800104078000080FB009E0F500095
:1013B000EAFF3C001E00900067004000904078006B
:1013C000A0608000630040001040780080CF500093
:1013D000100039001E009000670040009040780027
:1013E000A0608000630040001040780080CF500073
:1013F00047003A001E0090006600400090407800D0
:10140000A06080000080E8001040780080CF50008D
:101410003F0031001E009000660040001040780040
:101420008080FB001E0090006700400010407800A4
:101430000080FB004800DD0000804000B0608800B4
:10144000330037001E0090000080E8001040780054
:101450008080FB00305E8000808F500001003500EE
:10146000E6010700205E8000A0608800A060800088
:10147000104078000080FB00B06088000000EB00A6
:10148000000F780009003700A1608000B060800084
:1014900000804000A0608800A060800010407800BC
:1014A0000080FB00B06088001E0FE8001E00900066
:1014B0000080E800104078000080FB009E0F500084
:1014C000F1FF3C001E0090006700400010407800D3
:1014D0000004E0000E003A001E009000660040008C
:1014E00090407800A06080001040780080CF5000CD
:1014F000070031001E009000660040001040780098
:101500000080FB00B060880001003700BB010700CD
:10151000D701070081E320000000EB007101070004
:1015200022003700F05D8000900090008060800015
:1015300080487800F05D800011002000A1010700C4
:101540001A0037001E0090000080E800104078006C
:10155000E14F500012003E001E0090000080E800A5
:10156000104078000080FB00806088008060800070
:101570000000E0000400320000C2B30012ECB7002B
:10158000350207000200370000C1B30012ECB700BB
:10159000F05D80008000EB008A0107000300370047
:1015A0009601070001003700940107000080FA004F
:1015B000000006000600FA00100798001E009000C8
:1015C00090009000010F78001E00E80010407800A5
:1015D0000080FB00200798002E0090000000E00033
:1015E0000A003200AE0090000100E0003200350039
:1015F0002E009000EA0F500011003200AE00900063
:10160000EB8F50001D0032002B003700F05D800092
:10161000900090000040EB0080487800F05D800072
:10162000100090008000E8000040EB008048780047
:10163000F05D800021002000620107001F003700DC
:101640009E0078006480400010407800E14F500018
:1016500008003E00F05D8000900090000040EB002C
:1016600080487800F05D80001100200055010700DF
:101670001200370061010700100037009E0078005B
:101680006480400010407800E14F500008003E00A8
:101690001E80E800104078000004E00004003A00DA
:1016A000F05D80008000EB0046010700030037007A
:1016B0005201070001003700500107000080FA00C6
:1016C000000006000A00FA00300798003E00900073
:1016D00090009000210798002E0090000000E80084
:1016E000104078000080FB00400798004E009000FA
:1016F000E10F500051003200CE009000E38F500007
:10170000800032004E0090000000E0000100320036
:10171000AD003700F05D8000900090000040EB00CD
:1017200080487800F05D8000100090008000E800A4
:101730000040EB00804878002E00900064004000DC
:10174000104078006F406000304798002E009000F5
:1017500064004000104078000080FB004700DE007D
:10176000204798003E4090000080FB0000004000B1
:10177000800078002E4090000080FB000080400038
:101780004200DD008000780000802000008F4000D3
:101790001E00780090409000B0CFB30080C0600081
:1017A0001E007800114098001E0078001040900044
:1017B0000004E00004003200F05D80009000900022
:1017C00010C0B300804878003E4090000080FB00CD
:1017D00000004000800078002E4090000080FB0058
:1017E000008040004200DD00800078000080200082
:1017F000008F40001E00780090409000B0CFB300F2
:1018000080C060001E007800114098001E00780023
:10181000104090000004E00004003200F05D800001
:101820009000900010C0B30080487800F05D800008
:1018300021002000E3000700640037002E00900024
:1018400064004000104078006F406000304798000E
:101850002E00900064004000104078000080FB00E3
:101860004700DE00204798003E4090000080FB00CB
:1018700000004000800078002E4090000080FB00B7
:10188000008040004200DD008000780000802000E1
:10189000008F40001E00780090409000B0CFB30051
:1018A00080C060001E007800114098002E4090001B
:1018B0000004E000060032001E0078009040900016
:1018C00000C4B30080C070001E0078001140980072
:1018D0002E4090000004E00006003A001E00780050
:1018E00090409000F0CBB30080C060001E007800F4
:1018F00011409800F05D80008000EB00B10007000F
:10190000320037002E009000640040001040780044
:101910006F406000304798002E0090006400400047
:10192000104078000080FB004700DE002047980050
:101930003E4090000080FB000000400080007800E6
:101940002E4090000080FB00008040004200DD003F
:101950008000780000802000008F40001E0078008A
:1019600010409000804078000124A0001E00780004
:10197000114098003E4090000080FB0000004000B5
:10198000800078002E4090000080FB000080400026
:101990004200DD008000780000802000008F4000C1
:1019A0001E00780010409000804078000124A000C4
:1019B0001E00780011409800F05D80008000EB0070
:1019C00080000700010037008C0007000080FA004B
:1019D000000006000000FA00BACBBF000080FB0048
:1019E0004400DE000080FB006F006000C200DD00EC
:1019F000E0BC200000804000100078000000E00003
:101A00000A003200BACBBF000080FB004400DE00B9
:101A10000080FB006F006000C200DD00E0BC200021
:101A20000080400010007800000001000080FA00F3
:101A3000000006000000FA00BACBBF000080FB00E7
:101A40004400DE000080FB006F0060004200DD000B
:101A50008080E800E0BC200000804000100078009A
:101A60000000E0000B003200BACBBF000080FB009A
:101A70004400DE000080FB006F0060004200DD00DB
:101A80008080E800E0BC200000804000100078006A
:101A9000000001000080FA00000006000200FA00C9
:101AA000000F78001E007800405E88000080FA0079
:101AB000000006000200FA00000F78001E00780007
:101AC000505E88000080FA00000006000200FA0064
:101AD000000F78001E007800605E88000080FA0029
:101AE000000006000400FA00000F780011079800BB
:101AF0001E007800C200DD00E0BC20000080400035
:101B00009E009000010878000080FA0000000600A6
:101B10000400FA00000F7800110798001E007800FA
:101B20004200DD008080E800E0BC20000080400032
:101B30009E009000010878000080FA000000060076
:101B40000200FA00000F78001E007800904090001C
:101B500000C4B30000C0680002C4B300824060004B
:101B600080C8B30000C07000804078001E0078007C
:101B7000114098000080FA00000006000200FA0000
:101B8000000F78009E0078000040EB00804878004D
:101B90001E0078009040900000C4B30000C06800B0
:101BA00002C4B3008240600080C8B30000C070006F
:101BB000804078001E007800114098000080FA00F4
:101BC000000006000400FA00000F780011079800DA
:101BD0001E0090008040780000C0EB0080C06000D4
:101BE0001E007800014878009E00780080CCB30089
:101BF000904098000080FA00000006000000FA0003
:101C000080C0B30000E8B70080C0B30000E8B700B0
:101C100040C8B30005E8B70040C8B30001E8B7000A
:101C200040C8B30005E8B70040C8B30001E8B700FA
:101C30000080FA00000006000000FA0013CCBF008C
:101C40000004E0000500350013CCBF000080FB005D
:101C5000B024880000C0EB0013ECB7008000EB005C
:101C60000000EB009FFF07000080FA000000060064
:101C70000600FA00B06080000000E0001C003200A6
:101C8000B0608000200798002E009000E80F500000
:101C90000200360083002000230798002E009000E9
:101CA000000F78000000EB00100798000C003700D0
:101CB000F05D8000900090001E00900000814000C8
:101CC000A16080001E00900000804000104078005D
:101CD000004978001E0090000000E80010079800FE
:101CE0001E0090009E0F5000F1FF390005003700E4
:101CF0000000EB00000F78008000EB000000EB001C
:101D000078FF0700F15D80001E00780080487800B1
:101D1000F25D8000F05D80009040900000C4B30050
:101D200000C0680003C4B3008340600080C8B300F3
:101D300000C0700010419800A16080001E00780073
:101D400000804000A0608800B06080001E0050004D
:101D5000B06088000080FA00000006000200FA006F
:101D60008EC0BF000044B2000004E000200032003A
:101D70008AC4BF00614060000004E0000600320039
:101D8000CCFB07001000200050248800F00F20003A
:101D9000000F7800180037008AC4BF006840600058
:101DA0000004E0001100320090248000BAEBB7007C
:101DB000BACBBF000080FB004400DE000080FB00C7
:101DC0006F0060000000E000060032001BFC07000E
:101DD0008000200050248800F00F2000000F7800C1
:101DE0000500370080002000502488008EC0A90024
:101DF0000000EB00000F78001E0078000080FA0061
:101E0000000006000000FA0000202C001100200055
:101E1000D05C8800E15C88000000EB00F05C88008A
:101E20000000EB00005D880080C0B300A2EBB700AB
:101E3000A40BA900A42BA900C0F720001DFF0700D8
:101E40000000EB00905D8800905D8000805D880060
:101E50000080FA00000006000000FA008000EB009D
:101E6000100020001FFF07008000EB002000200072
:101E70001CFF07008000EB002000200024FF07006B
:101E80005001200060258800D001200070258800C6
:101E90000040EB000CE8B700E0B420007040880080
:101EA00080C4B3000DE8B70000C4B30010E8B70069
:101EB000E0AC20009040880080C8B30011E8B70073
:101EC0000040EB0014E8B700E0B02000B04088000C
:101ED00080C4B30015E8B700C0F72000F5FE070086
:101EE00000812000A05D880040812000B05D880056
:101EF0000080FA00000006000600FA00CDC2BF0014
:101F00000080FB000000D10061406000804078004C
:101F1000CDC2BF000080FB000000D1006140600026
:101F200000C0680061406000614060000041400006
:101F3000D12C200091407800D0CFB30000C06000C9
:101F400002407000CDE2B700E05D8000900090009C
:101F5000110798001E009000104078008080FB0060
:101F6000300620008080600010022000808F50002A
:101F7000010032004B0037001E0090000000E80016
:101F8000104078000080FB00200798002E00900091
:101F9000E40F50000A003C00AE009000E28F5000B9
:101FA0001C003D002E0090000000E00011003200F7
:101FB000AE009000E18F5000120032003700370071
:101FC00010022000AE009000808F500017003200F9
:101FD00020022000AE009000808F500024003200CC
:101FE00000022000AE009000808F50000B003200F5
:101FF0002A003700F05D80008000EB00F1FE070052
:1020000029003700F05D80008000EB00EDFE070046
:1020100025003700F9FE07002300370041062100A4
:102020000000EB00BAFE07001F0037001E00900002
:1020300066004000100F7800A00020009E0F1000E6
:1020400002003600A0002000000F7800F05D800044
:1020500010009000A1B920001E0178003CFA070092
:102060009E007800F05D8000D6FE07000E0037006D
:102070001E0090000080E80010007800205D8800BD
:10208000010A21000000EB0096FE0700F05D8000D1
:102090008000EB00CBFE070003003700D7FE0700EF
:1020A00001003700D5FE07000080FA00000006009E
:1020B0000000FA008000EB000000EB0089FE070042
:1020C0000080FA00000006000000FA00E05D8000D9
:1020D00010009000A1B9200009000900B058780054
:1020E000A000B1008000EB000000EB0088FE0700BC
:1020F000410921000000EB007AFE0700F05D80003E
:102100008000EB00AFFE0700E15D800080C0B300FF
:1021100080487800E15D800080C8B300904098005E
:102120000080FA00000006000000FA008000EB00CA
:102130000000EB006BFE07000080FA0000000600C4
:102140000000FA008000EB000000EB0065FE0700D5
:102150000080FA00000006000000FA00C05D800068
:102160000000E00003003200C05D80000000E900D4
:10217000C05D88000080FA00000006000200FA003E
:102180000A0037009EC0BF000044B2000004E00017
:1021900006003A00F1FE07000004E00003003200F0
:1021A0000000EB00000F780006003700A05D800003
:1021B000104090000004E000F2FF35001000200005
:1021C000000F78001E0078000080FA000000060072
:1021D0000200FA000A0037009EC0BF000044B200AF
:1021E0000004E00006003A00DCFE07000004E00006
:1021F000030032000000EB00000F780006003700FB
:10220000B05D8000104090000004E000F2FF350057
:1022100010002000000F78001E0078000080FA00F7
:10222000000006000600FA00000F78002147980021
:102230000A0037009EC0BF000044B2000004E00066
:1022400006003A00C5FE07000004E000030032006B
:10225000F00F20002007980018003700B05D8000C4
:10226000104090000004E000F2FF3500B05D8000F7
:102270009E00780011009800B05D8000AE41900093
:1022800003487800B25D8000B05D8000904090000F
:1022900000C4B30000C0680003C4B3008340600002
:1022A00080C8B30000C0700010419800ABFE07006A
:1022B0002E4090000080FB00200798002E00900028
:1022C0000080FA00000006000200FA00A05D800015
:1022D000104090008000EB00010F78000004E00047
:1022E0000200350010002000000F78001E0078006A
:1022F0000080FA00000006000200FA00B05D8000D5
:10230000104090008000EB00010F78000004E00016
:102310000200350010002000000F78001E00780039
:102320000080FA00000006000400FA00000F7800A8
:10233000214798000040EB00A7EBB700A05D8000AC
:10234000104090000004E0002E003500A05D8000E9
:10235000904078002E40900080CF50000300310064
:10236000A05D800090407800214798000040EB007D
:10237000A7EBB7000C003700A7CBBF000080FB0025
:102380001E014000A7CBBF008080FB00E0AC200016
:10239000008040001040780000497800A7CBBF00C3
:1023A0000040E800A7EBB70071BA20009140780028
:1023B0002E40900080CF5000EFFF39009EC0BF003C
:1023C0000044B2000004E00001003A0063FE070090
:1023D000A15D800000C4B30080487800A25D800049
:1023E000A05D80009040900000C4B30000C0680071
:1023F00003C4B3008340600080C8B30000C0700015
:1024000010419800A7CBBF000080FB000080FA00BD
:10241000000006000000FA0098CBBF000004E000B6
:1024200007003A0001C4B30080B52000BEFF0700DA
:1024300098EBB700E3F907000040EB0099EBB70019
:102440000080FA00000006000200FA00000F780089
:10245000F0FF070098CBBF000004E000FCFF320053
:1024600099CBBF008080FB0080B520000080400039
:10247000904078001E0078000148780098CBBF009B
:102480000040E90098EBB70099CBBF000040E8009E
:1024900099EBB700100020000080FA000000060051
:1024A0000800FA000040EB0006EAB7000000370021
:1024B000C4F90700D7FF070000A02000E2FF0700D3
:1024C0000004E000FAFF320001A0200091407800F3
:1024D00010CCB30080CF5000F5FF3A003CFF07005E
:1024E00010CFB3000EEBB70040C0B3000FEBB70046
:1024F00060C0B30010EBB70031C0B300E0B0200003
:1025000048FF0700B0C4B30007EAB7000000370077
:10251000ACF907002EFF070007CABF000EEBB7009B
:1025200011C0B300E0B020003EFF07000040EB0008
:10253000004F780080A02000C3FF070008CABF003A
:102540001E4F400090A02000BFFF070009CABF0037
:102550001E4F4000A0A02000BBFF07000ACABF001A
:102560001E4F4000B0A02000B7FF07000BCABF00FD
:102570001E4F4000C0A02000B3FF07000CCABF00E0
:102580001E4F400008CABF000080FB009001880079
:102590000CCABF00E14F5000180036000000EB00ED
:1025A000100798000E0037001E0090008000780091
:1025B000E0A0200000804000A3FF07001E00900064
:1025C000E800400060A0200000804000104078003B
:1025D0001E4F40001E0090000000E8001007980009
:1025E0000CCABF000080FB000000E90080007800FA
:1025F0001E009000808F5000EBFF3E00D0A0200016
:1026000091FF07000DCABF001E4F40001E04E000EE
:1026100003003200E0C4B30007EAB700BCFF370094
:1026200008CABF000080FB00010020001050880095
:10263000215088001050800021508000C808DD0023
:102640000080FD00804078000040EB0010508800C2
:102650002150880009CABF000081FB000300200050
:10266000105080002150800002004000838048000C
:1026700010508800215088001050800021508000A8
:10268000C808DD000080FD00804078000040EB00BD
:1026900010508800215088000ACABF000081FB004A
:1026A00003002000105080002150800002004000F4
:1026B0008380480010508800215088000BCABF005A
:1026C0000080FB00300798003E009000E20F5000B1
:1026D0000B003200F00F2000BE009000808F5000F1
:1026E000090032003E009000E10F5000010032006E
:1026F0001800370010C0B30006EAB7001700370013
:102700001B000700150037009404A9000080EB00AF
:1027100020079800080037000080EB0010079800A1
:102720001E0090000000E900100798001E009000B5
:10273000E10F4000FAFF3A002E0090000000E9008F
:10274000200798002E009000E10F4000F2FF3A00B1
:102750000000FE0050C5B30007EAB7006ACCBF0016
:102760000004E0006AFF32000080FA00000006006A
:102770000C00FA000040EB00004F78001050800081
:1027800021508000E00F5000E08F58000C003A000C
:1027900040C0B3000EEAB7000040EB000FEAB700FC
:1027A00040C0B30010EAB7000040EB0011EAB700E8
:1027B0000040EB0012EAB7000040EB0013EAB7005C
:1027C0001250800023508000F0FF21000100200003
:1027D000800F5100818F59000B003C001250800087
:1027E00023508000F03F200001002000800F5100A6
:1027F000818F59000400340000C5B30007EAB70018
:1028000010C0B300004F78001250800023508000A9
:10281000F07F2A0021002000800F5100818F590095
:102820000400340000C5B30007EAB70010C0B300CD
:10283000004F78001E04E000AD003A0006CABF0059
:102840000004E0001600320020042400003B880051
:102850001050800021508000800078000080EB0044
:102860008008BB004E00900050052000303B8800DF
:10287000A00A2000303B880061E7A80000000000AB
:102880000000000061C7BF0001C8B3000140600044
:102890000004E000FBFF3A000040EB0006EAB7004E
:1028A0001050800021508000100798001000240074
:1028B000003B88000040EB00604798002D00370087
:1028C0006E4090000080FB00E800400060A0200007
:1028D00000804000104078000080FB002007980036
:1028E000AE0090001E0090000188BB006E4090007A
:1028F0000040E800604798006E4090000080FB00B8
:10290000E800400060A020000080400010407800F7
:102910000080FB00200798006E4090000040E80017
:10292000604798006E4090000080FB00E800400087
:1029300060A0200000804000104078000080FB0074
:10294000C800DD002E0090000100700020079800F4
:102950006E4090000040E80060479800AE00900094
:102960001E0090000108BB001E0090000080E800DF
:10297000100798006E4090008080FB000CCABF00DA
:102980000080FB000000E900808F5000CCFF350084
:102990005E00900050052000303B8800A00A200017
:1029A000303B880061E7A800000000000000000044
:1029B00061C7BF0001C8B300014060000004E0002F
:1029C000FBFF3A0061C7A900105080002150800031
:1029D00010079800B0C4B30007EAB7000040EB004E
:1029E000604798003B0037001E0090001080BA003E
:1029F00020079800AE009000F00F200000806000DB
:102A0000200798006E4090000080FB00E800400026
:102A100060A0200000804000104078008080FB0013
:102A20002E009000808F50000200320060C5B3007D
:102A300007EAB7006E4090000040E8006047980049
:102A40001E0090001000BA00200798002E00900091
:102A5000004178006E4090000080FB00E8004000DC
:102A600060A020000080400010407800804F51009E
:102A70000200320060C5B30007EAB7006E40900064
:102A80000040E800604798002E0090004880DE007B
:102A9000004178006E4090000080FB00E80040009C
:102AA00060A020000080400010407800804F51005E
:102AB0000200320060C5B30007EAB7006E40900024
:102AC0000040E800604798001E0090000080E80089
:102AD000100798006E4090008080FB000CCABF0079
:102AE0000080FB000000E900808F5000BEFF350031
:102AF0000080FA00000006000200FA000080EB00EF
:102B000060198800C8E2A8006F20A800CCC2A90004
:102B1000C8C2A90080382100000F78001E0078008C
:102B20000000E900000F78001E007800E10F40006F
:102B3000FAFF3A000000EB00000F78000A003700AF
:102B4000CAC2BF0001C8B300014060000004E00039
:102B50000200320001002200014001001E00780046
:102B60000000E800000F78001E007800F30F50000E
:102B7000F3FF34006F20A900C8C2A80003000700BB
:102B80000000EB000080FA00000006000000FA00E0
:102B900016000700C902A900C922A900C942A9005C
:102BA000CD42A800CD02A900CD22A80043002000FC
:102BB00082C12000814C2800604B280099F7070053
:102BC000F2F707008FFC0700CD22A900FDF70700F0
:102BD00012CCBF00FF4F5000FCFF3600CD22A800F2
:102BE0002FFE07000080FA00000006000000FA0037
:102BF0004440A8000000EB00A00188000000EB00AA
:102C0000203A88000000EB00900188000080EB0073
:102C10006019880020002000501988000080EB0017
:102C2000401688000080EB00801688000080EB00D2
:102C3000C01688000080EB00001788000080EB00C1
:102C4000401788000080EB00801788004227A90009
:102C50000080FA00000006006A0C0000020000007C
:102C60000200000000000000000A0000CE0000008A
:102C70000000000000200000020000000000000032
:102C80006C0C0000020000000200000000000000C8
:102C9000580B00006200000000000000CE0A000097
:102CA0008A00000000000000180C00005200000024
:102CB0000200000004030900042A0300440061002C
:102CC000006E000067006500007200006F00750074
:102CD0000073000020005000007200006F007400BC
:102CE000006F000074007900007000006500730040
:102CF0000012030043004400004300002000540081
:102D00000065000073007400001203003000300002
:102D10000030000030003000003000003000310092
:102D20000000000000080000000200000000000099
:102D3000BA0B00005E000000000000000000000070
:102D40000000FE00FFFFFF00FFFFFF00FFFFFF008E
:102D5000FFFFFF00FFFFFF00FFFFFF00FFFFFF007F
:102D6000FFFFFF00FFFFFF00FFFFFF00FFFFFF006F
:102D7000FFFFFF00FFFFFF00FFFFFF00FFFFFF005F
:102D8000FFFFFF00FFFFFF00FFFFFF00FFFFFF004F
:103FE000FFFFFF00FFFFFF00FFFFFF0006040000D0
:103FF0000000FA00E5FA07000080FA000000060061
:104000006F6A2200007F2400000188000000000089
:104010000C00070040F12B000100200011000700F8
:10402000000020000000E00002003200000002005A
:1040300000000000CACA0200000000000040DA00D0
:104040000000FE004440A900205920000000E000CC
:104050000300320000002000A00188004440A800B6
:104060000000060091018800800078000000EB004D
:1040700015003700E280400032A0B4009101BA0080
:10408000E280400032A0B4009102BA00E280400019
:1040900032A0B4000002EB00472BDE00F507B200AF
:1040A000602CE10004003A000059EB008301E900B4
:1040B000FDFF3E00040037006128E10001003200EE
:1040C0000082EB00040007001101BA000200E000CA
:1040D000E8FF3A00000006003159BA008301E90008
:1040E0000C0032002159BA008301E90008003200B7
:1040F0000400E00003003A00E280400032A0B40077
:10410000F5FF370011D9BA008301E900FAFF3A0040
:104110008100E800E180400032A0B4000000060009
:1041200046CD04000000000058CD0400000000004F
:104130006ECD04000000000082CD040000000000ED
:1041400096CD040000000000ACCD0400000000008B
:10415000C2CD040000000000D0CD0400000000002B
:10416000548C040000000000D4880400000000000B
:10417000C8880400000000001E8904000000000040
:104180000A89040000000000FE880400000000000E
:10419000F088040000000000E48804000000000033
:1041A000548904000000000032890400000000006F
:1041B000468C04000000000072760400000000003D
:1041C000D276040000000000F47504000000000036
:1041D000A275040000000000387804000000000010
:1041E000467704000000000024780400000000006E
:1041F000DE790400000000001877040000000000D1
:10420000706A040000000000386A0400000000002A
:10421000A86A040000000000E26A04000000000038
:10422000D66A040000000000EC6D040000000000ED
:104230008C6B040000000000E46D0400000000002E
:10424000046F040000000000066B04000000000082
:1042500028AE04000000000042AE04000000000090
:1042600018AE0400000000000EAE040000000000C4
:1042700080AE04000000000074AE040000000000E6
:10428000A4AE04000000000098AE0400000000008E
:1042900068AE0400000000008CAE040000000000C6
:1042A0005CAE040000000000ACAF040000000000A1
:1042B000E8AE040000000000E4AF040000000000CD
:1042C000B0AE04000000000068C20400000000005E
:1042D00028C2040000000000A8C204000000000082
:1042E00002C2040000000000F6C10400000000004B
:1042F0000CC304000000000018C30400000000000C
:1043000024C304000000000030C3040000000000CB
:10431000F4C204000000000000C30400000000001C
:10432000E8C204000000000082C304000000000096
:10433000BCC40400000000003CC3040000000000F6
:1043400026BC0400000000003EBC04000000000089
:104350000CBC040000000000B4BC0400000000001D
:1043600056BC040000000000BA6F0400000000000A
:104370001EBE04000000000068CE04000000000023
:1043800060CE0400000000005ACE040000000000CF
:10439000A85B0400000000005EA404000000000010
:1043A00044A504000000000036A504000000000041
:1043B000A0A504000000000092A504000000000079
:1043C0002288040000000000528804000000000061
:1043D000889FBE008A9FBE00010578000100E000B2
:1043E0000400350008003C000000E000200032001E
:1043F0000500370060001000E080180002003B005C
:1044000001F02C001A0037000004BE006011B80053
:104410006B0920000982CF00020039000882CF001A
:104420000441B000694252000E00320008003B0017
:1044300082817100610164008904D1000884D30085
:104440008B05E8000442E800F9FF3A000500370058
:104450000804440089844C008B05E9000442E9000B
:10446000FBFF3A000B0107000AF0A70001F0A000D3
:104470004F05BE004F04BE0000000600F4FF2F00F1
:104480002A0137001400200028013700889FBE0051
:104490008A9FBE008C1F78003F0107004601330051
:1044A00003866C006450E1002E0032006420E100BD
:1044B000330032006150E1002F0032006120E10042
:1044C0003100320085855500EB07B000090020005F
:1044D00008042000050037000804440089844C00CB
:1044E0000A0031000603430087834B00000153009C
:1044F00081815B00F8FF33000203BE000800A000CA
:104500000804440089844C00F6FF3900C639DD00F8
:104510008301730001003200130020008904D100E0
:104520000884D3000998A300050032000800A70002
:104530000300A0008904D1000884D3008B05E800A3
:104540008904D1000884D3000001EB000281D2006D
:10455000D000070001F0A1000CF0A70001F0A000BE
:104560001E0137006420E100200132000801BE0076
:104570000200BE00F7FF37006120E1001B0132009E
:104580006000B800F3FF37000000200001F82700AA
:10459000F0FF370003F0A200889FBE008A9FBE0094
:1045A0008C1F7800FC000700030133006450E10019
:1045B0004F0032006420E1005200320003826C00A0
:1045C00007003B000905D0000306D000820F54000D
:1045D0000C065D00020039000200320089017800FB
:1045E000030678008582550004003D000003FD00AD
:1045F0008103FD008502EA008B854200840F720072
:1046000002003B0060001000E08018006011B8005C
:104610000005EB007A28E1000A0039000600780066
:10462000C75DDD00F707B200878075002D003700F9
:10463000828171000A017800610560008180D100EB
:104640000080D3008502E900F9FF3B00060440002A
:104650008784480002003B0060041400E0841C00D2
:104660000988A300070032008A81710082817100ED
:10467000610164008904D1000884D3008B05E8003F
:10468000170037000978A30013003A000B00E00080
:10469000130034008B05E9000804440089844C00B1
:1046A0000A4474000978A3000D003A000B00E000F2
:1046B000070034008B05E9000804440089844C009D
:1046C00001003A000B0020000978A300F7FF320038
:1046D0000001EB0002003700828171000A017800BE
:1046E0006C0007000CF0A70001F0A000BB00370031
:1046F0006420E10002003A00838F6C00BB003300AD
:104700000801BE000200BE00B4003700889FBE0052
:104710008A9FBE008C1F78009F000700A600330010
:1047200003866C006450E100240032006420E10044
:10473000270032006150E100220032006120E100D8
:10474000210032008B854200EB07B1000134B80034
:10475000003AB8000804420089844A00013AB800CF
:104760000030B8008880400009014A00040033008E
:104770000000400081804800020149008B05E900EB
:10478000C909DD0083017000010032001300200020
:10479000C814DE004814DD004709DE001200B20034
:1047A000C808DE00088470003A00070001F0A1008C
:1047B0000CF0A70001F0A000880037006120E100A4
:1047C0008A0032000801BE000200BE00F7FF370079
:1047D0006150E100FCFF3A00840037000001BE0098
:1047E000850007000470A70003F0A10003F8A300F0
:1047F00013003A006509B1001000320009003500CD
:104800006928E100020035000100280000000500D1
:1048100000004000818048008502E900FCFF3A006A
:1048200000000600F88F4200050035008100D1002D
:104830000080D3008502E800FCFF3A00000006007B
:104840008000EB00000005006022B8000602200096
:104850000000D0008180D2000482D2008582D20084
:104860000000A0000202520083825A0003003100BF
:104870000202420083824A000000A1000603E90010
:10488000F3FF3A0000000600EFFF07000400BE003F
:104890000000060081002000618055000B003D00F3
:1048A0000B00200061FE2F000100E1001D0034001C
:1048B00082817100610164008904D1000884D30001
:1048C0000000E800FAFF3A00710020006100640077
:1048D000030070000200600009003200610444001F
:1048E000E0844C000988A500050032008B05E80033
:1048F0006808E10002003A008904D1000884D3006E
:10490000F20F20000258E10005003D00C75DDD0008
:10491000F907B200898075000800780000000600E1
:104920000BF827008B00780000000500889FBE0070
:104930008A9FBE00841F7800170007004F00780090
:1049400011003300F0FF2F00838F6C0006003B0046
:10495000040565000A00A7000800370009F0A6005A
:104960001000200008003700820F5400838F5C0085
:10497000030039001000200001003E00000020006C
:1049800009F0A7000000EA004F05BE004F04BE007A
:104990000000E000000006000004BE001600070052
:1049A0000003BE000405BE000200BE0012000700A6
:1049B000844F7500000006000200BE006450E10054
:1049C000050036006420E100020036000968A300FB
:1049D00001003A000800BE000160A0004F06780008
:1049E0004F05BE004F04BE0000000600F0FF2F0080
:1049F000F1FF2700F9FF3700C70ADE00F107B20018
:104A0000F50FB20008003200E1CF42000200320090
:104A10000170A00024000500810F70000100320029
:104A20000408050044000500810F700002003A00F0
:104A3000140005008502E9000000400081C0480024
:104A4000FCFF3B000170A000240005008001EB008A
:104A50000200370061F079008301E800828F510085
:104A6000FCFF3A00000006003E00000008200000A5
:104A7000080000001B5B0000440000001B5B0000FE
:104A800000440000001B00005B430000001B00000E
:104A90005B3200004B0D00000043000000000000EE
:104AA0001B5B00003244000000410000555800002C
:104AB00031200000736500006C6500006374000025
:104AC00065640000004100005558000032200000DD
:104AD000736500006C65000063740000656400008D
:104AE00000570000617200006E6900006E670000F0
:104AF0003A2000006E6F0000207600006F6C00000E
:104B00007461000067650000206F00006E200000E7
:104B100056700000756C00006C750000702000007D
:104B2000706900006E000000203D000020000000C1
:104B30005652000045470000207400006F6F0000CF
:104B4000206C00006F7700002C20000069730000CB
:104B5000207400006865000072650000206100009C
:104B600020730000686F0000727400003F000000B6
:104B70002E2000003C0000002E200000000D000050
:104B80000A280000002900003E00000042750000D5
:104B9000732000005069000072610000746500001D
:104BA000207600003400000046690000726D0000AD
:104BB000776100007265000020760000362E00004C
:104BC000302D00006133000020000000202800008C
:104BD00032340000464A00003235000036470000FB
:104BE0004231000030360000200000004133000058
:104BF0000041000035000000554E00004B00000051
:104C00002900000043460000473000003A20000021
:104C100000560000707500003D350000562C000065
:104C20002000000056700000753D00003356000063
:104C3000332C000020000000612F0000412F0000F5
:104C400040200000636F00006E740000726F00006F
:104C50006C73000020410000555800003120000016
:104C6000706900006E000000612F0000412F0000FD
:104C700040200000636F00006E740000726F00003F
:104C80006C730000204100005558000032200000E5
:104C9000706900006E00000049090000004F00002C
:104CA0000900000048090000004C00000900000055
:104CB000456E000074650000722000007261000003
:104CC00077200000766100006C7500006520000010
:104CD000666F000072200000425200004700000092
:104CE00057610000726E0000696E0000673A0000B4
:104CF000206100006C7200006561000064790000B2
:104D000020610000207600006F6C000074610000DC
:104D100067650000206F00006E20000056700000E4
:104D2000756C00006C750000702000007069000058
:104D30006E000000536500006C65000063740000A5
:104D40002056000070750000207300006F75000091
:104D5000726300006500000020310000292000007F
:104D60004E6F00006E650000206F00007220000092
:104D70006578000074650000726E0000616C0000D0
:104D80000020000032290000204F00006E62000069
:104D90006F61000072640000203300005633000091
:104DA00020560000726500006700000020330000FC
:104DB000292000004F6E0000626F00006172000049
:104DC0006420000035560000205600007265000087
:104DD000670000006F6E00002D6200006F61000030
:104DE0007264000020700000756C00006C7500009B
:104DF00070200000766F00006C7400006167000096
:104E0000652000006469000073610000626C0000AE
:104E1000656400000033000056330000206F00007E
:104E20006E2D0000626F00006172000064200000BF
:104E3000707500006C6C000075700000207600003A
:104E40006F6C000074610000676500002065000061
:104E50006E610000626C00006564000000350000B7
:104E6000562000006F6E00002D6200006F61000090
:104E70007264000020700000756C00006C7500000A
:104E800070200000766F00006C7400006167000005
:104E900065200000656E0000616200006C65000026
:104EA00064000000005E0000BCE20000613F000002
:104EB000DD830000C29C00007E200000A3FD0000F6
:104EC0001F4100009DC30000217F0000FCA20000E4
:104ED000401E00005F010000E3BD00003E600000D6
:104EE00082DC0000237D00009FC10000421C000006
:104EF000FEA00000E1BF00005D03000080DE0000B6
:104F00003C620000BEE00000025C0000DF810000A7
:104F1000633D00007C220000C09E00001D43000095
:104F2000A1FF000046180000FAA400002779000045
:104F30009BC5000084DA000038660000E5BB000075
:104F400059070000DB85000067390000BAE4000063
:104F50000658000019470000A5FB00007826000055
:104F6000C49A0000653B0000D9870000045A000085
:104F7000B8E60000A7F900001B450000C698000035
:104F80007A240000F8A60000441A000099C7000027
:104F9000257B00003A64000086D800005B05000015
:104FA000E7B900008CD20000306E0000EDB30000C5
:104FB000510F00004E100000F2AC00002F710000F5
:104FC00093CD0000114F0000ADF30000702E0000E3
:104FD000CC920000D38D00006F310000B2EC0000D5
:104FE0000E500000AFF10000134D0000CE90000005
:104FF000722C00006D330000D18F00000C520000B5
:10500000B0EE0000326C00008ED00000530D0000A6
:10501000EFB10000F0AE00004C12000091CF000094
:105020002D730000CA94000076280000ABF5000044
:105030001749000008560000B4EA00006937000074
:10504000D58B000057090000EBB500003668000062
:105050008AD4000095CB000029770000F4AA000054
:1050600048160000E9B70000550B000088D6000084
:10507000346A00002B75000097C900004A14000034
:10508000F6A80000742A0000C8960000154B000026
:10509000A9F70000B6E800000A540000D789000014
:1050A0006B3500004C4500005400000049460000EC
:1050B00000540000484500004E000000454C000030
:1050C00053450000004700004F5400004F0000000F
:1050D000474F0000535500004200000052450000B9
:1050E00054550000524E000000520000454D000093
:1050F00000500000524900004E54000000490000DA
:105100004E50000055540000004600004F52000071
:10511000005400004F0000004E45000058540000AD
:1051200000520000454100004400000044410000DE
:10513000544100000053000054410000525400004C
:10514000520000005354000041520000540000007F
:10515000535400004F500000520000005354000010
:105160004F50000000530000454E00004400000076
:10517000524500004345000049560000450000002C
:10518000434C00004B00000044410000540000006C
:105190004249000054520000454100004400000014
:1051A00041440000430000004155000058500000F9
:1051B000494E000000500000535500000050000010
:1051C000554C00004C5500005000000044450000C4
:1051D0004C410000590000004155000058000000FB
:1051E00046520000455100000044000055540000A4
:1051F000590000004D410000435200004F000000E4
:10520000454E00004400000000520000554E0000D2
:10521000004C0000495300005400000045580000B5
:10522000495400000044000045420000554700007A
:10523000004E0000455700000000000044690000D7
:10524000736300006F6E00006E6500006374000001
:10525000206100006E790000206400006576000087
:105260006963000065730000004300006F6E00007A
:105270006E650000637400002028000041440000B7
:1052800043200000746F0000202B0000332E00002C
:105290003356000029000000454500005052000030
:1052A0004F4D000000530000434C0000005300002D
:1052B000444100000057000050000000414300003E
:1052C0004B000000567500007362000000350000BE
:1052D00056300000205600005055000000330000FA
:1052E000563300002056000050550000004D0000CD
:1052F0004F440000452C000020560000524500009D
:10530000472C0000206100006E6400002055000062
:1053100053420000204C0000454400007320000070
:10532000736800006F7500006C640000206200006C
:10533000652000006F6E00002100000000290000C1
:10534000002000005700000020520000004E000026
:105350006F77000020750000736900006E67000021
:10536000206F00006E2D0000626F0000617200006F
:105370006420000045450000505200004F4D0000E1
:105380002049000032430000206900006E740000D4
:10539000657200006661000063650000004F000058
:1053A0006E2D0000626F000061720000642000003A
:1053B00045450000505200004F4D0000207700008E
:1053C000726900007465000020700000726F0000B8
:1053D00074650000637400002064000069730000BD
:1053E000616200006C65000064000000493200004A
:1053F0004331000000000000120100001001000015
:105400000200000000080000D804000000FB0000BB
:105410000200000001020000030100000902000078
:105420004300000002010000008000006409000049
:105430000400000000010000020200000100000062
:1054400005240000001000000104000024020000F8
:1054500002050000240600000001000005240000F1
:10546000010100000107000005810000030A00009F
:10547000004000000904000001000000020A0000D2
:1054800000000000000700000502000002400000CC
:1054900000400000070500008202000040000000FC
:1054A000400000003062000000300000303000009A
:1054B0002C000000303000000030000031320000CD
:1054C0003334000035360000373800003941000021
:1054D00042430000444500004630000078000000D0
:1054E000436F0000756C0000646E000027740000BC
:1054F000206B0000656500007020000075700000E2
:10550000000000005350000049310000000000007E
:105510003A200000000000002E000000315700007B
:105520003031000000000000314100004C53000009
:105530000042000050760000330000000808000020
:1055400008080000080000000000000020480000DB
:105550007A0000000000000042420000494F0000B5
:1055600031000000524100005731000000000000EF
:105570004E4F0000454D00005300000000000000A9
:105580002900000000000000000000002800FA00D0
:105590000000EB00600F98000000EB00100889008D
:1055A0000000EB0000088900000881002007980037
:1055B0000000EB00100798000000EB00000F7800DF
:1055C0000000EB00A02789000000EB0050079800C6
:1055D0000000EB00200889000000EB004007980065
:1055E0000000EB00000F9800140037000000EB00F3
:1055F000600798000B0037000E089000EE00900046
:105600004500DD00810040006010220080804000E5
:105610000040EB00804878006E0090000000E80039
:10562000600798006E009000FF0F5000F2FF3400FA
:105630000E0890000000E800000F98000E0890008F
:10564000E40F5000E9FF34000000EB00300D89004A
:10565000A1278100E00220000088B900610220003B
:105660008080400080C6210000804000809E0200B3
:1056700000000000D1278100002020000080600091
:105680000000E0000400320071002000C05920003A
:105690005CC902000000000040532A00809E020006
:1056A0000000000031043700300D81000000E000F0
:1056B00064003200300D81000000E900300D8900E7
:1056C0000000EB00600798001E0037000208810010
:1056D000300D8100EE0090004500DD0081004000AB
:1056E00060102200008040009040780000002200FE
:1056F0000000410001487800300D8100EE0090006C
:105700004500DD0081004000601022000080400064
:105710001040780084A20200000000000008810010
:105720000000E800000889006E0090000000E8001A
:105730006007980001088100F00F200000806000E1
:1057400000088900300D8100EE0090004500DD006A
:10575000810040006010220000804000104078006E
:105760000004E000D9FF3A000000EB00300D890092
:1057700034003700A0DE2100104078006440600053
:105780000004E0002E003200A1278100E00220008A
:105790000088B900FA00400080C621000080400067
:1057A00010007800000001000000E000240032003A
:1057B000A1278100E00220000088B90061022000DA
:1057C0008080400080C6210000804000809E020052
:1057D0000000000040532A00809E020000000000EC
:1057E0001108810000088100808F500014003200F1
:1057F00010088100600798000D003700EE0090004F
:1058000000002200008040001040780084A20200C6
:1058100000000000EE009000F00F2000008060000B
:10582000600798006E0090000000E8006007980094
:10583000EE00900000088100808F5000EFFF3A00DA
:10584000D3C2BF0004A30200000000000004E00077
:10585000C8FF32004EA30200000000000004E00078
:105860000300320056A3020000000000BF0337000F
:1058700010A3020000000000604F98006E489000E6
:105880000080FB006101B90002179800131798000F
:10589000F0072000010020000E1190009E119000E2
:1058A000800F5100818F59003C033E000E10900084
:1058B0009E109000006001002D033700E2023700C7
:1058C0003E01370035033700D8003700F9023700B2
:1058D0005301370031033700770037002F033700BB
:1058E0000F0337002D0337002C0337000C0337005C
:1058F000FE013700290337005A013700270337001C
:10590000260337002503370024033700230337001D
:105910002203370021033700200337001F0337001D
:105920001E033700020137001C0337001B0337003A
:105930001A0337001903370018033700170337001D
:10594000160337001503370014033700130337001D
:105950001203370011033700100337000F0337001D
:105960000E0337000D0337000C0337000B0337001D
:105970000A0337000903370008033700070337001D
:10598000060337000503370004033700030337001D
:10599000020337000103370000033700FF0237001E
:1059A000FE023700FD023700FC023700FB02370021
:1059B000FA023700F9023700F8023700F702370021
:1059C000F6023700F5023700F4023700F302370021
:1059D000F2023700F1023700F0023700EF02370021
:1059E000EE023700ED023700EC023700EB02370021
:1059F000EA023700E9023700E8023700E702370021
:105A0000E6023700E5023700E4023700E302370020
:105A1000E2023700E1023700E0023700DF02370020
:105A2000DE023700DD023700DC023700DB02370020
:105A3000DA023700D9023700D8023700D702370020
:105A4000D6023700D5023700D4023700D302370020
:105A5000D2023700D1023700D0023700CF02370020
:105A6000CE023700CD023700CC023700CB02370020
:105A7000CA023700C9023700C8023700C702370020
:105A8000C6023700C5023700C4023700C302370020
:105A9000C2023700C1023700C0023700BF02370020
:105AA000BE023700BD023700BC023700BB02370020
:105AB000BA0237005D003700110881002E00900007
:105AC000810F500055003200010881002E00900027
:105AD000810F500010003A00000881008000E900AA
:105AE000F00F20000080600000088900010881009C
:105AF00000002200808040000040EB0080487800D9
:105B0000010881002107980060532A00809E02004E
:105B100000000000150337000000EB00000F9800A4
:105B20002E0090008000E900F00F2000008060004F
:105B300020079800A0532A00809E02000000000069
:105B40002E01900062079800210037006E0190003E
:105B50006E0090008000E8000000220000804000FD
:105B600090407800000022000000410001487800C9
:105B7000EE009000000022000080400010407800FD
:105B80000004E00007003200EE0090000000220058
:105B9000008040001040780084A202000000000055
:105BA0000300370000C2B30084A20200000000001E
:105BB0000E0890000000E800000F98006E009000B2
:105BC0008000E800F00F200000806000600798006F
:105BD000EE00900000088100808F5000DBFF3A004B
:105BE000000881008000E900F00F200000806000C4
:105BF00000088900E0532A00809E02000000000097
:105C00000E08900018A102000000000010542A00A5
:105C1000809E020000000000D402370070C0B30074
:105C200084A2020000000000D002370001088100B9
:105C30002E009000810F5000390032000000EB0070
:105C4000000F9800AE019000630798002100370014
:105C50006E0190006E0090008000E80000002200BD
:105C600000804000904078000000220000004100C9
:105C700001487800EE009000000022000080400003
:105C8000104078000004E00007003200EE009000B1
:105C900000002200008040001040780084A2020032
:105CA000000000000300370000C2B30084A202001D
:105CB000000000000E0890000000E800000F9800AF
:105CC0006E0090008000E800F00F2000008060006F
:105CD00060079800EE00900000088100808F50005F
:105CE000DBFF3A00000881008000E900F00F20008F
:105CF0000080600000088900E0532A00809E0200B6
:105D0000000000000E08900018A102000000000032
:105D100010542A00809E0200000000009302370009
:105D200070C0B30084A20200000000008F023700A0
:105D300010A3020000000000604F9800EE489000A1
:105D4000B0C5B30080CF500088023A0010A3020013
:105D500000000000604F98006E4890000080FB003B
:105D6000700F980020042000FE089000808F5000E3
:105D7000DE003200200420007E099000800F5100D8
:105D800005003C0010042000FE099000808F5100A7
:105D9000340032007502370030042000FE08900005
:105DA000808F50001E003200400420007E099000C9
:105DB000800F5100010032006C0237004E0090004D
:105DC000E40F500005003400A8B1020000000000FC
:105DD0000000EB00400798006402370011088100C2
:105DE0002E009000810F5000090032002E0090001C
:105DF0008000E900F00F200000806000200798007C
:105E0000A0532A00809E02000000000057023700C5
:105E100070C0B30084A202000000000053023700EB
:105E2000010881002E009000810F5000090032000F
:105E30002E0090008000E800F00F2000008060003D
:105E40002007980030542A00809E020000000000C5
:105E50004602370070C0B30084A2020000000000B8
:105E6000420237000000EB00000F780010088100AC
:105E70000000E90080007800F00F20000080600042
:105E8000600798008D003700EE00900000002200AF
:105E900000804000104078000004E00082003A00DA
:105EA0006E0090008000E900F00F2000808060000C
:105EB0000000220000804000104078000004E00054
:105EC000790032001E0FE8001E0090009E0F1000A7
:105ED000750036001E0090000000E80010079800D2
:105EE0001108810000088100808F500014003200EA
:105EF0000A00370001088100000022008080400075
:105F00000040EB0080487800000881008000E90034
:105F1000F00F200000806000000889000108810067
:105F200010088100808F5000F2FF3A0001088100C4
:105F300000002200808040000040EB008048780094
:105F40006E0090008000E900F00F200000806000EB
:105F5000000F9800110037008E089000000022000A
:105F600000804000104078000004E00006003A0085
:105F70000E0890008000E800F00F20000080600014
:105F800050079800090037000E0890008000E900D3
:105F9000F00F200000806000000F98008E08900035
:105FA00000088100808F5000EBFF3A0070542A00F7
:105FB000809E020000000000A1278100E002200076
:105FC0000088B900610220008080400080C6210066
:105FD00000804000809E020000000000D127810068
:105FE00000202000008060000000E000040032007B
:105FF00071002000C05920005CC9020000000000B0
:1060000040532A00809E020000000000DE01900044
:10601000030F9800180037008E089000000022003F
:10602000008040001040780084A2020000000000C0
:10603000020881008E0890000000220000804000CD
:1060400090407800000022000000410001487800E4
:10605000000881008000E800F00F20000080600050
:10606000000889000E0890008000E800F00F200072
:1060700000806000000F98008E0890006E00900075
:10608000808F5000E4FF3A000108810000002200E8
:10609000808040000040EB008048780000088100CC
:1060A00020079800090037006E0090008000E9008A
:1060B000F00F20000080600060079800EE00900064
:1060C00000088100808F50006FFF3A00EE009000C2
:1060D00000088100808F5000A4013A0070C0B30016
:1060E00084A2020000000000A00137000000EB00C5
:1060F000000F7800100881000000E900800078009F
:10610000F00F200000806000600798008E003700CC
:10611000EE00900000002200008040001040780057
:106120000004E00083003A006E0090008000E90067
:10613000F00F2000808060000000220000804000FE
:10614000104078000004E0007A0032001E0FE800E2
:106150001E0090000000E9009E0F500075003A00FC
:106160001E0090000000E90010079800110881004F
:1061700000088100808F5000140032000A003700B0
:106180000108810000002200808040000040EB00F8
:1061900080487800000881008000E900F00F2000AE
:1061A000008060000008890001088100100881005B
:1061B000808F5000F2FF3A000108810000002200A9
:1061C000808040000040EB00804878006E00900026
:1061D0008000E900F00F200000806000000F9800B0
:1061E000110037008E08900000002200008040005F
:1061F000104078000004E00006003A000E0890000D
:106200008000E800F00F2000008060005007980038
:10621000090037000E0890008000E900F00F200010
:1062200000806000000F98008E0890000008810038
:10623000808F5000EBFF3A0070542A00809E0200CD
:1062400000000000A1278100E00220000088B900C2
:10625000610220008080400080C621000080400054
:10626000809E020000000000D12781000020200055
:10627000008060000000E000040032007100200097
:10628000C05920005CC902000000000040532A00F1
:10629000809E020000000000DE009000010F9800C8
:1062A000180037008E089000000022000080400097
:1062B0001040780084A20200000000000208810063
:1062C0008E0890000000220000804000904078007E
:1062D0000000220000004100014878000008810011
:1062E0008000E800F00F20000080600000088900B6
:1062F0000E0890008000E800F00F20000080600091
:10630000000F98008E0890006E009000808F500063
:10631000E4FF3A0001088100000022008080400074
:106320000040EB00804878000208810022079800B6
:10633000090037006E0090008000E900F00F200097
:106340000080600060079800EE0090000008810067
:10635000808F50006EFF3A00EE0090000008810030
:10636000808F500001013A001E009000E10F5000A4
:1063700031003A0070542A00809E020000000000A4
:10638000A1278100E00220000088B90061022000FE
:106390008080400080C6210000804000809E020076
:1063A00000000000D1278100002020000080600054
:1063B0000000E0000400320071002000C0592000FD
:1063C0005CC902000000000040532A00809E0200C9
:1063D000000000000A0037000108810000002200D0
:1063E000808040000040EB00804878000008810079
:1063F0008000E900F00F20000080600000088900A4
:106400000108810010088100808F5000F2FF3A00DF
:106410000108810000002200808040000040EB0065
:106420008048780003088100230798000000EB00F3
:1064300010079800CD00370070C0B30084A202009E
:1064400000000000C9003700110881002E009000F4
:10645000810F500013003200110881002E009000BF
:106460000100500080007800F00F200000806000E4
:10647000000F9800E0532A00809E020000000000F8
:106480000E08900018A102000000000010542A001D
:10649000809E020000000000100881002007980084
:1064A000B200370070C0B30084A2020000000000F8
:1064B000AE003700010881002E009000810F5000CF
:1064C00013003200010881002E009000008050006F
:1064D00080007800F00F200000806000000F98001E
:1064E000E0532A00809E0200000000000E08900089
:1064F00018A1020000000000D0542A00809E020073
:106500000000000001088100210798009700370073
:1065100070C0B30084A202000000000093003700A6
:1065200010002000600F98000000EB00100798009A
:106530000108810000002200808040000040EB0044
:1065400080487800000881008000E800F00F2000FB
:10655000008060000008890002088100220798007E
:10656000F0542A00AC9E0200000000007F003700BB
:106570004E0090000000E800400798004E00900098
:10658000F40F500079003A000AA902000000000050
:106590000000EB00400798007400370000088100FD
:1065A0008000E800F00F200080806000100881006B
:1065B000808F50006A0032006E489000FF4F5000FC
:1065C00067003600EE489000E0C7B30080CF50006F
:1065D00063003E00010881002E009000808F500073
:1065E00015003A006E48900084A2020000000000EE
:1065F000010881006E4990000000220000804000E8
:1066000002487800000881008000E800F00F2000B8
:10661000008060000008890001088100000022005D
:10662000808040000040EB00804878000308810033
:10663000230798004D003700010881002E009000CC
:106640000080500080007800F00F20000080600083
:10665000000F9800E0532A00809E02000000000016
:106660000E08900018A1020000000000D0542A007B
:10667000809E020000000000000881006007980072
:106680001D0037006E0090000001E800EE00900051
:1066900000002200008040009040780000002200AE
:1066A0000000410001487800EE0090000000220048
:1066B00000804000104078000004E0000900320033
:1066C000EE009000000022000080400010407800A2
:1066D00084A202000000000000552A00809E0200F3
:1066E000000000006E0090008000E900F00F200024
:1066F00000806000600798006E0190002E009000FE
:106700008000E900F00F200000806000800F510041
:10671000DCFF3A006E48900084A2020000000000F6
:10672000AE0090006E499000000022000080400002
:10673000024878002E0090008000E800F00F200052
:106740000080600020079800000881008000E800B9
:10675000F00F20000080600000088900030037006F
:1067600070C0B30084A20200000000006E08900018
:106770000000E000CCFB320000088100400F9800D0
:1067800010088100300F98000000EB00600F9800A7
:106790000000EB00500F98000000EB00200889007B
:1067A000D127810000202000008060000000E00070
:1067B0001F05320028580200000000005100200090
:1067C000305A2000E6C9020000000000100020003E
:1067D000500F9800160537001108810000002200B4
:1067E0000080400010407800604F98006E48900094
:1067F0000080FB006101B900221798003317980050
:10680000E0072000010020002E119000BE11900032
:10681000800F5100818F5900D9043E002E10900046
:10682000BE10900000600100D7043700D404370088
:10683000D3043700D2043700D1043700D004370026
:10684000CF043700CE043700CD043700CC04370026
:10685000CD043700CA043700C9043700CA04370022
:10686000C7043700C6043700C5043700C404370026
:10687000C3043700C2043700C1043700C004370026
:10688000BF043700BE043700BD043700BC04370026
:10689000BB043700BA043700B9043700B804370026
:1068A000B7043700B6043700B70437009404370044
:1068B000D40237004101370046013700EB013700B1
:1068C000D9013700AE043700AD023700AC04370001
:1068D000AB043700AC043700AB043700400437008A
:1068E00059043700240437004D0337004C033700A8
:1068F0004B0337004A03370049033700480337008A
:106900004703370046033700450337004403370089
:106910009B0437009A043700F4013700DF0037008A
:10692000970437003F003700540137004601370015
:106930009304370065003700B80137009004370032
:106940008F0437008E0437008D0437008C04370025
:106950008B043700720037007B0037008804370053
:106960008704370086043700A3003700840437000B
:1069700083043700D20137008104370080043700D8
:106980007F043700530137007D0437007C04370053
:106990007B043700FE023700040437000E03370083
:1069A000380437001B04370075043700190137001D
:1069B000270037003A0037008A013700B50037005A
:1069C000290037002B0037006D043700180037000E
:1069D0006B04370048003700680037001A003700A2
:1069E000670437001C00370071003700640437006B
:1069F00087033700AE0137006104370060043700B9
:106A000017003700650137005D0437005C0437006C
:106A10005B043700E7023700BB003700F70237009E
:106A2000D9003700FCC902000000000056043700FE
:106A3000C5070700A02781000000E00052043200D3
:106A4000F9070700500437007A0607004E043700A4
:106A50006B0907004C043700450907004A0437005A
:106A6000B108070048043700049B02000000000042
:106A700045043700A02781000000E00005003A002F
:106A8000D1012000305D2000E6C9020000000000B6
:106A90003D0437006C990200000000003A04370002
:106AA000A0DE2100104078000000A1000010A1002D
:106AB000A1DE21008048780061012000805A20007A
:106AC000E6C90200000000002F043700A0DE21000C
:106AD000104078000000A0000010A100A1DE2100FD
:106AE0008048780051012000E05B2000E6C90200E8
:106AF0000000000024043700A0DE210010407800D0
:106B00000000A1000010A000A1DE21008048780054
:106B100050552A00AC9E0200000000001A04370005
:106B2000A0DE2100104078000000A0000010A000AE
:106B3000A1DE21008048780030562A00AC9E020079
:106B40000000000010043700A0DE21001040780093
:106B50000030A000A1DE210080487800C1012000A3
:106B6000B07E20005CC9020000000000F0542A0042
:106B7000AC9E02000000000003043700A0DE2100EC
:106B8000104078000030A100A1DE2100804878008C
:106B9000B1012000007D20005CC90200000000005F
:106BA000F0542A00AC9E020000000000F6033700FB
:106BB000A02781000000E00005003A00D10120007C
:106BC000305D2000E6C9020000000000EE0337003F
:106BD000E282A900E082A90051012000005F2000AC
:106BE0005CC9020000000000F0542A00AC9E0200C4
:106BF00000000000E4033700A02781000000E0004F
:106C000005003A00D1012000305D2000E6C90200F5
:106C100000000000DC033700A0DE210010407800F7
:106C2000704060000004E00004003A0021022000EF
:106C300050E82000E6C9020000000000E082A80041
:106C4000E282A90041012000506020005CC90200DE
:106C500000000000F0542A00AC9E0200000000007A
:106C600021E3A80050C0B3008EC502000000000060
:106C700080007800F0042000808F500003003E0068
:106C800010572A00AC9E02000000000021E3A9007A
:106C9000BD03370033090700BB033700100881002C
:106CA0008000E800F00F20000080600010088900DC
:106CB000D0050700E8030700600798006E00900009
:106CC0007AA102000000000040592A00809E0200C4
:106CD000000000006E00900018A1020000000000FB
:106CE00040592A00809E0200000000006E009000C3
:106CF000E09E020000000000F0542A00AC9E02005A
:106D000000000000A0033700100881008000E800A8
:106D1000F00F20000080600010088900B505070012
:106D2000CD030700600798006E0090000080FB0014
:106D300020C7020000000000600798006E0090006D
:106D40007AA102000000000040592A00809E020043
:106D5000000000006E00900018A10200000000007A
:106D600040592A00809E0200000000006E00900042
:106D7000E09E020000000000F0542A00AC9E0200D9
:106D80000000000080033700A02781000000E00021
:106D900005003A0011C0B30010C0B300B4B802003F
:106DA0000000000078033700A1012000906120005E
:106DB000E6C9020000000000730337005100200004
:106DC00030632000E6C90200000000000000FE0061
:106DD0006D0337008CCA0200000000000000E000D4
:106DE00069033200A100200080632000E6C9020090
:106DF0000000000040062000BEC6020000000000A7
:106E000000C502000000000081BF2A00014001000F
:106E10005D033700350507000000E800000F98000B
:106E200002003700A09C0200000000000E08900045
:106E30000000E900000F98000E0890000000E0003C
:106E4000F8FF3A0050033700280507000000E8006B
:106E5000000F980002003700509C02000000000064
:106E60000E0890000000E900000F98000E08900046
:106E70000000E000F8FF3A00430337001B0507005D
:106E80000000E800000F98000B00370061012000AF
:106E9000206420005CC9020000000000F09C020099
:106EA000000000006A9E020000000000F0542A006A
:106EB000AC9E0200000000000E0890000000E900F7
:106EC000000F98000E0890000000E000EFFF3A006D
:106ED0002D033700A02781000000E00005003A00E4
:106EE000D1012000305D2000E6C902000000000052
:106EF00025033700C922A900CB22A80021E3A8005E
:106F000020002000BEC60200000000000040EB0090
:106F10008EC502000000000080007800001B2000E9
:106F2000808F50000F00360020C0B3008EC50200D5
:106F30000000000080007800702B2000808F50003F
:106F40000800360011012000806520005CC90200A5
:106F500000000000F0542A00AC9E02000000000077
:106F60000C003700C922A900CB22A90080592A00B1
:106F7000AC9E02000000000021012000906620006D
:106F80005CC9020000000000F0542A00AC9E020020
:106F90000000000021E3A900FB023700A0278100C8
:106FA0000000E00005003A00D1012000305D200023
:106FB000E6C9020000000000F3023700C922A90060
:106FC000CB22A90021012000906620005CC90200AC
:106FD00000000000F0542A00AC9E020000000000F7
:106FE000E9023700F1002000A03920005CC902004E
:106FF00000000000A8C502000000000011002000F1
:10700000903A20005CC9020000000000F0542A0001
:10701000AC9E020000000000DB023700BAC502008F
:1070200000000000D8023700B0040700000F9800ED
:1070300061002000706820005CC9020000000000B0
:107040000E089000BAA002000000000021002000FD
:10705000D0682000E6C90200000000000E08900081
:10706000EAC6020000000000C70237009F040700C4
:10707000000F980061002000706820005CC90200C9
:10708000000000000E089000BAA0020000000000FE
:107090002100200090EC2000E6C902000000000062
:1070A0000E089000BEC6020000000000B6023700C5
:1070B000D02781000090A000D0278900B2023700BD
:1070C000A02781000000E00005003A00D101200067
:1070D000305D2000E6C9020000000000AA0237006F
:1070E000629D020000000000A7023700100020008F
:1070F0002008890010002000600798001000370069
:10710000110881006E00900080804000F00F200088
:1071100080806000000022000080400090407800E5
:10712000E0C3B30080CF500002003A000000EB0043
:10713000200889006E0090000000E80060079800B9
:10714000110881006E00900080804000F00F200048
:107150008080600000002200008040001040780025
:107160000004E000E6FF3A00EE009000200220005C
:10717000808F500002003400100020002008890099
:10718000200881000000E0007F023A001008810022
:107190008000E800F00F20000080600010088900E7
:1071A000AD0207006007980011088100F00F200071
:1071B0008080600000002200008040009040780045
:1071C000D0C3B30080CF500040003A006E00900062
:1071D0000000E0003A0034006E009000E50F50001F
:1071E00037003C00100881008000E800F00F20000C
:1071F00000806000100889006E0090000000E90027
:10720000600798000000EB00000F98000B003700AB
:107210006E0090008E0890004500DD008100400067
:1072200060102200808040000040EB008048780021
:107230000E0890000000E800000F98000E08900073
:10724000FF0F5000F2FF34000000EB00000F980029
:1072500013003700EE0190000E0A90001108810023
:107260000000220000804000104178004518DD0039
:107270008400400060102200008040000248780036
:107280000E0890000000E800000F98001008810030
:107290008000E800F00F20000080600010088900E6
:1072A000110881000000220000804000904078001A
:1072B000E0C3B30080CF5000E6FF3A00320237004F
:1072C00010002000200889002F0237006E00900077
:1072D0000000E0001B003A000000EB00000F9800E7
:1072E000140037000E0890000040E80018A10200CA
:1072F00000000000805B2A00809E02000000000069
:107300000E0890004500DD0080007800601022002B
:1073100000804000809E02000000000040532A00D0
:10732000AC9E0200000000000E0890000000E80083
:10733000000F98000E089000E40F5000E9FF3400A1
:10734000110237006E0090000000E00009003400D8
:107350006E009000E50F500006003C00F0542A003B
:10736000AC9E020000000000EE009000310D89008C
:1073700005023700100020002008890002023700B3
:10738000100881008000E800F00F200000806000FD
:107390001008890030020700200F9800150407002C
:1073A00011088100F00F20008080600000002200A2
:1073B000008040009040780090C2B30080CF500021
:1073C0000D003A00A1278100E00220000088B900EA
:1073D000FC00400080C62100008040009000780042
:1073E0002E08900001000100F0542A00AC9E02001B
:1073F00000000000E4013700100020002008890090
:10740000E101370010002000200889001000200052
:107410006007980010003700110881006E0090008E
:1074200080804000F00F200080806000000022007B
:10743000008040009040780020C2B30080CF500010
:1074400002003A000000EB00200889006E00900066
:107450000000E80060079800110881006E009000AD
:1074600080804000F00F200080806000000022003B
:1074700000804000104078000004E000E6FF3A0081
:10748000200881000000E000BF013A0071002000E8
:10749000F06820005CC902000000000020C2B300B8
:1074A00084A20200000000002200370011088100C1
:1074B000F00F200000806000100889001108810092
:1074C00000002200008040001040780084A20200EA
:1074D0000000000011088100000022000080400030
:1074E000104078000000FB00200F9800A0DE210073
:1074F00010407800684060000004E00004003200A2
:107500002E08900020C7020000000000200F980005
:10751000A1278100E00220000088B900E8004000B7
:1075200080C6210000804000900078002E08900066
:1075300001000100100881000000E8001008890027
:1075400011088100F00F2000808060000000220000
:10755000008040009040780020C2B30080CF5000EF
:10756000D2FF3A0010088100F10F200001006000F6
:107570001008890020C2B30084A2020000000000AD
:10758000F0542A00AC9E0200000000007E0137008B
:10759000A1278100E00220000088B9008000780067
:1075A00080C621000080400010007800000001002B
:1075B00075013700A1278100E00220000088B90092
:1075C0008080E80080C62100008040001000780024
:1075D000000001006C013700A1278100E0022000BB
:1075E0000088B900E400400080C62100008040000F
:1075F000100078000000010063013700A12781001E
:10760000E00220000088B900E600400080C62100AA
:107610000080400010007800000001005A0137008F
:1076200071002000F06820005CC90200000000002A
:1076300089010700200F9800100881000000E90070
:107640001008890011088100F00F20000080600000
:1076500010088900250307000000E800000F9800CB
:1076600045030700300798003E0090000000E0004E
:107670005D0032003E0090008040780090DD2100E7
:10768000014878003E009000E80F500006003400EA
:10769000A0DE2100104078000050A000A1DE2100F3
:1076A0008048780050003700A0DE210010407800AC
:1076B0000050A100A1DE2100804878004A00370078
:1076C0002E08900018C6020000000000A0DE210075
:1076D000104078000042B2000004E00004003A00CC
:1076E00090DD210010407800E84F500009003A007A
:1076F000A0DE2100104078000042B2000004E0004B
:107700000B00320090DD210010407800F04F500057
:1077100007003200B0C3B30084A2020000000000E2
:1077200090DD21001040780018A102000000000048
:10773000A0DE210010407800684060000004E000F6
:10774000040032002E08900020C702000000000054
:10775000200F9800A1278100E00220000088B900D6
:10776000E800400080C621000080400090007800C2
:107770002E08900001000100100F980000C2B30015
:1077800084A2020000000000A0DE2100104078006A
:107790000044B2000004E000130032006100200049
:1077A000606920005CC9020000000000A0DE21002A
:1077B00010407800684060000004E00004003200DF
:1077C0001E08900020C7020000000000100F980063
:1077D0001E08900018C602000000000000C2B3009E
:1077E00084A20200000000000E0890000000E900E2
:1077F000000F98000E0890000000E000B0FF3A0073
:10780000F0542A00AC9E020000000000DE003700A9
:1078100061002000606920005CC9020000000000D7
:10782000B20207000000E800000F9800D202070033
:10783000300798003E0090000000E0004400320055
:107840003E0090008040780090DD210001487800E3
:107850003E009000E80F500006003400A0DE21003A
:10786000104078000050A000A1DE21008048780080
:1078700037003700A0DE2100104078000050A10042
:10788000A1DE21008048780031003700A127810067
:10789000E00220000088B900EA00400080C6210014
:1078A000008040001000780000000100100F9800D8
:1078B000A0DE210010407800684060000004E00075
:1078C000040032001E08900020C7020000000000E3
:1078D000100F98001E08900018C60200000000005B
:1078E000A0DE2100104078000042B2000004E00059
:1078F00004003A0090DD210010407800E84F50006D
:1079000009003A00A0DE2100104078000042B200D9
:107910000004E0000B00320090DD210010407800F0
:10792000F04F500007003200B0C3B30084A2020041
:107930000000000090DD21001040780018A1020036
:107940000000000000C2B30084A20200000000009A
:107950000E0890000000E900000F98000E0890004B
:107960000000E000C9FF3A00F0542A00AC9E02007B
:10797000000000008400370081002000C069200062
:10798000E6C9020000000000A1278100E0022000FB
:107990000088B900EC00400080C621000080400053
:1079A00010007800000001007700370081002000FF
:1079B000406A2000E6C9020000000000A127810003
:1079C000E00220000088B900EE00400080C62100DF
:1079D0000080400010007800000001006A003700BD
:1079E000E1002000C06A2000E6C90200000000009B
:1079F000A1278100E00220000088B900F0004000CB
:107A000080C62100008040001000780000000100C6
:107A10005D003700E1002000A06B2000E6C90200F5
:107A200000000000A1278100E00220000088B900CA
:107A3000F200400080C62100008040001000780065
:107A40000000010050003700C1002000B067200096
:107A50005CC9020000000000A1278100E0022000B4
:107A60000088B900F400400080C62100008040007A
:107A700010007800000001006A9E02000000000073
:107A80004100370019020700000F9800D1002000C4
:107A9000806D20005CC90200000000000E0890000C
:107AA00018C60200000000000E0890000000E80068
:107AB000000F980008003700A1278100E002200095
:107AC0000088B900F600400080C621000080400018
:107AD00010007800000001000E0890000000E9008E
:107AE000000F98000E0890000000E000F2FF3A003E
:107AF000F0542A00AC9E0200000000002200370073
:107B0000FA0107000000E800000F9800A100200023
:107B1000506E20005CC90200000000000D0037001C
:107B2000A1278100E00220000088B900F800400091
:107B300080C6210000804000100078000000010095
:107B40006A9E02000000000000C2B30084A202008E
:107B5000000000000E0890000000E900000F9800EF
:107B60000E0890000000E000EDFF3A000101200047
:107B7000806C2000E6C9020000000000020037000F
:107B80001000200020088900100881008000E80013
:107B9000F00F20000080600010088900200881009C
:107BA0000000E0001C00320051012000F06E2000B7
:107BB0005CC9020000000000BE08900010088100AF
:107BC000808F50000700310010088100804078004D
:107BD0003E08900000C0500018A102000000000004
:107BE0000600370010088100804078003E089000B1
:107BF00000C0500018A10200000000000000EB00CF
:107C00002008890010002000500F9800F0542A002E
:107C1000AC9E0200000000001108810000088100F5
:107C2000808F500002003A0010002000500F980092
:107C30005E0890000000E000E7FA32004E08900075
:107C4000100889004E089000000889000000EB0031
:107C5000600F98007EF637000600FA000000EB0087
:107C6000100798000000EB00000F78001108810059
:107C70001E00900080804000F00F20008080600097
:107C800000002200008040009040780000C3B30054
:107C900080CF500043003400110881001E00900086
:107CA00080804000F00F20008080600000002200F3
:107CB000008040009040780090C3B30080CF500017
:107CC00038003C00110881001E00900080804000B8
:107CD000F00F200080806000000022000080400043
:107CE000104078008000FB0000FD2F00008F400056
:107CF0001E0090000000E8001007980012003700F6
:107D00001E0078006A00B900000F78001108810099
:107D10001E00900080804000F00F200080806000F6
:107D20000000220000804000104078000000FB00AE
:107D30009E00400000FD2F00008F40001E009000BC
:107D40000000E80010079800110881001E00900054
:107D500080804000F00F2000808060000000220042
:107D60000080400090407800F0C2B30080CF500007
:107D700051013400110881001E00900080804000F5
:107D8000F00F200080806000000022000080400092
:107D90009040780090C3B30080CF5000D8FF3400EB
:107DA00045013700110881001E00900080804000CE
:107DB000F00F200080806000000022000080400062
:107DC0009040780000C3B30080CF500035013A00E6
:107DD0001E0090000000E8001007980011088100C4
:107DE0001E00900080804000F00F20008080600026
:107DF00000002200008040009040780020C6B300C0
:107E000080CF50000B003200110881001E0090004E
:107E100080804000F00F2000808060000000220081
:107E2000008040009040780020C4B30080CF500014
:107E30002D003A001E0090000000E8001007980096
:107E4000120037001E00780000004000000F78008C
:107E5000110881001E00900080804000F00F20007B
:107E60008080600000002200008040001040780008
:107E70000000FB009E00400000FD2F00008F40002E
:107E80001E0090000000E800100798001108810013
:107E90001E00900080804000F00F20008080600075
:107EA00000002200008040009040780010C3B30022
:107EB00080CF5000E3FF3200110881001E009000C7
:107EC00080804000F00F20008080600000002200D1
:107ED000008040009040780000C3B30080CF500085
:107EE000D8FF3200F4003700110881001E00900016
:107EF00080804000F00F20008080600000002200A1
:107F0000008040009040780080C7B30080CF5000D0
:107F10000B003200110881001E009000808040009C
:107F2000F00F2000808060000000220000804000F0
:107F30009040780080C5B30080CF50008E003A009A
:107F40001E0090000000E80010079800470037006E
:107F50001E0078004400DD00000F78001108810049
:107F60001E00900080804000F00F200080806000A4
:107F7000000022000080400090407800F0C2B30072
:107F800080CF500018003400110881001E009000BE
:107F900080804000F00F2000808060000000220000
:107FA000008040009040780090C3B30080CF500024
:107FB0000D003C00110881001E00900080804000F0
:107FC000F00F200080806000000022000080400050
:107FD000104078000000FB009E00400000FD2F00D4
:107FE000008F40001E003700110881001E00900025
:107FF00080804000F00F20000081600011088100A7
:108000001E00900080804000F00F20008080600003
:1080100000002200008040009040780000C2B300C1
:1080200080C070000000220000004100014878007C
:10803000110881001E00900080804000F00F200099
:108040008080600000002200008040001040780026
:108050000000FB009E00400090FA2F00008F4000BF
:108060001E0090000000E800100798001108810031
:108070001E00900080804000F00F20008080600093
:10808000000022000080400090407800F0C2B30061
:1080900080CF50000B003400110881001E009000BA
:1080A00080804000F00F20008080600000002200EF
:1080B000008040009040780090C3B30080CF500013
:1080C000A3FF3400110881001E0090008080400052
:1080D000F00F20008080600000002200008040003F
:1080E0009040780000C4B30080CF50000B003400F3
:1080F000110881001E00900080804000F00F2000D9
:1081000080806000000022000080400090407800E5
:1081100060C4B30080CF50008DFF3400110881008F
:108120001E00900080804000F00F200080806000E2
:1081300000002200008040009040780000C6B3009C
:1081400080CF50005C003400110881001E009000B8
:1081500080804000F00F200080806000000022003E
:10816000008040009040780060C6B30080CF50008F
:1081700077FF340050003700110881001E00900086
:1081800080804000F00F200080806000000022000E
:108190000080400090407800F0C2B30080CF5000D3
:1081A00045003400110881001E00900080804000CE
:1081B000F00F20008080600000002200008040005E
:1081C0009040780090C3B30080CF50003A003C004C
:1081D000110881001E00900080804000F00F2000F8
:1081E0008080600000002200008040001040780085
:1081F0008000FB0000FD2F00008F400012003700C0
:108200001E0078006A00B900000F78001108810094
:108210001E00900080804000F00F200080806000F1
:108220000000220000804000104078000000FB00A9
:108230009E00400000FD2F00008F40001E009000B7
:108240000000E80010079800110881001E0090004F
:1082500080804000F00F200080806000000022003D
:108260000080400090407800F0C2B30080CF500002
:1082700011003400110881001E0090008080400031
:10828000F00F20008080600000002200008040008D
:108290009040780090C3B30080CF5000D8FF3400E6
:1082A0000500370010002000200889000000EB00C6
:1082B000200798000A003700110881001E00900076
:1082C000008040001008890011088100F00F200094
:1082D00000806000100889001E00780020079800C8
:1082E0002E0090000080FA00000006000400FA0052
:1082F000100881008000E800F00F200080806000FE
:10830000000022000080400090407800A0C3B3002D
:1083100080CF500013003A00100881000080E80070
:108320001008890011088100F00F20000080600013
:108330001008890048FE0700000F7800100881002F
:108340000000E9001008890011088100F00F2000EA
:1083500000806000100889001E0078001007980057
:108360000200370010002000100798001E00900047
:108370000080FA00000006000400FA0010088100E6
:108380008000E800F00F20008080600000002200E4
:108390000080400090407800B0C3B30080CF500010
:1083A0000F003A00100881008080E800F00F2000E4
:1083B000008060001008890027FE0700000F780089
:1083C000100881008000E900F00F200000806000AC
:1083D000100889001E00780010079800020037007E
:1083E0000000EB00100798001E0090000080FA00CB
:1083F000000006000000FA000500370010088100A8
:108400008000E800F00F2000008060001008890064
:108410001108810000002200008040009040780098
:1084200000C2B30080CF5000F4FF32000080FA0099
:10843000000006000400FA000000EB00000F7800C6
:10844000100881008000E800F00F2000008060002C
:1084500010088900E7FF0700FFFD0700000F780004
:108460001E00E0004D003A000000EB0010079800ED
:10847000130037001E0090000040E80018A1020021
:1084800000000000C05B2A00809E02000000000087
:108490009E009000E00220000088B90061022000E8
:1084A0008080400080C6210000804000AC9E020019
:1084B000000000001E0090000000E8001007980077
:1084C0001E009000E70F5000EAFF34007101200009
:1084D00040702000E6C90200000000000000EB0030
:1084E00020088900130020008200200011002000D5
:1084F0001000200055000700000FE900E0FF2F00EA
:108500009E0F1000030032000080EB009E0F100051
:1085100005003A00E1002000B0712000E6C9020029
:108520000000000042003700A1278100E002200087
:108530000088B900010220008080400080C6210030
:1085400000804000100078000000010000C502001B
:10855000000000001E007800A0278900A1278100EC
:10856000E00220000088B900FE00400080C6210023
:108570000080400010007800000001001E00E000B4
:1085800001003200CB02A80051002000305A200028
:10859000E6C9020000000000250037001E0FE900B8
:1085A000700020009E0F10001D003C00A1278100DC
:1085B000E00220000088B900010220008080400015
:1085C00080C62100008040001000780000000100FB
:1085D00000C50200000000001E007800A0278900EE
:1085E000A1278100E00220000088B900FE004000C1
:1085F00080C62100008040001000780000000100CB
:108600001E00E00001003200CB02A8005100200053
:10861000305A2000E6C902000000000004003700C4
:108620005101200090722000E6C902000000000005
:10863000000881008000E900F00F20000080600049
:10864000100889000080FA00000006001E00FA00F1
:10865000100F9800210F9800320F9800430F9800D8
:108660000000EB00400798000000EB002007980096
:108670000000EB00100798000000EB00000F7800EE
:10868000F05B2A00809E0200000000001E0890009F
:1086900018A1020000000000305C2A00809E020049
:1086A000000000006700370010A302000000000077
:1086B000204F98002E4890000000FB00600F9800AB
:1086C0006E089000ED0F500029003200EE08900077
:1086D000ED8F500007003C006E099000E80F51003C
:1086E0000D0032006E089000EA0F500020003200AA
:1086F00035003700D0022000EE089000808F500037
:108700001E003200800720006E099000800F51008B
:10871000270032002C0037004E0090000000E000DF
:10872000070032004E0090000000E900400798006A
:1087300060532A00809E02000000000041003700C4
:108740001E00E000060032000000EB00000F780081
:1087500060532A00809E02000000000039003700AC
:1087600070C0B30084A20200000000003500370092
:108770001000200020079800320037004E009000C3
:108780000000E00006003A00D0C2B30084A202005C
:108790000000000010002000000F780029003700C2
:1087A00070C0B30084A20200000000002500370062
:1087B0004E0890000000E000030032000080EB0053
:1087C000500F98005D003700AE489000F0C2B30033
:1087D00080CF500018003400AE48900090C3B30022
:1087E00080CF500014003C004E009000E30F50007A
:1087F0000600340070C0B30084A202000000000034
:1088000040002000400798000E0037002E489000DE
:1088100084A2020000000000CE0090006B00470020
:108820002E499000827078004E0090000000E80011
:10883000400798000300370070C0B30084A2020014
:10884000000000002E0090000000E00096FF3200C3
:10885000F0542A00AC9E0200000000004E00900080
:108860000000E00003003A001E089000500F98003E
:10887000320037000000EB00100798004E00900017
:108880000000E90040079800CE00900031079800F2
:10889000110037001E0090006A00B9001007980010
:1088A000BE0090004E009000808050006B0047009A
:1088B000614078008000FB001E0090008080400036
:1088C00000FD2F0000804000100798004E0090002F
:1088D0000000E900400798004E0090000000E00012
:1088E000ECFF3D009E0090002E089000808F50000D
:1088F0000D0035009E0090003E089000808F5000D3
:1089000009003C001E00E000040032001E00900040
:108910000000EA00500F9800080037001E01900088
:10892000520F980005003700B1012000E0EA200056
:10893000E6C902000000000049FF37005E08900011
:108940000080FA00000006000400FA00605C2A00C3
:10895000AC9E020000000000405D2A00809E0200E4
:1089600000000000F0542A00AC9E0200000000004D
:1089700061002000007620005CC9020000000000B9
:10898000B0278100D2A10200000000007100200089
:1089900070EA20005CC9020000000000C0278100CE
:1089A000D2A1020000000000605E2A00809E02004A
:1089B00000000000C0278100100798001E009000F2
:1089C000E10F5000040032001E009000E30F500041
:1089D0000500320008003700605F2A00809E020018
:1089E0000000000007003700905F2A00809E020010
:1089F0000000000003003700C05F2A00809E0200D4
:108A00000000000000602A00AC9E02000000000090
:108A1000E101200060762000E6C9020000000000AD
:108A20000080FA00000006000200FA0020602A0020
:108A3000809E020000000000A17F250010002000A1
:108A400060A2020000000000D2A1020000000000AD
:108A500000C2B30084A20200000000005100200008
:108A6000209220005CC9020000000000C17F2500A8
:108A70001000200060A2020000000000D2A102004D
:108A80000000000061002000709220005CC902001C
:108A900000000000E17F25001000200060A202001D
:108AA00000000000D2A1020000000000F0542A00E3
:108AB000AC9E020000000000C100200040782000B1
:108AC000E6C902000000000097000700CBC2BF000B
:108AD000624060000004E000050032001101200047
:108AE000806520005CC9020000000000040037001F
:108AF00021012000906620005CC9020000000000F7
:108B0000C0C2B30084A202000000000000C2B30093
:108B100084A2020000000000E2C2BF0070406000BA
:108B20000004E000050032004101200050602000F8
:108B30005CC9020000000000040037005101200061
:108B4000005F20005CC9020000000000C0C2B3004A
:108B500084A202000000000000C2B30084A2020050
:108B600000000000E8C2BF000042B2000004E000C4
:108B700003003A0090602A00809E0200000000007E
:108B8000E8C2BF00704060000004E00003003A004B
:108B900020612A00809E020000000000A0DE21006B
:108BA00010407800704060000004E00005003200D2
:108BB0002102200000792000E6C902000000000028
:108BC00004003700E1012000207B2000E6C90200FC
:108BD00000000000A0DE2100104078006840600026
:108BE0000004E00005003A00B1012000007D2000F3
:108BF0005CC902000000000004003700C101200031
:108C0000B07E20005CC9020000000000C0C2B300BA
:108C100084A202000000000000C2B30084A202008F
:108C200000000000B1012000101921005CC9020001
:108C30000000000090DD21001040780018A1020023
:108C400000000000F0542A00AC9E0200000000006A
:108C5000A0DE210010407800634060000080FB002F
:108C6000000F78001E007800E10F50001300320062
:108C70001E007800E10F500004003C001E00780048
:108C80000000E00008003200180037001E007800E5
:108C9000E20F50000E0032001E007800E30F50007B
:108CA0000F0032001100370051012000E05B20006E
:108CB000E6C90200000000000C003700610120003E
:108CC000805A2000E6C902000000000007003700BB
:108CD000C0612A00AC9E02000000000003003700C3
:108CE00040632A00AC9E020000000000A127810022
:108CF000E00220000088B90041022000808040008E
:108D000080C62100008040001000780000000100B3
:108D1000C100200040782000E6C9020000000000E9
:108D20000080FA00000006000000FA00A100200008
:108D3000A0052100E6C90200000000007105200026
:108D4000801E2100E6C90200000000004102200050
:108D5000F02321005CC9020000000000A12781006F
:108D6000E00220000088B90021022000808040003D
:108D700080C6210000804000100078000000010043
:108D8000A1002000E00721005CC9020000000000F3
:108D900010002000580007000010200056000700B7
:108DA00000022000540007000001200052000700CC
:108DB0008000200050000700400020004E00070007
:108DC000200020004C000700F0542A00AC9E020056
:108DD0000000000041002000800F21005CC902005B
:108DE0000000000021E3A80020C0B3008EC50200EF
:108DF000000000001CA20200000000001100200082
:108E0000903A20005CC902000000000090C0B3004E
:108E100084A20200000000000040EB008EC50200AA
:108E2000000000001CA20200000000001100200051
:108E3000903A20005CC902000000000090C0B3001E
:108E400084A202000000000050C0B3008EC50200E2
:108E5000000000001CA20200000000001100200021
:108E6000903A20005CC902000000000090C0B300EE
:108E700084A202000000000010C0B3008EC50200F2
:108E8000000000001CA202000000000011002000F1
:108E9000903A20005CC902000000000090C0B300BE
:108EA00084A202000000000021E3A90010002000BD
:108EB00020000700001020001E0007000002200014
:108EC0001C000700000120001A000700800020009D
:108ED00018000700400020001600070020002000B6
:108EE00014000700F0542A00AC9E020000000000AD
:108EF0000080FA00000006000200FA00000F78006F
:108F0000C01680001E0060000000E0000400320077
:108F1000C0642A00809E02000000000003003700A9
:108F2000F0642A00809E0200000000000080FA0029
:108F3000000006000200FA00000F7800D016800042
:108F40001E0060000000E0000400320020652A00DE
:108F5000809E0200000000000300370050652A00D8
:108F6000809E0200000000000080FA000000060061
:108F70000200FA00100881008000E800F00F2000D5
:108F800000806000100889001AFD070032FB07000E
:108F9000000F78001E00E0000600340040002000B2
:108FA0009E0F100003003C001E00E900902789007E
:108FB0000D0037000000EB0020088900210220008E
:108FC00040812000E6C90200000000008001EB00A3
:108FD0004200200011002000100020009BFD07002F
:108FE0000000E90090278900210120006083200013
:108FF000E6C90200000000000080FA000000060040
:109000000200FA000040EB00004F780010088100D9
:109010008000E800F00F2000008060001008890048
:10902000F4FC07000CFB0700104798001E4090005E
:109030000004E000090032001E409000EA4F50009A
:1090400006003E001E4090000040E900804078008D
:10905000004F2200014878000F0037000000EB00AD
:1090600020088900D108200030872000E6C90200CE
:10907000000000008001EB00A20020001100200091
:109080009000200071FD07000040E900804078005A
:10909000004F220001487800004F22001040780065
:1090A000E94F500010003A00D2FC0700EAFA07002E
:1090B000004F78001E04E0000B003A000000EB00B7
:1090C0002008890080652A00AC9E02000000000094
:1090D0008001EB00F2FF27008000EB00200220005F
:1090E0005AFD0700004F7800410120000090200049
:1090F000E6C9020000000000110120000018210054
:10910000E6C9020000000000004F22001040780075
:10911000E94F500003003A001E40780062A30200AD
:10912000000000005CA30200000000000000370007
:1091300004A30200000000000004E000FCFF320075
:1091400010A30200000000008040780000C2B300BD
:1091500080CF500001003200F5FF37000080FA0098
:10916000000006000400FA00A02781000000E000D3
:1091700007003A00D1012000305D2000E6C902005E
:109180000000000010002000200889006100370066
:10919000A0DE210010407800704060000004E00074
:1091A00007003A002102200050E82000E6C9020032
:1091B0000000000010002000200889005500370042
:1091C000E8A2A800E882A80020002000BEC6020095
:1091D0000000000021E3A80050C0B3008EC50200CB
:1091E000000000008000780000102000808F5000F8
:1091F0000300360000672A00AC9E02000000000059
:1092000021E3A900100881008000E800F00F200091
:10921000008060001008890076FC07008EFA0700C5
:10922000000F7800200881000000E00014003200E8
:109230000000EB0020088900A0692A00AC9E020013
:1092400000000000C06A2A00AC9E0200000000007E
:10925000106C2A00AC9E020000000000606D2A0025
:10926000AC9E0200000000008001EB0032002000F4
:109270001100200010002000F4FC0700000F78000F
:109280001E007800100798001E009000E20F5000AA
:109290000D0032001E009000E30F5000110032005C
:1092A0001E009000E10F5000010032001400370052
:1092B000E8A2A800E882A800A06E2A00AC9E0200E6
:1092C0000000000013003700E8A2A800EA82A9000D
:1092D000E882A900B0702A00AC9E020000000000E5
:1092E0000C003700E882A800EAA2A900E8A2A900C1
:1092F000F0722A00AC9E020000000000050037005A
:10930000E8A2A800E882A800A06E2A00AC9E020095
:10931000000000000080FA00000006000000FA00D3
:1093200001C38000808621000080400090407800CA
:1093300030C8B30080CF50000E003A0000C3800058
:109340000000E80000C388000300370000C380006D
:109350000000E80000C3880001C38000808621006F
:10936000008040009040780000CEB30080CF5000D5
:10937000F6FF36000080FA00000006000A00FA003E
:10938000300798000000EB0020079800AE00900026
:1093900080862100008040009040780000CEB3001D
:1093A00080CF500003003E000080EB004007980093
:1093B00023003700AE00900080862100008040002E
:1093C000104078008080FB0000F22F0000804000F9
:1093D000100798002E0090008000E8008086210091
:1093E00000804000104078000080FB004801DD0054
:1093F0002E0090008080E8008086210000804000E0
:10940000104078000080FB00000F41009E007800B3
:109410003E009000808F500003003A002E00900024
:1094200040079800060037009E0090002E00900034
:10943000008040006300400020079800D3FF370001
:109440004E0090000080FA00000006000600FA00BE
:10945000881F78000000EB00000F780001C3800037
:1094600080862100008040009040780080C2B300D8
:1094700080CF500010003A0000C380000000E800D8
:1094800000C3880021010700000F780001C380009D
:1094900080862100008040009040780090C2B30098
:1094A00080CF5000BC003A0000C380000000E800FC
:1094B00000C38800B800370001C380008086210007
:1094C000008040009040780000C4B30080CF50007E
:1094D0001600360001C38000808621000080400015
:1094E00090407800A0C5B30080CF50000F003E0030
:1094F00002C38000808621000000410010407800F7
:109500008080FB00F0FB2F000080400080004000C6
:1095100000802100008040001000780020079800A3
:109520000200E80000C388009D00370001C38000EE
:1095300080862100008040009040780000C8B30081
:1095400080CF50008600360001C380008086210055
:1095500000804000104078000080FB001007980059
:109560000100E80000C38800700920009E00900000
:10957000808F50004A003200700920009E00900049
:10958000808F50000D003C00400920009E0090009C
:10959000808F50001F003200600920009E00900064
:1095A000808F500034003200300920009E0090006F
:1095B000808F50002100320058003700A0092000A1
:1095C0009E009000808F50003F003200A0092000D4
:1095D0009E009000808F500005003C008009200014
:1095E0009E009000808F5000450032004B003700F5
:1095F000B00920009E009000808F5000390032009A
:10960000D00920009E009000808F5000160032008C
:1096100042003700A1278100E00220000088B90045
:10962000EA00400080C62100008040001000780061
:1096300000000100000F780057003700A1278100CB
:10964000E00220000088B900E800400080C6210048
:109650000080400010047800AC0007000800010002
:10966000000F78004C003700F09C02000000000062
:10967000000F780048003700A1278100E002200099
:109680000088B900F400400080C62100008040003E
:109690001000780000000100000F78003E00370045
:1096A000A1278100E00220000088B900F8004000F6
:1096B00080C62100008040001000780000000100FA
:1096C000000F780034003700CBC2BF000080FB00E1
:1096D0000000D100614060000080FB00000F7800B6
:1096E0002D003700E2C2BF000080FB004400DE0016
:1096F000614060000080FB00008FEA002600370018
:1097000021E3A80010C0B3008EC5020000000000D5
:10971000000F780021E3A9001F0037000000EB00D4
:10972000000F78001C0037001E0078006A00B900A6
:10973000000F780001C38000808621000080400077
:10974000104078000080FB009E00400000FD2F00CC
:10975000008F400000C380000000E80000C38800C4
:1097600001C3800080862100008040009040780086
:10977000F0C2B30080CF50000700360001C3800064
:1097800080862100008040009040780090C3B300A4
:1097900080CF5000E4FF36001E00780020079800BC
:1097A0002E0090004F0478000080FA0000000600B0
:1097B0000600FA0025FF0700000F780000003700C0
:1097C00001C3800080862100008040009040780026
:1097D000A0C2B30080CF50001800320001C3800047
:1097E000808621000080400090407800F0C2B300E5
:1097F00080CF50001100320001C38000808621001C
:10980000008040009040780060C2B30080CF5000DC
:109810000A00320001C380008086210000804000E1
:1098200090407800C0C7B30080CF500003003200E2
:109830001E007800200798003100370001C3800027
:109840008086210000804000104078000080FB00EE
:10985000100798000100E80000C38800A002200063
:109860009E009000808F500012003200A002200065
:109870009E009000808F500005003C006002200098
:109880009E009000808F500017003200CCFF370000
:10989000F00220009E009000808F50000B003200EC
:1098A000C00720009E009000808F50001100320001
:1098B000C3FF3700E5FE0700800078001E00780037
:1098C0000180B900000F7800BDFF3700DFFE070000
:1098D000000178001E007800110009000200D80085
:1098E000000F7800B6FF3700D8FE07001E0F60009B
:1098F000B3FF3700D5FE07001E0F7000B0FF370022
:109900002E0090000080FA00000006001200FA000D
:10991000A7FF0700000F78000000370001C3800098
:10992000808621000080400090407800D0C2B300C3
:1099300080CF50001F00320001C3800080862100CC
:109940000080400090407800B0C2B30080CF50004B
:109950001800320001C38000808621000080400092
:1099600090407800C0C3B30080CF50001100320097
:1099700001C3800080862100008040009040780074
:10998000E0C3B30080CF50000A00320001C3800062
:10999000808621000080400090407800D0C3B30052
:1099A00080CF5000030032001E007800200798008E
:1099B0008500370001C380008086210000804000C0
:1099C000104078000080FB00100798000100E800BC
:1099D00000C38800C00320009E009000808F5000CC
:1099E0003B003200C00320009E009000808F50009A
:1099F00009003C00B00220009E009000808F5000C3
:109A000011003200D00220009E009000808F500094
:109A10000A003200C1FF3700D00320009E009000F2
:109A2000808F50005E003200E00320009E00900016
:109A3000808F500007003200B8FF37005CFF07003E
:109A40001E0F1000B5FF370059FF07001E0F400022
:109A5000B2FF370000C380008000E800808621004C
:109A60000080400090407800D0C3B30080CF500009
:109A70000D003A004EFF07008000EB003107980010
:109A80009E0F500002003E0010002000300798009A
:109A9000BE009000010F780000C380000000E800C5
:109AA00000C388009DFF370041FF07008000EB00E6
:109AB000410798009E0F5000020031001000200066
:109AC00040079800CE009000010F780093FF370008
:109AD00000C380008000E8008086210000804000F4
:109AE00090407800E0C3B30080CF50000D003A00F2
:109AF0002FFF07008000EB00510798009E0F5000D9
:109B0000020032001000200050079800DE00900094
:109B1000010F780000C380000000E80000C3880047
:109B20007EFF370000C380008000E80080862100AF
:109B30000080400090407800D0C3B30080CF500038
:109B40000D003A001AFF07008000EB006107980043
:109B50009E0F50000200390010002000600798009E
:109B6000EE009000010F780000C380000000E800C4
:109B700000C3880069FF37000DFF07008000EB007D
:109B8000710798009E0F5000020036001000200060
:109B900070079800FE009000010F78005FFF37000B
:109BA00003FF07008000EB00010F98009E0F50009C
:109BB00002003A0010002000000F98008E0890006C
:109BC000010F780055FF37002E0090000080FA004A
:109BD000000006001C00FA00881F78000000EB005F
:109BE00000C388000000EB00300798000000EB0085
:109BF000200798000000EB00100798000000EB0021
:109C000010C388000000EB0020C388000000EB00B8
:109C100030C388000000EB0050079800D027810077
:109C20000080A000D02789000000EB0040079800CA
:109C3000090037004E0090008000400000802100A5
:109C4000808040000000EB00800878004E0090000B
:109C50000000E800400798004E009000F90F500007
:109C6000F4FF3400340437001E0090000000E000D0
:109C700021003A0001C3800080862100008040005E
:109C800090407800F0CDB30080CF500003003E003C
:109C900020002000300798002A04370001C380000C
:109CA0008086210000804000104078008080FB000A
:109CB00000F22F00008040006007980000C3800081
:109CC0008000E8008086210000804000104078007D
:109CD0000080FB004801DD0000C380008080E800B8
:109CE0008086210000804000104078000080FB004A
:109CF00000007100500798000000EB00100798006A
:109D000000C38000E3004000808621000080400006
:109D1000104078000080FB006101B90000F82F00BE
:109D2000F1FF2F000201400083814800420F98009C
:109D3000530F980010022000010020004E099000EF
:109D4000DE099000800F5100818F5900EE033E0024
:109D50004E089000DE0890000060010021003700EE
:109D600035003700E8033700E7033700710037009C
:109D700081003700A3003700B7003700BE0037006E
:109D80003B01370088013700DF033700EE01370061
:109D90003502370099023700AF0237009F023700C3
:109DA000CB023700BB023700D8023700D60337009A
:109DB000780337005C033700D3033700D203370042
:109DC00000033700F00237009F033700AD03370070
:109DD000DE0237001203370032033700B5033700C5
:109DE000C6033700100020002007980000C3800041
:109DF0006600400000C3880000C380008080E90046
:109E00008086210000804000104078008080FB00A8
:109E1000F0FB2F0000844000BCFE0700000178002A
:109E20008800440000802100008040000208780083
:109E30003AFD0700B6033700100020002007980005
:109E400000C380006400400000C38800AFFE07002C
:109E50000000E0001C00320001C38000310F9800B8
:109E6000808621003E09900000004100904078006B
:109E70008041EB004357980020C8B30080CF5000CA
:109E800002003A0010C0B30040579800BE0890008E
:109E90000100E80000C388004E5190000204E00079
:109EA0009B033200100020001007980000C38000C0
:109EB0006300500000C388009503370000C3800092
:109EC0000000E80000C3880001C3800080862100F4
:109ED000008040009040780030C8B30080CF500030
:109EE0000700320001C3800080862100008040000E
:109EF0009040780000CEB30080CF5000EFFF3600D6
:109F000001C38000808621000080400090407800DE
:109F100030C8B30080CF50007D033A00100020000D
:109F20001007980000C380000080E90000C388008B
:109F300077033700100020002007980000C380003E
:109F40006400400000C3880070FE07000BFD07009E
:109F5000000F78008081EB009E8F1100030032001B
:109F60001E00780000C388006903370060002000ED
:109F70003007980066033700100020002007980083
:109F800000C380006400400000C3880020C380003C
:109F9000E90F500018003C0022C3800001C380007C
:109FA0006E009000008040008001E90082004100C6
:109FB00040832100008040000308780020C3800017
:109FC0000000E80020C3880050FE0700EBFC0700FB
:109FD000000F78008080EB009E8F1000030032009D
:109FE0001E01780002C3880049033700600020008A
:109FF00030079800460337007000200030079800B3
:10A0000043033700E0862A00809E02000000000023
:10A01000100020002007980020C380000000E0000E
:10A020000A00320020C380000000E90020C388003D
:10A0300020C3800080004000408321000080400059
:10A040001000780000C38800310337008000200032
:10A05000300798002E0337001000200020079800DA
:10A0600001C380006E00900000804000630040004B
:10A0700000C3880026033700100020002007980046
:10A0800000C380006400400000C388005700370010
:10A0900001C380008086210000804000904078004D
:10A0A00020C2B30080CF50001F003A0000C38000E0
:10A0B0000000E80000C3880010003700D0278100AE
:10A0C0000080A100D027890001C380008086210084
:10A0D0000080400010407800004178000100E80056
:10A0E00000C388000240780084A202000000000043
:10A0F000D02781000080A000D027890001C3800004
:10A1000080862100008040009040780020C2B3008B
:10A1100080CF5000E9FF3A0000C380000000E80053
:10A1200000C388003100370001C380008086210011
:10A13000008040009040780000C4B30080CF500001
:10A140000700360001C380008086210000804000A7
:10A1500090407800A0C5B30080CF50000D003600BD
:10A1600001C38000808621000080400010407800FC
:10A170000004E00013003D0001C380008086210040
:10A180000080400090407800F0CDB30080CF5000B8
:10A190000C003E00DDFD0700000F7800D027810095
:10A1A0000080A100D02789001E007800BAA002001C
:10A1B00000000000D02781000080A000D027890087
:10A1C0000A00370001C38000808621000080400023
:10A1D00090407800B0C3B30080CF500003003A0035
:10A1E00000C380000000E80000C3880001C38000B5
:10A1F000808621000080400090407800F0CDB300C0
:10A2000080CF500007003E0001C3800080862100FF
:10A21000008040009040780030C8B30080CF5000EC
:10A220009BFF3A0000C380008000E9008086210087
:10A230000080400090407800B0C3B30080CF500051
:10A2400009003200D02781000080A100D0278900BA
:10A2500040902A00AC9E020000000000D027810040
:10A260000080A000D02789002CFC0700A80237003E
:10A270001000200020079800D02781000080A10056
:10A28000D027890000C380006400400000C388001C
:10A2900001C380008086210000804000904078004B
:10A2A00020C2B30080CF500018003A0000C38000E5
:10A2B0000000E80000C388000A00370001C38000E6
:10A2C0008086210000804000104078000041780026
:10A2D0000100E80000C388000240780084A2020068
:10A2E0000000000001C38000808621000080400043
:10A2F0009040780020C2B30080CF5000EFFF3A00BA
:10A3000000C380000000E80000C3880001C3800093
:10A31000808621000080400090407800C0C2B300D9
:10A3200080CF500004003A0000C380000000E80025
:10A3300000C388000200370030002000300798007A
:10A3400001C380008086210000804000104078001A
:10A350008080FB00F0FB2F00008440008001EB00B8
:10A36000F2FF27008000EB000000EB002643020014
:10A3700000000000000178008800440000802100F7
:10A38000008040000208780000C380000000E80060
:10A3900000C38800E1FB0700D02781000080A000F7
:10A3A000D02789005A0237001000200020079800AB
:10A3B00000C380006400400000C3880010C3800018
:10A3C000E30F500004003C0010C380000000E800D0
:10A3D00010C38800020037004000200030079800BA
:10A3E00012C3800003C380008086210000804100EA
:10A3F000104078008080FB0000FC2F0000824000AD
:10A400006610B9008080E800808421000080400050
:10A41000040878000300E80000C3880001C380003E
:10A42000808621000080400090407800D0C3B300B7
:10A4300080CF500011003A0000C380000000E80007
:10A4400000C3880010C380006600B9008080E80067
:10A450008084210000804000100078000004E900A2
:10A460002AFD0700000178008800440000802100D8
:10A470000080400002087800020037003000200011
:10A480003007980003C38000130F980080862100D6
:10A490009E08900000804000904078000041EB0052
:10A4A00002579800B0C8B30080CF500002003A00B5
:10A4B00013C0B300035798009E0890000100E80005
:10A4C00000C388000E5190000204E0000900320031
:10A4D00018C380000DFD0700000178006640B90038
:10A4E000E4004000808421000080400002087800E1
:10A4F00002003700300020003007980001C38000C0
:10A50000808621000080400090407800F0CDB300AC
:10A5100080CF50000800360010C3800002C38000C6
:10A520006600B9008000780080842100008040002F
:10A530000208780002003700300020003007980041
:10A5400076FB0700F201370010002000200798007A
:10A5500000C380006400400000C3880002C3800084
:10A560008086210000004100104078008080FB00C0
:10A5700000FC2F00008F40000200E80000C38800AC
:10A5800050002000300798000000EB0040079800C2
:10A590002F0037004E0090006600B9008080E80070
:10A5A0008084210000804000100078009E0F500041
:10A5B00024003A001E00E9008000400000802100D5
:10A5C00000804000100178004E0090006600B90045
:10A5D000E4004000808421000080400010007800EA
:10A5E000800F510012003D009E00E90001814000F3
:10A5F0000080210000004100100078000001E80008
:10A600008180400000802100008040000208780026
:10A610004E0090006600B900800078008084210020
:10A62000008040001000780000C38800030037005D
:10A6300010C380000000E90010C388000000EB0098
:10A64000300798004E0090000000E8004007980096
:10A6500011C380004E009000810F5000CDFF3400E8
:10A660002EFB0700AA0137001000200020079800E9
:10A6700000C380006400400000C3880030C3800035
:10A680000000E00027003A000000EB0040079800BF
:10A690000A003700CE009000808621000080400034
:10A6A000104078008080FB004E00900080804000C9
:10A6B00030F22F0000804000400798004E009000CC
:10A6C000E300400080862100008040009040780038
:10A6D000E0C8B30080CF500006003200CE009000EA
:10A6E0008086210000804000104078000004E000D7
:10A6F000E8FF3A00CE0090008086210000804000F4
:10A70000104078000004E000040032004E00900089
:10A710006400400030C38800020037009000200031
:10A720003007980003C38000030F780030C3800017
:10A7300000C388009E0078008086210000804000D1
:10A74000104078008080FB00F0FB2F000084400068
:10A750003EFB0700000178008800440000802100D3
:10A76000008040000208780000C3800030C38800E9
:10A770001E00E80000C3880031C3800080862100ED
:10A780000080400090407800C0C2B30080CF5000ED
:10A7900003003A0030C380000000E80030C38800A6
:10A7A00031C3800080862100008040009040780006
:10A7B00000CEB30080CF50000E00360030C38000C2
:10A7C000E300400080862100008040009040780037
:10A7D000E0C8B30080CF5000030032000000EB005F
:10A7E00030C388000300370030C38000640040009D
:10A7F00030C38800C9FA0700450137001000200067
:10A800002007980001C380006E0090000080400087
:10A810006300400000C388003D01370010002000A5
:10A820002007980000C380006400400000C3880037
:10A83000A1278100E00220000088B9008000780094
:10A8400080C6210000804000100078000000010058
:10A85000B2FA07002E0137001000200020079800F0
:10A8600000C380006400400000C38800A12781006D
:10A87000E00220000088B9008080E80080C6210046
:10A88000008040001000780000000100A3FA0700DB
:10A890001F013700100020002007980000C380002F
:10A8A0006400400000C38800A1278100E00220006E
:10A8B0000088B900E400400080C62100008040000C
:10A8C000100078000000010094FA07001001370022
:10A8D000100020002007980000C3800064004000A2
:10A8E00000C38800A1278100E00220000088B90091
:10A8F000E600400080C62100008040001000780083
:10A900000000010085FA0700010137001000200057
:10A910002007980000C380006400400000C3880046
:10A92000A1278100E00220000088B900E800400073
:10A9300080C621000080400010047800F3FB07006F
:10A940000800010075FA0700F10037001000200030
:10A950002007980000C380006400400000C3880006
:10A96000EAFB07000000E00003003200509C0200F8
:10A970000000000002003700A09C02000000000060
:10A9800066FA0700E2003700100020002007980058
:10A9900000C380006400400000C38800DBFB0700A8
:10A9A0000000E00003003200C922A900CB22A80069
:10A9B00002003700C922A900CB22A90057FA0700DC
:10A9C000D3003700100020002007980000C380004B
:10A9D0006400400000C38800CCFB07000000E000DA
:10A9E00007003200A0DE2100104078000000A00027
:10A9F0000010A100A1DE2100804878000600370089
:10AA0000A0DE2100104078000000A0000010A1008E
:10AA1000A1DE21008048780040FA0700BC00370022
:10AA2000100020002007980000C380006400400050
:10AA300000C38800B5FB0700103389001033810084
:10AA40000000E00002003D000000EB001033890030
:10AA50001133810000FA2000808F50000200340082
:10AA600000FA20001033890020338100E10F5000EC
:10AA700002003C00200020002033890021338100A7
:10AA800030062000808F5000020034003006200085
:10AA900020338900CA980200000000001FFA070056
:10AAA0009B003700100020002007980000C38000A2
:10AAB0006400400000C3880094FB07002033890035
:10AAC000103381000000E00002003D000000EB00B8
:10AAD000103389001133810000FA2000808F50006C
:10AAE0000200340000FA2000103389002033810076
:10AAF000E10F500002003C002000200020338900BC
:10AB00002133810030062000808F50000200340085
:10AB10003006200020338900CA980200000000009F
:10AB2000FEF907007A003700100020002007980087
:10AB300000C380006400400000C3880073FB07006E
:10AB40000000E00009003200A1278100E00220009F
:10AB50000088B900F000400080C62100008040005D
:10AB6000100078000000010008003700A1278100D4
:10AB7000E00220000088B900F200400080C62100F9
:10AB8000008040001000780000000100E3F9070099
:10AB90005F003700100020002007980000C38000ED
:10ABA0006400400000C3880058FB0700700798004D
:10ABB0007E009000E10F500010003200FE00900077
:10ABC000E28F5000160032007E0190000200E0008B
:10ABD000010032001A003700A1278100E0022000A6
:10ABE0000088B900EE00400080C6210000804000CF
:10ABF000100078000000010011003700A12781003B
:10AC0000E00220000088B900EC00400080C621006E
:10AC100000804000100078000000010008003700AC
:10AC2000A1278100E00220000088B900F600400062
:10AC300080C6210000804000100078000000010064
:10AC4000B6F90700320037001000200020079800F6
:10AC500000C380006400400000C388002BFB070095
:10AC60000000E00003003200E082A800E282A900B8
:10AC700002003700E282A900E082A900A7F90700DC
:10AC800023003700100020002007980000C3800038
:10AC90006400400000C388001CFB0700000F780020
:10ACA0001E007800BEC60200000000009BF90700ED
:10ACB00017003700100020002007980000C3800014
:10ACC0006400400000C3880010FB0700000F7800FC
:10ACD000A1278100E00220000088B900FC004000AC
:10ACE00080C6210000804000900078001E0078009F
:10ACF0000100010089F9070005003700100020005D
:10AD0000300798000200370030002000300798001C
:10AD10002E0090000000E00005003A0001C3800012
:10AD20006E009000008040006300400000C3880077
:10AD30000000EB00200798003E0090000000E000BB
:10AD4000C9FB3200D02781000080A100D0278900F4
:10AD50003E009000E10F500018003200610020001A
:10AD6000A03A20005CC90200000000003E009000F4
:10AD7000BAA002000000000081002000003B20007B
:10AD80005CC90200000000005E009000BAA0020052
:10AD900000000000B1002000803B20005CC90200E0
:10ADA0000000000000C38000BAA002000000000004
:10ADB00040902A00AC9E0200000000004F04780082
:10ADC0000080FA00000006000200FA00000F780080
:10ADD00000C2B30084A20200000000001E00780040
:10ADE000809E02000000000000C2B30084A20200A6
:10ADF000000000000080FA00000006000400FA00D5
:10AE00000000EB0000C388003F00370001C3800052
:10AE10008086210000804000904078002147980003
:10AE20002E4090000004E000040035002E40900009
:10AE300084A202000000000030003700AE40900005
:10AE400000CEB30080CF50001C00360040902A0096
:10AE5000AC9E02000000000000C380008000E800FB
:10AE60008086210000804000104078000080FB00B8
:10AE70004801DD0000C380008080E800808621005A
:10AE800000804000104078000080FB00000041007E
:10AE9000000F780000C380000080E80000C3880035
:10AEA0001E007800BAA002000000000000C2B3003B
:10AEB00084A20200000000001000370000C2B300AE
:10AEC00084A20200000000002E4090008080FB0061
:10AED00000F82F000080400080004000805B2200CE
:10AEE0000080400010007800809E020000000000FA
:10AEF00000C2B30084A202000000000000C3800072
:10AF00000000E80000C3880001C3800080862100A3
:10AF100000804000104078000004E000BBFF3A00D1
:10AF200040902A00AC9E02000000000000C3800098
:10AF30000000E900BAA0020000000000710020003B
:10AF4000303C2000E6C90200000000000080FA004A
:10AF5000000006000600FA001007980010088100A3
:10AF6000000F7800150037001E0090001041780097
:10AF7000110881000000220000804000104078008D
:10AF8000804F5100050032001E0078001008890033
:10AF90000000EB00200798000E0037001008810029
:10AFA0008000E800F00F2000008060001008890099
:10AFB0001E0090000000E800100798001E0090009E
:10AFC000104078000004E000E7FF3A001000200085
:10AFD000200798002E0090000080FA000000060074
:10AFE0000400FA000000EB00000F780010003700AA
:10AFF0001E00780080004000805B2200008040003E
:10B0000010007800D3FF07000000E00007003200C6
:10B010001E0078008040780000C8B30000C04000E7
:10B020000080FB0010079800060037001E0FE800A4
:10B03000100220009E0F1000EDFF34000000EB0016
:10B04000100798001E0090000080FA000000060023
:10B050003600FA0010088100000F98001F0037002A
:10B060008E08900000002200008040009040780090
:10B0700000C6B30080CF5000110034008E0890004D
:10B08000000022000080400090407800A0C7B3007C
:10B0900080CF50000A003C000E0990008E089000FE
:10B0A000000022000080400090407800F0CDB30006
:10B0B00080C06000000022000000410001487800CC
:10B0C0000E0890000000E800000F98008E08900025
:10B0D000F00F200000806000000F98008E089000A4
:10B0E00000088100808F5000DDFF3A000000EB0077
:10B0F000000F98001108810000002200008040002D
:10B1000090407800F0C2B30080CF50002E01340090
:10B11000110881000000220000804000904078006B
:10B1200090C3B30080CF500027013C000000EB002B
:10B13000000F9800080037008E089000720047004A
:10B14000808040000040EB00804878000E089000AE
:10B150000000E800000F98008E08900020022000F8
:10B16000808F5000F4FF34002C3E020000000000ED
:10B17000600798006E0090004880DE0080407800F4
:10B1800072004700114098006E00900080407800E7
:10B1900000C0EB0080C060007200470021409800B2
:10B1A0006E00900075F80700500798005E00900050
:10B1B000E10F40002B003200DE009000808621006D
:10B1C00000804000104078008080FB0030F22F00AB
:10B1D00000804000300798005E009000000F98004B
:10B1E0000D0037000E0990008E0890003E00900080
:10B1F00080804000808621000080400090407800E0
:10B200008086210000004100014878000E0890006F
:10B210000000E800000F9800014020003E00900070
:10B22000808050000E089000808F5000EDFF3C00A1
:10B23000080037008E089000808621008080400042
:10B240000040EB00804878000E0890000000E80005
:10B25000000F98008E089000F03F2000808F500073
:10B26000F4FF340030002000000F98000000EB00D5
:10B2700020079800FA410200000000004200370059
:10B280002E0090000000E00002003A00FA410200A7
:10B29000000000002E0090000000E00004003A00D2
:10B2A0004FFF07000080FB00600798000200370096
:10B2B0000000EB00600798006E0090000000E000C6
:10B2C0000D0032000E0990006E0090008040780062
:10B2D000720047000000410001487800EE00900035
:10B2E00070082000808F50001B003A0010002000E2
:10B2F0002007980018003700110881000000220084
:10B30000008040009040780020C2B30080CF500001
:10B3100003003A002E0090000000A20020079800D1
:10B320000E099000110881000000220000804000FA
:10B330001040780080407800720047000000410013
:10B3400001487800100881008000E800F00F20001C
:10B3500000806000100889000E0890000000E800DE
:10B36000000F98008E08900030022000808F50005F
:10B370000500340091002000A03C2000E6C9020036
:10B3800000000000D500370011088100000881008E
:10B39000808F5000BAFF3A000E089000E30F500073
:10B3A000CE0032000E089000E40F5000CB003200B7
:10B3B0000E08900080407800C0CDB30000C040006F
:10B3C0008040780072004700014878000000EB00E0
:10B3D000000F98000000EB00400798000000EB0011
:10B3E00050079800460037008E08900080862100A4
:10B3F000008040009040780000CEB30080CF500025
:10B400002E0036008E0890008086210000804000CB
:10B41000104078008080FB0000F22F000080400088
:10B42000300798000E0890008000E8008086210018
:10B4300000804000104078000080FB004801DD00E3
:10B440000E0890008080E800808621000080400087
:10B45000104078000080FB000000410010079800B9
:10B4600072004700104090000080FB00C800DD0023
:10B4700072004700204090000080FB0000804000E8
:10B48000000F78001E0090009E0F50000500310054
:10B490008E0890003E009000008040006300400055
:10B4A00050079800BE0090000E08900000804000F9
:10B4B00063004000000F9800020037000E08900063
:10B4C000400798000E0890008000E8008086210068
:10B4D00000804000104078000080FB004801DD0043
:10B4E0000E0890008080E8008086210000804000E7
:10B4F000104078000080FB000000410060079800C9
:10B500004E0090000000E000B7FF320072004700DC
:10B51000104078008080FB0030F22F000080400057
:10B52000600798004E009000000F98000D00370053
:10B530008E0890006E009000008140008E08900000
:10B5400080862100008040009040780080862100A5
:10B5500000004100014878000E0890000000E9005A
:10B56000000F98008E0890005E009000808F5000C1
:10B57000EFFF3D000000EB00000F98000D003700CA
:10B58000DE0090000E089000008140008E089000C0
:10B5900072004700008040009040780080862100C3
:10B5A00000004100014878000E0890000000E8000B
:10B5B000000F98008E0890006E009000808F500061
:10B5C000EFFF35004500370050902A0061FE07006C
:10B5D0000000E000050032007EF9070040902A00DC
:10B5E000AC9E0200000000003C00370090902A0052
:10B5F00058FE07000000E00002003200FFFD0700D7
:10B6000036003700E0902A0052FE07000000E000FC
:10B6100004003200D02781000090A100D0278900CB
:10B620002E00370030912A004AFE07000000E0009B
:10B63000200032000000EB00000F980018003700D7
:10B640000000EB00700798000F0037008E08900094
:10B650007E009000808040008086210000804000B5
:10B66000104078000080FB007AA10200000000007A
:10B6700000C2B30084A20200000000007E0090001F
:10B680000000E800700798007E009000EF0F500067
:10B69000EEFF34000E08900070004000000F98008C
:10B6A0008E089000F03F2000808F5000E4FF3400AF
:10B6B0000A00370090912A0026FE07000000E000F3
:10B6C000020032000700070004003700C10020001C
:10B6D000303D2000E6C90200000000000080FA00B2
:10B6E000000006000200FA000000EB00000F7800E6
:10B6F000060037009E007800808621008080400090
:10B700000040EB00804878001E0FE800F03F20006A
:10B710009E0F1000F7FF340011CEB3008086210089
:10B720000148780080C0EB00908621000148780035
:10B7300080C0EB00A08621000148780011CAB30048
:10B74000B0862100014878000080FA000000060061
:10B750005752490054452000424954003A202000E5
:10B760002A6E650078742000636C6F00636B2000A4
:10B77000285E2900207769006C6C200075736500D5
:10B78000207468006973200076616C007565310073
:10B7900057495200452072006F757400696E65004C
:10B7A00073202800432920003230300030204D0023
:10B7B0006963680061656C00205065006172630018
:10B7C000652047004E55200047504C004E6F20002A
:10B7D00064657600696365002C207400727920002E
:10B7E00028414C0041524D00292053004541520050
:10B7F000434820006D616300726F2000666972002B
:10B80000737441004444520045535300204D41009D
:10B8100043524F00202030002E4D610063726F00B4
:10B82000206D65006E754D00616372006F20200011
:10B8300020202000315749005245200061646400F7
:10B8400072657300730D0A00202020002A31570012
:10B850004952450020524F004D2043004F4D4D00AE
:10B86000414E4400204D410043524F00733A0D00B9
:10B870000A203500312E52004541440020524F002D
:10B880004D20280030783300332920002A666F00CD
:10B8900072207300696E67006C6520006465760035
:10B8A0006963650020627500730D0A002038350059
:10B8B0002E4D41005443480020524F004D20280097
:10B8C00030783500352920002A666F006C6C6F00D7
:10B8D0007765640020627900203634006269740064
:10B8E000206164006472650073730D000A203200E9
:10B8F00030342E00534B4900502052004F4D200051
:10B900002830780043432900202A66006F6C6C00C1
:10B910006F77650064206200792063006F6D6D00B1
:10B92000616E64000D0A2000323336002E414C0057
:10B9300041524D0020534500415243004820280009
:10B940003078450043290D000A20320034302E00A3
:10B95000534541005243480020524F004D202800DB
:10B9600030784600302941004C4152004D205300B0
:10B9700045415200434820002830780045432900C3
:10B98000534541005243480020283000784630009B
:10B9900029446500766963006520490044732000EE
:10B9A000617265002061760061696C0061626C0003
:10B9B0006520620079204D00414352004F2C200049
:10B9C0007365650020283000292E5200454144004F
:10B9D00020524F004D2028003078330033293A00A0
:10B9E000204D41005443480020524F004D20280074
:10B9F00030783500352953004B49500020524F0014
:10BA00004D20280030784300432955006E6B6E00AE
:10BA10006F776E00206D610063726F002C207400E0
:10BA2000727920003F206F0072202800302920000A
:10BA3000666F7200206865006C70420055532000EC
:10BA40005245530045542000576172006E696E00E4
:10BA5000673A20002A5368006F727400206F7200EA
:10BA6000206E6F00207075006C6C2D0075702000CA
:10BA70002A4E6F00206465007669630065206400CB
:10BA800065746500637465006420440053313800B8
:10BA9000533230002048690067682000507265000A
:10BAA000732044006967200054686500726D44008B
:10BAB0005331380042323000205072006F6720004E
:10BAC0005265730020446900672054006865720065
:10BAD0006D4453003138320032204500636F6E00F0
:10BAE0002044690067205400686572006D4453006B
:10BAF0003234300034204500636F6E0072616D0097
:10BB0000207469006D65200043686900704453002B
:10BB100032343300312031004B2045004550520073
:10BB20004F4D55006E6B6E006F776E0020646500A0
:10BB300076696300655057004D20640069736100A9
:10BB4000626C650064314B00487A2D00342C300063
:10BB500030304B00487A200050574D004672650047
:10BB6000717565006E63790020696E00204B480096
:10BB70007A2050007265730063616C00653A500072
:10BB800052323A00447574007920630079636C0086
:10BB9000652069006E202500205057004D2061006F
:10BBA000637469007665450052524F00523A200096
:10BBB00050574D002061630074697600652C2000A9
:10BBC000672074006F20640069736100626C650017
:10BBD000415558002046720065717500656E63001E
:10BBE000793A20004155580020494E0050555400E4
:10BBF0002F4849002D5A4100555820004849470018
:10BC00004841550058204C004F5756004F4C5400A7
:10BC10004D455400455220004D4F440045564F00BD
:10BC20004C5441004745200050524F0042453A00D5
:10BC30002056450072726F007228290020406C0067
:10BC4000696E65003A20400070676D007370610096
:10BC500063653A0020627900746573002E546F00AA
:10BC60006F206C006F6E6700215379006E74610065
:10BC70007820650072726F00724E6F00204545009B
:10BC800050524F004D457200617369006E67640049
:10BC90006F6E650053617600696E670020746F00F7
:10BCA00020736C006F742000496E7600616C69002F
:10BCB000642073006C6F74004C6F610064696E00E7
:10BCC00067206600726F6D0020736C006F74200037
:10BCD000455252004F523A0020636F006D6D610073
:10BCE0006E64200068617300206E6F00206566003E
:10BCF00066656300742068006572650041434B000F
:10BD00004E4143004B4932004320530054415200FE
:10BD100054204200495449003243200053544F00FC
:10BD20005020420049544900324320006D6F6400A6
:10BD3000653A0D000A2031002E2053006F66740012
:10BD400077617200650D0A0020322E0020486100E4
:10BD5000726477006172650053657400207370002F
:10BD6000656564003A0D0A0020312E00207E350002
:10BD70004B487A000D0A2000322E20007E3530001C
:10BD80004B487A000D0A2000332E20007E3130000F
:10BD9000304B48007A0D0A0020342E00207E3400FB
:10BDA00030304B00487A570041524E00494E470010
:10BDB0003A20480041524400574152004520490072
:10BDC000324320006973200062726F006B656E0061
:10BDD000206F6E0020746800697320005049430092
:10BDE0002120280052455600204133002953650088
:10BDF0007420730070656500643A0D000A203100FC
:10BE00002E20310030304B00487A0D000A203200DD
:10BE10002E20340030304B00487A0D000A203300C9
:10BE20002E2031004D487A004932430020286D0011
:10BE30006F64200073706400293D280020203000CA
:10BE40002E4D610063726F00206D65006E750D00F0
:10BE50000A2031002E37620069742000616464009A
:10BE600072657300732073006561720063680D0072
:10BE70000A2032002E493200432073006E696600AA
:10BE8000666572005365610072636800696E6700E1
:10BE900020493200432061006464720065737300BE
:10BEA00020737000616365002E2046006F756E0080
:10BEB0006420640065766900636573002061740026
:10BEC0003A536E006966660065722800424153006D
:10BED0004943290052656100647961002F412F00B8
:10BEE000402063006F6E7400726F6C00732041001D
:10BEF0005558200070696E00612F41002F402000CE
:10BF0000636F6E0074726F006C73200043532000E7
:10BF100070696E00436F6D006D616E0064206E008D
:10BF20006F74200075736500642069006E207400D2
:10BF300068697300206D6F0064655000756C6C005B
:10BF40002D7570002072650073697300746F720044
:10BF500073204F0046465000756C6C002D757000C4
:10BF60002072650073697300746F720073204F0054
:10BF70004E5365006C662D00746573007420690073
:10BF80006E204800695A20006D6F640065206F00C4
:10BF90006E6C790052455300455442004F4F540097
:10BFA0004C4F4100444552004155580020494E0035
:10BFB000505554002F4849002D5A2C00205245005E
:10BFC00041443A0020506F0077657200207375007D
:10BFD00070706C0069657300204F4E00506F7700E1
:10BFE0006572200073757000706C690065732000C5
:10BFF0004F464600444154004120530054415400F0
:10C00000453A200044454C004159200075735700C3
:10C0100052495400453A200052454100443A20001C
:10C02000434C4F00434B2C00203143004C4F430006
:10C030004B2C200030444100544120004F55540007
:10C04000505554002C2031004441540041204F00F1
:10C050005554500055542C00203020002A7069009F
:10C060006E20690073206E006F77200048695A00C7
:10C07000434C4F00434B2000544943004B533A007C
:10C080002052450041442000424954003A205300C8
:10C09000796E740061782000657272006F72200002
:10C0A0006174200063686100722078002E206500B2
:10C0B000786974002877690074686F0075742000CF
:10C0C000636861006E676500296E6F00206D6F0008
:10C0D00064652000636861006E6765004E6F6E00E6
:10C0E00065786900737465006E74200070726F006B
:10C0F000746F63006F6C2100782E200065786900F2
:10C10000740D0A00496E7600616C6900642063005A
:10C11000686F690063652C002074720079206100EB
:10C12000676169006E444500564944003A687400EE
:10C1300074703A002F2F6400616E670065726F00A3
:10C1400075737000726F74006F747900706573009E
:10C150002E636F006D2A2D002D2D2D002D2D2D000D
:10C160002D2D2D002A4F7000656E20006472610035
:10C17000696E20006F75740070757400732028005C
:10C18000483D4800692D5A002C204C003D474E0088
:10C1900044294E006F726D00616C20006F75740051
:10C1A0007075740073202800483D33002E337600EC
:10C1B0002C204C003D474E0044294D0053422000A6
:10C1C000736574003A204D004F535400207369008A
:10C1D00067206200697420006669720073744C0005
:10C1E00053422000736574003A204C0045415300CF
:10C1F000542073006967200062697400206669003A
:10C200007273740020426F006F746C006F61640081
:10C2100065722000762031002E20480045580D0020
:10C220000A2032002E20440045430D000A2033002E
:10C230002E204200494E0D000A2034002E205200CC
:10C2400041574400697370006C61790020666F008B
:10C25000726D610074207300657456006F6C740019
:10C2600061676500206D6F006E6974006F72730006
:10C270003A203500563A2000207C2000332E33002F
:10C28000563A2000207C2000565055004C4C55005A
:10C29000503A200053657400207365007269610094
:10C2A0006C2070006F72740020737000656564000C
:10C2B0003A20280062707300290D0A0020312E00F8
:10C2C00020333000300D0A0020322E0020313200A1
:10C2D00030300D000A2033002E2032003430300080
:10C2E0000D0A2000342E200034383000300D0A00B2
:10C2F00020352E002039360030300D000A2036005F
:10C300002E20310039323000300D0A0020372E0047
:10C3100020333800343030000D0A2000382E200041
:10C320003537360030300D000A2039002E2031001C
:10C330003135320030300D000A3130002E204200FD
:10C340005247200072617700207661006C756500AD
:10C3500041646A007573740020796F007572200063
:10C36000746572006D696E00616C41007265200039
:10C37000796F75002073750072653F002043460099
:10C3800047313A002043460047323A00285C2D00EE
:10C390002F5F5C002D2928005C5F2F002D295300A2
:10C3A000656C6500637420006F75740070757400AF
:10C3B0002074790070653A000D0A2000312E2000AB
:10C3C0004F7065006E206400726169006E20280065
:10C3D000483D4800692D5A002C204C003D474E0036
:10C3E00044290D000A2032002E204E006F726D008D
:10C3F000616C200028483D00332E3300562C20006D
:10C400004C3D47004E44290052325700202873000B
:10C410007064200068697A00293D280020203000DF
:10C420002E4D610063726F00206D65006E750D000A
:10C430000A2031002E4953004F37380031362D0085
:10C440003320410054520D000A2032002E4953007F
:10C450004F37380031362D00332070006172730081
:10C4600065206F006E6C790049534F00203738000B
:10C4700031362D003320410054522000285245000F
:10C4800053455400206F6E0020435300290D0A00CD
:10C49000524553004554200048494700482C20008D
:10C4A000434C4F00434B2000544943004B2C200089
:10C4B00052455300455420004C4F570049534F00FC
:10C4C0002037380031362D003320720065706C0043
:10C4D00079202800757365007320630075727200FF
:10C4E000656E7400204C5300422073006574740024
:10C4F000696E6700293A200050726F00746F630004
:10C500006F6C3A0020736500726961006C33200023
:10C5100077697200653220007769720065524600C3
:10C5200055756E006B6E6F00776E5200656164002A
:10C530002074790070653A0020746F0020656E00E9
:10C540006476610072696100626C6500206C650050
:10C550006E6774006844610074612000756E690044
:10C5600074733A00206E6F0020696E006469630086
:10C57000617469006F6E44006174610020756E0023
:10C58000697420006C656E00677468002028620082
:10C5900069747300293A200043532000454E41003E
:10C5A000424C45004443530020444900534142005B
:10C5B0004C4544005233570020287300706420001B
:10C5C00063736C00206869007A293D0028202900E7
:10C5D0000D0A4400697363006F6E6E00656374003A
:10C5E00020616E00792064006576690063657300E0
:10C5F0000D0A43006F6E6E006563740020285600BC
:10C6000070752000746F20002B35560029206100C2
:10C610006E64200028414400432074006F202B00EA
:10C62000332E33005629430074726C004155580074
:10C630004D4F440045204C0045445000554C4C00A3
:10C6400055502000485055004C4C550050204C008F
:10C650005652450047414400432061006E6420006B
:10C6600073757000706C7900355656005055330064
:10C670002E33560041444300427573002068690020
:10C68000676842007573200048692D005A20300009
:10C6900042757300204869002D5A2000314D4F002B
:10C6A00044452000616E640020565200454720003A
:10C6B0004C45440073207300686F75006C64200063
:10C6C000626520006F6E2100466F75006E64200069
:10C6D00020657200726F7200732E4D004F53490037
:10C6E000434C4B004D4953004F435300204F4B00E8
:10C6F00020464100494C530065742000737065006A
:10C7000065643A000D0A2000312E200033304B00C2
:10C71000487A0D000A2032002E20310032354B00BD
:10C72000487A0D000A2033002E20320035304B00AD
:10C73000487A0D000A2034002E2031004D487A003E
:10C74000436C6F00636B2000706F6C006172690056
:10C7500074793A000D0A2000312E200049646C00E3
:10C7600065206C006F7720002A64650066617500A3
:10C770006C740D000A2032002E204900646C6500A4
:10C780002068690067684F00757470007574200038
:10C79000636C6F00636B200065646700653A0D0091
:10C7A0000A2031002E204900646C650020746F005F
:10C7B0002061630074697600650D0A0020322E0046
:10C7C0002041630074697600652074006F20690061
:10C7D000646C6500202A640065666100756C7400F5
:10C7E000496E70007574200073616D00706C650097
:10C7F00020706800617365003A0D0A0020312E0038
:10C80000204D690064646C0065202A006465660040
:10C8100061756C00740D0A0020322E0020456E00F8
:10C8200064535000492028007370640020636B003B
:10C83000702073006B652000736D700020637300BF
:10C840006C206800697A29003D28200020302E00E5
:10C850004D616300726F20006D656E00750D0A00FA
:10C8600020312E00536E690066662000435320007D
:10C870006C6F77000D0A2000322E53006E6966003F
:10C88000662061006C6C200074726100666669004D
:10C89000632D7000202D6600202A42007974650007
:10C8A00073206400726F7000706564002A46410056
:10C8B000494C4500442C20004E4F20004441540078
:10C8C000414461007461200062697400732061005A
:10C8D0006E64200070617200697479003A0D0A007C
:10C8E00020312E0020382C00204E4F004E452000D5
:10C8F0002A646500666175006C7420000D0A2000D2
:10C90000322E2000382C2000455645004E200D00C8
:10C910000A2033002E2038002C204F0044442000F1
:10C920000D0A2000342E2000392C20004E4F4E00DE
:10C93000455374006F70200062697400733A0D00F3
:10C940000A2031002E203100202A64006566610033
:10C95000756C74000D0A2000322E200032526500E2
:10C960006365690076652000706F6C006172690014
:10C9700074793A000D0A2000312E200049646C00C1
:10C9800065203100202A640065666100756C7400C2
:10C990000D0A2000322E200049646C006520300012
:10C9A00055415200542028007370640020627200C8
:10C9B000672064006270200073622000727870004B
:10C9C000206869007A293D0028202000302E4D0083
:10C9D000616372006F206D00656E75000D0A2000A6
:10C9E000312E540072616E007370610072656E00CA
:10C9F000742062007269640067650D000A203200CD
:10CA00002E204C0069766500206D6F006E69740001
:10CA10006F720D000A2033002E42720069646700B5
:10CA2000652077006974680020666C006F772000CD
:10CA3000636F6E0074726F006C5541005254200099
:10CA40006272690064676500526573006574200056
:10CA5000746F20006578690074526100772055007A
:10CA60004152540020696E007075740055415200A7
:10CA700054204C00495645002044490053504C0076
:10CA800041592C00207D2000544F200053544F006A
:10CA9000504C49005645200044495300504C410039
:10CAA00059205300544F5000504544005741520004
:10CAB0004E494E00473A200070696E0073206E00A8
:10CAC0006F7420006F7065006E20640072616900F1
:10CAD0006E20280048695A00292052004556490016
:10CAE000443A0D000A496E0076616C0069642000CA
:10CAF00063686F00696365002C2074007279200000
:10CB000061676100696E6D0073525300204C4F00E5
:10CB1000572C2000434F4D004D414E0044204D0006
:10CB20004F4445005253200048494700482C2000FC
:10CB30004441540041204D004F444500416464008D
:10CB40007265730073206F00662050004346380002
:10CB5000353734003F546800697320006D6F6400FE
:10CB6000652072006571750069726500732061004F
:10CB70006E20610064617000746572004C43440073
:10CB80002074790070653A000D0A2000312E2000D3
:10CB90004844340034373800302028007573690069
:10CBA0006E67200050434600383537003420490076
:10CBB0004F206500787061006E64650072294C003A
:10CBC000434420002874790070206100646472007E
:10CBD00029203D002028200020302E004D616300D8
:10CBE000726F20006D656E00750D0A0020312E00F9
:10CBF0004C43440020526500736574000D0A200008
:10CC0000322E49006E697400204C4300440D0A0026
:10CC100020332E00436C6500617220004C434400B9
:10CC20000D0A2000342E4300757273006F722000CD
:10CC3000706F7300697469006F6E200065783A0048
:10CC40002834290020300D000A2036002E577200AB
:10CC50006974650020746500737420006E756D0042
:10CC60006265720073206500783A2800362920003A
:10CC700038300D000A2037002E57720069746500A5
:10CC80002074650073742000636861007261630042
:10CC90007465720073206500783A280037292000F7
:10CCA00038304400697370006C617900206C690051
:10CCB0006E6573003A0D0A0020312E0020312000ED
:10CCC0000D0A2000322E20004D756C007469700032
:10CCD0006C6549004E495400434C450041524300A5
:10CCE000555253004F522000534554004E6F2000C0
:10CCF00041434B002C206300686563006B2061009A
:10CD00006461700074657200434C4B00094D4F0024
:10CD100053490900435309004D4953004F506900DE
:10CD20006E73740061746500733A47004E440900E5
:10CD3000332E3300560935002E3056000941440089
:10CD40004309560050550900415558000950090043
:10CD5000500950000949090049092D00094F5700A1
:10CD600044092D00092D2D000954780044092D0097
:10CD700009527800445343004C09530044410900D0
:10CD80002D092D00504743000950470044092D004C
:10CD9000092D31002E28420052290900322E280088
:10CDA0005244290009332E00284F5200290934002B
:10CDB0002E28590057290900352E2800474E2900F2
:10CDC00009362E0028424C00290937002E28500031
:10CDD00055290900382E28004752290009392E000C
:10CDE00028575400290930002E2842006C6B290076
:10CDF000474E440009474E0044094100444309009E
:10CE0000352E3000560933002E3356000956500097
:10CE1000550941005558090065786500637574002F
:10CE200065203A002020610075746F0072616E0009
:10CE3000676520002B4D48007A292B006B487A004B
:10CE40002952610077207600616C750065206600CC
:10CE50006F7220004252470020284D00494449008B
:10CE60003D3132003729570041524E00494E4700AC
:10CE70003A2050006F73730069626C006520620095
:10CE80007566660065726F0076657200666C6F008D
:10CE900077416E0079206B0065792000746F200067
:10CEA00065786900745370006163650020746F00D9
:10CEB00020636F006E7469006E7565004E756D00BD
:10CEC00062657200206F6600206269007473200042
:10CED00072656100642F770072697400653A200002
:10CEE00043533A000D0A2000312E200043530D0019
:10CEF0000A2032002E202F00435320002A646500B0
:10CF0000666175006C7450006F73690074696F001E
:10CF10006E2069006E2064006567720065657300AD
:10CF200053657200766F2000616374006976650056
:10CF300031322E002852440029093100312E2800B8
:10CF400042522900093130002E2842004C4B290062
:10CF500009392E0028575400290938002E28470087
:10CF600052290900372E28005055290009362E0075
:10CF700028424C00290935002E2847004E29090077
:10CF8000342E28005957290009332E00284F52000B
:10CF9000290932002E28520044290900312E280088
:10CFA00042522900474E440009352E0030560900F0
:10CFB000332E3300560956005055090041444300B2
:10CFC00009415500583209004155580031094100C6
:10CFD00055580900435309004D4953004F09430078
:10CFE0004C4B09004D4F5300492D09002D092D00D0
:10CFF000094F5700442D090052784400092D0900BB
:10D00000547844002D092D00095343004C09530066
:10D0100044412D00092D09005047430009504700A5
:10D02000444765006E657200616C090009090900DA
:10D03000095072006F746F00636F6C0020696E009E
:10D040007465720061637400696F6E002D2D2D0090
:10D050002D2D2D002D2D2D002D2D2D002D2D2D00B4
:10D060002D2D2D002D2D2D002D2D2D002D2D2D00A4
:10D070002D2D2D002D2D2D002D2D2D002D2D2D0094
:10D080002D2D2D002D2D2D002D2D2D002D2D2D0084
:10D090002D2D2D002D2D2D002D2D2D002D2D2D0074
:10D0A0002D2D2D002D2D2D002D2D2D002D2D2D0064
:10D0B0003F09540068697300206865006C700900BE
:10D0C00009092800302909004C69730074206300A5
:10D0D00075727200656E7400206D610063726F007E
:10D0E000733D58002F7C580009436F006E76650031
:10D0F0007274730020582F00726576006572730099
:10D100006520580009092800782909004D6163004D
:10D11000726F2000787E090053656C0066746500AC
:10D120007374090009095B0009537400617274008B
:10D1300023095200657365007409090009095D003F
:10D14000095374006F702400094A75006D70200047
:10D15000746F2000626F6F00746C6F006164650013
:10D16000720909007B095300746172007420770012
:10D170006974680020726500616426002F2509002B
:10D1800044656C006179200031207500732F6D00BB
:10D1900073090900097D090053746F0070612F0045
:10D1A000412F400009415500585049004E202800A9
:10D1B0006C6F77002F4849002F52450041442900E9
:10D1C000090922006162630022095300656E640050
:10D1D0002073740072696E00676209005365740001
:10D1E00020626100756472006174650009090900BC
:10D1F00031323300632F430009415500582061004C
:10D2000073736900676E6D00656E7400202861009D
:10D2100075782F0043532900090930007831320016
:10D2200033642F0044094D00656173007572650019
:10D2300020414400432028006F6E6300652F4300A7
:10D240004F4E54002E290900306231003130090060
:10D2500053656E0064207600616C75006566090098
:10D260004D6561007375720065206600726571001E
:10D2700075656E00637909000972090052656100E5
:10D2800064672F0053094700656E65007261740082
:10D2900065205000574D2F0053657200766F0900CE
:10D2A000092F0900434C4B002068690068094300BE
:10D2B0006F6D6D00616E640068697300746F720059
:10D2C00079090900095C0900434C4B00206C6F0090
:10D2D0006909560065727300696F6E00696E6600B9
:10D2E0006F2F730074617400757369006E666F0050
:10D2F00009095E0009434C004B20740069636B0010
:10D300006C2F4C0009426900746F720064657200F2
:10D3100020286D0073622F004C5342002909090038
:10D320002D0944004154200068696D0009436800DC
:10D33000616E670065206D006F6465000909090072
:10D340005F094400415420006C6F6F000953650071
:10D3500074206F007574700075742000747970000B
:10D3600065090900092E0900444154002072650036
:10D37000616470002F50090050756C006C7570006E
:10D380002072650073697300746F72007320280047
:10D390006F6666002F4F4E0029092100094269007F
:10D3A0007420720065616400730953006372690040
:10D3B00070742000656E6700696E650009090900D8
:10D3C0003A0952006570650061742000652E67009F
:10D3D0002E2072003A31300076095300686F7700D2
:10D3E00020766F006C7473002F7374006174650095
:10D3F000730909002E0942006974730020746F00DC
:10D400002072650061642F007772690074652000E6
:10D41000652E67002E203000783535002E327700DB
:10D420002F5709005053550020286F0066662F00C3
:10D430004F4E290009093C00783E2F003C783D0002
:10D44000203E2F003C303E000955730065726D0090
:10D45000616372006F2078002F6173007369670049
:10D460006E2078002F6C690073742000616C6C0072
:10D470000000FA00A0DE2100104078000060A0004B
:10D48000A1DE210080487800006922001040780069
:10D49000684060000004E00002003200DA82A90067
:10D4A00001003700DA82A8000069220010407800ED
:10D4B000684060000004E00003003200F0C2B300E6
:10D4C00084A2020000000000A100200060AB200048
:10D4D000E6C90200000000000080FA00000006001B
:10D4E0000000FA00A0DE2100104078000060A100DA
:10D4F000A1DE2100804878000069220010407800F9
:10D50000684060000004E00002003200DA82A900F6
:10D5100001003700DA82A80000692200104078007C
:10D52000684060000004E00003003200F0C2B30075
:10D5300084A2020000000000A100200060AB2000D7
:10D54000E6C90200000000000080FA0000000600AA
:10D550000000FA0000692200104078006840600076
:10D560000004E00002003200DA82A8000100370067
:10D57000DA82A9000069220010407800684060004B
:10D580000004E00003003200F0C2B30084A20200F5
:10D5900000000000B100200000AC2000E6C902003D
:10D5A000000000000080FA00000006000000FA0001
:10D5B00000C0EB00860207000080FB000080FA003C
:10D5C000000006000600FA00100798001E009000F8
:10D5D0007F020700004F7800A0DE21001040780095
:10D5E0000044B2000004E000030032001E80FB0093
:10D5F00020079800020037000000EB002007980089
:10D600002E0090000080FA00000006000000FA00E2
:10D6100001022000D0C920005CC902000000000007
:10D6200080DD2100104078000040E80018A10200D1
:10D630000000000000C2B30084A20200000000004D
:10D6400000692200104078006140600018A10200CB
:10D650000000000000C2B30084A20200000000002D
:10D6600000692200104078000080FB000000D1001B
:10D670006140600018A102000000000000C2B30079
:10D6800084A202000000000000692200104078001F
:10D690000080FB004200DE006140600018A1020033
:10D6A0000000000000C2B30084A2020000000000DD
:10D6B00000692200104078000080FB004300DE007B
:10D6C0006140600018A102000000000000C2B30029
:10D6D00084A2020000000000A0DE210010407800BB
:10D6E0000080FB004400DE006140600018A10200E1
:10D6F0000000000000C2B30084A20200000000008D
:10D7000031002000F0AD20005CC9020000000000E4
:10D710000080FA00000006000C00FA00FA41020046
:10D72000000000002C3E020000000000500798009E
:10D73000FA410200000000002C3E02000000000040
:10D7400040079800FA410200000000002C3E020051
:10D750000000000030079800FA41020000000000BD
:10D760002C3E02000000000020079800FA41020051
:10D77000000000002C3E020000000000000F7800B6
:10D78000FA410200000000002C3E020000000000F0
:10D79000100798005E0090000000E00009003400CF
:10D7A0005E009000E40F500006003C005E00900018
:10D7B0000040E9008040780080DD210001487800C9
:10D7C000020037000000EB00500798004E00900068
:10D7D0000000E0000F0034004E009000E20F500007
:10D7E0000C003C004E0090000040E900E140600069
:10D7F000006922001040780061C16000E1CFB300F1
:10D8000001406000024070000169220080487800F9
:10D81000020037000000EB00500798003E00900027
:10D820000000E000100034003E009000E20F5000C5
:10D830000D003C003E0090000040E90061416000A6
:10D840000069220090407800614061000041400082
:10D85000D0CFB30080C0600082C070000069220099
:10D8600001487800020037000000EB0050079800E4
:10D870002E0090000000E000100034002E00900008
:10D88000E20F50000D003C002E0090000040E90027
:10D8900061416000006922009040780061406100B1
:10D8A0004201DD00B0CFB30080C0600082C07000D4
:10D8B0000069220001487800020037000000EB00F8
:10D8C000500798001E00E0001000340020002000E7
:10D8D0009E0F10000D003C001E0078000040E90083
:10D8E0006141600000692200904078006140610061
:10D8F0004301DD0070CFB30080C0600082C07000C3
:10D900000069220001487800020037000000EB00A7
:10D91000500798001E0090000000E0001000340046
:10D920001E009000E20F50000D003C001E00900011
:10D930000040EA0061416000A0DE210090407800D4
:10D94000614061004401DD00F0CEB30080C06000A2
:10D9500082C07000A0DE210001487800020037007C
:10D960000000EB00500798005E0090000000E0000F
:10D9700079003A000000EB002008890071032000C4
:10D98000D0BB2000E6C90200000000008001EB00CF
:10D990004200200011002000100020002643020059
:10D9A000000000000040E9008040780080DD210098
:10D9B000014878005103200040BF2000E6C9020062
:10D9C000000000008001EB00220020001100200078
:10D9D0001000200026430200000000000040E90083
:10D9E000E1406000006922001040780061C16000E1
:10D9F000E1CFB300014060000240700001692200E5
:10DA0000804878003104200090C22000E6C902005E
:10DA1000000000008001EB00220020001100200027
:10DA20002000200026430200000000000040E90022
:10DA3000614160000069220090407800614061000F
:10DA400000414000D0CFB30080C0600082C07000B1
:10DA5000006922000148780011032000C0C62000A0
:10DA6000E6C90200000000008001EB002200200057
:10DA700011002000100020002643020000000000DA
:10DA80000040E90061416000006922009040780098
:10DA9000614061004201DD00B0CFB30080C0600092
:10DAA00082C070000069220001487800D101200086
:10DAB000C01A2100E6C90200000000008001EB004E
:10DAC0002200200011002000200020002643020038
:10DAD000000000000040E900614160000069220090
:10DAE00090407800614061004301DD0070CFB300D9
:10DAF00080C0600082C07000006922000148780088
:10DB0000F1042000B0932000E6C9020000000000EC
:10DB10008001EB00220020001100200010002000F6
:10DB200026430200000000000040EA00614160005E
:10DB3000A0DE210090407800614061004401DD00DA
:10DB4000F0CEB30080C0600082C07000A0DE210073
:10DB50000148780001003700ACFE0700A0DE21007C
:10DB6000104078000060A100A1DE2100804878000C
:10DB700080DD2100104078008080FB0020DF210044
:10DB80000080400010407800A600070000692200D5
:10DB9000104078000080FB004300DE006140600020
:10DBA000614060004401DD00A12D2000914078001B
:10DBB000F0CEB30000C0600002407000DAE2B700AF
:10DBC0000080FA00000006000000FA00E9000700EB
:10DBD0000080FA00000006000600FA00000F78003E
:10DBE0001E0078006101B800120798002307980012
:10DBF000F0002000010020001E019000AE01900006
:10DC0000800F5100818F590079003E001E00900066
:10DC1000AE009000006001000F00370013003700D5
:10DC20001E003700760037007100370070003700A3
:10DC30006F0037006E0037006D0037006C00370052
:10DC400022003700270037002C0037003100370052
:10DC5000360037003B00370041032000D0CB2000C6
:10DC6000E6C90200000000006500370071002000D6
:10DC700050592000E6C9020000000000F100200019
:10DC800010172100E6C902000000000011C0B30017
:10DC90000040EB00DC000700590037007100200055
:10DCA00050592000E6C9020000000000F1002000E9
:10DCB00010172100E6C902000000000011C0B300E7
:10DCC00010C0B300D00007004D00370000692200EB
:10DCD000104078000000A10001692200804878000F
:10DCE0001D00370000692200104078000000A000ED
:10DCF000016922008048780017003700006922007F
:10DD0000104078000010A1000169220080487800CE
:10DD10001100370000692200104078000010A000B8
:10DD200001692200804878000B003700006922005A
:10DD3000104078000020A10001692200804878008E
:10DD40000500370000692200104078000020A00084
:10DD500001692200804878000069220010407800A4
:10DD600061406000614060004601DD002124200028
:10DD700091407800F0CBB30000C06000024070001A
:10DD800042E2B70000692200104078000080FB00EA
:10DD90000000D1006140600061416000312420003A
:10DDA00091407800E0CFB30000C0600002407000F6
:10DDB00043E2B70000692200104078000080FB00B9
:10DDC0004200DE00614060006140600000414000B0
:10DDD0003124200091407800D0CFB30000C0600013
:10DDE0000240700043E2B70008FE0700040037005D
:10DDF00041022000C0202000E6C90200000000000F
:10DE00000080FA00000006000000FA000101200076
:10DE100030262100E6C90200000000000080FA0060
:10DE2000000006000200FA00004F780041E2A9005D
:10DE3000A0DE210010407800704060000004E00087
:10DE400004003200DE62A800DE42A800DE82A800E4
:10DE500003003700DE62A900DE42A900DE82A900CD
:10DE6000816A20009140780000CCB30000C06000BF
:10DE70007040B300A8E6B700916C20009140780094
:10DE800000CCB30000C060007040B300C9E6B7002A
:10DE9000816C20009140780000CCB30000C060008D
:10DEA0000034A000C8E6B700DA82A800D882A90032
:10DEB000D842A900D862A800D822A9001E80FB0081
:10DEC0001012880042A2A8000069220010407800C9
:10DED00061406000614060004601DD0021242000B7
:10DEE00091407800F0CBB30000C0600002407000A9
:10DEF00042E2B70000692200104078000080FB0079
:10DF00000000D100614060006141600031242000C8
:10DF100091407800E0CFB30000C060000240700084
:10DF200043E2B70000692200104078000080FB0047
:10DF30004200DE006140600061406000004140003E
:10DF40003124200091407800D0CFB30000C06000A1
:10DF50000240700043E2B7000000EB00201288008E
:10DF60000000EB000012880041E2A8000080FA00E7
:10DF7000000006000000FA0041E2A900816A2000CA
:10DF80009140780000CCB30000C06000F041B300C5
:10DF9000A8E6B700916C20009140780000CCB30057
:10DFA00000C06000C9E6B700816C20009140780095
:10DFB00000CCB30000C06000C8E6B700DE62A90074
:10DFC000DE42A900DE82A9000080FA0000000600FF
:10DFD0000200FA00004F78001E80FB00401288000B
:10DFE00085C0BF00644060000004E000FCFF320018
:10DFF00040128000004F78008540A9001E80FB0081
:10E000000080FA00000006000400FA002047980093
:10E010003147980010C0B300004F78002AA30200D7
:10E0200000000000D3FF0700820007002E40900090
:10E030000004E00002003A0042E2A80062E2A80008
:10E040002E409000E14F500002003E0041E2A80047
:10E0500061E2A8001E04E00009003A00DAC2BF0035
:10E06000704060000004E00005003200D0C5B3003D
:10E07000DEA202000000000010C0B300004F7800D4
:10E0800040C2BF000042B2000004E0002F003A008E
:10E0900060C2BF000042B2000004E0002B003A0062
:10E0A000401280001047980010C0B3009E4F10002F
:10E0B00005003A00B0C5B300DEA202000000000077
:10E0C0000040EB00004F78003E4090000004E0006C
:10E0D000050032001E4090000080FB00A4A1020059
:10E0E0000000000006003700C0C5B300DEA2020039
:10E0F000000000001E409000DEA2020000000000B0
:10E1000040138000104798003E4090000004E0005B
:10E110000B00320080C2B300DEA20200000000004B
:10E120001E4090000080FB00A4A10200000000003F
:10E1300090C2B300DEA2020000000000030037001E
:10E140001E409000DEA202000000000040C2BF009E
:10E150000044B2000004E00009003A0060C2BF00C1
:10E160000044B2000004E00005003A00D02781001E
:10E1700001402000010060000000E00014003200B7
:10E18000D027810001402000010060000000E00075
:10E1900002003A0036A30200000000000000EB007D
:10E1A000001288000000EB00001388003E40900041
:10E1B0000004E0000400320000A72A00AC9E020028
:10E1C0000000000093FF3700CB02A9000F003700CA
:10E1D00030A302000000000004A3020000000000C1
:10E1E000E14F50009BFF3A0010A302000000000026
:10E1F000104798003E4090000004E0000300320009
:10E2000010A82A00AC9E0200000000008800070051
:10E2100080DD2100104078008080FB0020DF21009D
:10E220000080400010407800FEFE07000080FA00E9
:10E23000000006000000FA00D882A800D842A8001A
:10E24000D862A800D822A800A16A200091407800D6
:10E2500000CCB30000C060006040B300AAE6B70085
:10E26000E16A20009140780000CCB30000C060005B
:10E270006040B300AEE6B700816A200091407800AC
:10E2800000CCB30000C060009040B300A8E6B70027
:10E29000916A20009140780000CCB30000C060007B
:10E2A0000034A000A9E6B700C16A200091407800C0
:10E2B00000CCB30000C060007040B300ACE6B70013
:10E2C000D16A20009140780000CCB30000C060000B
:10E2D0000034A000ADE6B70080DD210010407800DA
:10E2E0008080FB0020DF210000804000104078008B
:10E2F0000080FB00101288000069220010407800A6
:10E3000061406000614060004601DD002124200082
:10E3100091407800F0CBB30000C060000240700074
:10E3200042E2B70000692200104078000080FB0044
:10E330000000D10061406000614160003124200094
:10E3400091407800E0CFB30000C060000240700050
:10E3500043E2B7000000EB00201288000000EB0051
:10E360000012880080DD2100104078008080FB00D2
:10E3700020DF210000804000104078000080FB007A
:10E38000101388000069220010407800614060008E
:10E39000614060004601DD002126200091407800A8
:10E3A000F0CBB30000C060000240700062E2B70032
:10E3B00000692200104078000080FB000000D100BE
:10E3C000614060006141600031262000914078008A
:10E3D000E0CFB30000C060000240700063E2B7000D
:10E3E0000000EB00201388000000EB000013880001
:10E3F0000000EB00401288000000EB004013880092
:10E400004322A9006322A9004362A80042A2A900F6
:10E410006362A80062A2A90040C2A90060C2A9006C
:10E420004402A8006402A8000080FA000000060070
:10E430000000FA0041E2A9004362A90061E2A900DC
:10E440006362A900A16A20009140780000CCB3006B
:10E4500000C06000F041B300AAE6B700E16A200006
:10E460009140780000CCB30000C06000F041B300E0
:10E47000AEE6B700816A20009140780000CCB3007E
:10E4800000C06000F041B300A8E6B700916A200028
:10E490009140780000CCB30000C06000F041B300B0
:10E4A000A9E6B700C16A20009140780000CCB30013
:10E4B00000C06000F041B300ACE6B700D16A2000B4
:10E4C0009140780000CCB30000C06000F041B30080
:10E4D000ADE6B7000080FA00000006000000FA0078
:10E4E00020A82A00809E0200000000000080FA00A0
:10E4F000000006000A00FA00881F780011C0B3006F
:10E5000080DD210001487800006922001040780079
:10E510000000A10001692200804878000069220003
:10E52000104078000010A0000169220080487800A7
:10E5300000692200104078000020A100016922003B
:10E5400080487800A0DE2100104078000040A00044
:10E55000A1DE21008048780080DD21001040780095
:10E560008080FB0060DF21000080400010407800C8
:10E570002CFE0700D9FF07000000370010A302009F
:10E580000000000080407800E06822000148780028
:10E59000E0682200104078000080FB004400DE00AC
:10E5A00080407800D068220001487800D0682200BE
:10E5B000104078000080FB00400798004E0090005B
:10E5C000E40F5000EC0032004E009000E40F5000C9
:10E5D00007003C004E0090000000E0000B003200FD
:10E5E0004E009000E10F5000C00032004E01370095
:10E5F0004E009000E60F5000E70032004E00900001
:10E60000E80F5000F900320047013700E0682200AF
:10E61000104078000080FB00300798003E0090001A
:10E62000E30F5000270032003E009000E30F50003F
:10E630000A003C003E009000E10F5000170032003D
:10E640003E009000E10F500016003C003E0090009C
:10E650000000E0000F003200A00037003E009000F4
:10E66000ED0F50001E0032003E009000ED0F5000F4
:10E6700004003C003E009000E50F500097003C0075
:10E68000250037003E009000EE0F50001B003200C6
:10E690009200370037FE0700270137008FFF070081
:10E6A000B6FF3700E0168000F1FE2F000100600089
:10E6B000E016880010C0B30084A202000000000031
:10E6C000AEFF3700E01680000040A000E016880092
:10E6D00010C0B30084A2020000000000A7FF3700B2
:10E6E00010C0B30084A20200000000008040EB00D4
:10E6F00010C0B30044FE0700A0FF370010C0B300F5
:10E7000084A20200000000008040EB000040EB000B
:10E710003DFE070099FF370010A302000000000033
:10E720000080FB00100798001E0090004800DD00EC
:10E730001007980010A30200000000008080FB007A
:10E740001E009000010070001007980010A3020046
:10E75000000000000080FB00000F78001E00780021
:10E760004800DD00000F780010A302000000000048
:10E770000080FB001E0F70009E0090000000210032
:10E78000808F500003003E00000021009E0F10000B
:10E79000040036000040EB0084A2020000000000EC
:10E7A00076FF37000000EB002007980009003700D3
:10E7B000712781002E0090000084400010A3020009
:10E7C00000000000004C78002E0090000000E800DF
:10E7D00020079800AE0090001E009000808F50002F
:10E7E000F3FF3900E068220010407800E44F500049
:10E7F00001003A00DA82A9000000EB00200798002F
:10E8000008003700712781002E0090000080400032
:10E8100010407800EEFD07002E0090000000E80098
:10E8200020079800AE0090001E009000808F5000DE
:10E83000F4FF390010002000EAC6020000000000CA
:10E840000000EB00200798000900370071278100C5
:10E850002E0090000084400000C0EB00DCFD0700AB
:10E86000004C78002E0090000000E800200798007F
:10E870002E0090009E0F5000F4FF3900E068220047
:10E8800010407800E44F500001003A00DA82A800FE
:10E8900010C0B30084A20200000000000000EB00E2
:10E8A0002007980009003700712781002E00900092
:10E8B000008040001040780084A2020000000000A8
:10E8C0002E0090000000E800200798002E00900025
:10E8D0009E0F5000F4FF390028FF37000040EB0086
:10E8E00084A202000000000024FF3700E06822003C
:10E8F00090407800F0C0B30080C06000E068220063
:10E9000001487800E0682200104078008040E8006C
:10E91000E06822000148780010C0B30084A2020021
:10E92000000000008040EB00C06822000148780031
:10E930000A00370010A3020000000000A4FD070039
:10E9400084A2020000000000C0682200104078008D
:10E950008040E800C068220001487800C0682200BA
:10E9600090407800E06822001040780080CF50008E
:10E97000F0FF390001FF3700E06822001040780006
:10E98000DCCD02000000000010C0B30084A2020031
:10E9900000000000F9FE3700E06822009040780097
:10E9A00070C0B30080C06000E068220001487800B9
:10E9B000E06822009040780080DD21000148780066
:10E9C00080DD2100104078008080FB0060DF2100A6
:10E9D000008040001040780012FD070010C0B30016
:10E9E00084A2020000000000E4FE3700006922005B
:10E9F000104078000000A1000169220080487800E2
:10EA000000692200104078000010A1000169220076
:10EA10008048780000692200104078000020A100A2
:10EA20000169220080487800A0DE210010407800B3
:10EA30000040A100A1DE210080487800E0682200AB
:10EA4000104078000080FB004200DE0061006000A2
:10EA50000004E00005003200006922001040780048
:10EA60000000A0000169220080487800E0682200D0
:10EA7000104078000080FB000000D10061006000C1
:10EA80000004E00005003200006922001040780018
:10EA90000010A0000169220080487800E068220090
:10EAA000104078000080FB00610060000004E0007E
:10EAB0000500320000692200104078000020A0000C
:10EAC0000169220080487800E06822001040780048
:10EAD0000080FB004300DE000000A2006100600037
:10EAE0000004E00005003200A0DE210010407800A4
:10EAF0000040A000A1DE21008048780080DD2100D8
:10EB0000104078008080FB0060DF21000080400022
:10EB100010407800C3FC070010C0B30084A20200BC
:10EB20000000000095FE37000040EB0084A20200C8
:10EB30000000000091FE37004F0478000080FA00CA
:10EB4000000006000200FA000040EB00004F7800D1
:10EB5000503481000000E0001500320000C2B30014
:10EB600084A20200000000003100200010442000B8
:10EB70005CC902000000000000C2B30084A20200D1
:10EB800000000000403481000000E00004003A0072
:10EB90000040EB005AB702000000000002003700FE
:10EBA0000040EB00430207000000EB0050348900F6
:10EBB000403481000000E00004003A00EAB60200A0
:10EBC00000000000004F78000200370075020700C7
:10EBD000004F780010002000503489001E80FB0098
:10EBE0000080FA00000006000400FA00000F780020
:10EBF000503481000000E0001500320000C2B30074
:10EC000084A2020000000000310020001044200017
:10EC10005CC902000000000000C2B30084A2020030
:10EC200000000000403481000000E00004003A00D1
:10EC30000040EB005AB7020000000000020037005D
:10EC40000040EB001B0207000000EB00503489007D
:10EC5000403481000000E00008003A001E00780007
:10EC600096B602000000000038B702000000000065
:10EC70000080FB00000F7800050037001E007800C0
:10EC800033020700F80107000080FB00000F780046
:10EC900000C2B30084A20200000000001E00E000D9
:10ECA00007003A0031002000104420005CC9020037
:10ECB0000000000000302000100798000600370018
:10ECC00041002000404420005CC902000000000018
:10ECD00000102000100798001E0090000080FA002D
:10ECE000000006000000FA00503481000000E0003F
:10ECF0001200320041002000404420005CC90200A4
:10ED000000000000E0992A00AC9E02000000000014
:10ED1000403481000000E00004003A0010C0B3005D
:10ED20005AB70200000000000200370010C0B30014
:10ED3000E00107000000EB005034890040348100FE
:10ED40000000E00010003A00C4B50200000000001E
:10ED50000000E0000D00320091002000A023200000
:10ED60005CC9020000000000510120003024200096
:10ED70005CC9020000000000E0992A00AC9E02007D
:10ED8000000000000100370093010700D1002000BF
:10ED900080442000E6C90200000000000080FA0064
:10EDA000000006000000FA00503481000000E0007E
:10EDB0001200320041002000404420005CC90200E3
:10EDC00000000000E0992A00AC9E02000000000054
:10EDD000403481000000E00004003A0010C0B3009D
:10EDE0005AB70200000000000200370010C0B30054
:10EDF000B00107000000EB0050348900403481006E
:10EE00000000E00003003A0004B602000000000029
:10EE10000100370082010700C1002000504520009A
:10EE2000E6C90200000000000080FA0000000600B1
:10EE30000000FA0001012000205220005CC90200FD
:10EE4000000000004034810018A102000000000012
:10EE500000C2B30084A202000000000080DD210097
:10EE60001040780018A102000000000000C2B300AA
:10EE700084A2020000000000F0992A00AC9E02006B
:10EE8000000000000080FA00000006000400FA0004
:10EE90000000EB0010079800FA410200000000009B
:10EEA0002C3E02000000000010079800FA4102000A
:10EEB000000000002C3E020000000000000F78005F
:10EEC0001E0090000000E000070034001E009000CB
:10EED000E20F500004003C001E0090000000E9001A
:10EEE00040348900020037000000EB00000F78007A
:10EEF0001E00E00009003400400020009E0F1000BA
:10EF000006003C001E0078000040E90080407800C8
:10EF100080DD210001487800020037000000EB008E
:10EF2000000F78001E00E0002F003A000000EB0008
:10EF3000200889005102200010462000E6C9020086
:10EF4000000000008001EB002200200011002000E2
:10EF50001000200026430200000000000000E9002D
:10EF600040348900403481000000E0000F003A0086
:10EF7000B103200060482000E6C902000000000044
:10EF80008001EB0042002000110020001000200052
:10EF900026430200000000000040E90080407800A5
:10EFA00080DD21000148780012003700C1022000F6
:10EFB000604F20005CC90200000000008001EB00EF
:10EFC0003200200011002000100020002643020023
:10EFD000000000000040E9008040780080DD210052
:10EFE000014878000300370091FF07000000EB00A4
:10EFF00050348900A0DE2100104078000040A000BD
:10F00000A1DE210080487800403481000000E0004B
:10F010000A003A00D822A800D842A800DA42A90083
:10F02000DA22A90080DD21009040780020C0B300E2
:10F0300036B502000000000001003700740107002F
:10F040000080FA00000006000000FA000000EB005B
:10F050005034890040348100E10F500002003A0032
:10F0600007E2A90077E2A9000080FA00000006008C
:10F070000600FA00100798001E0090002007980074
:10F080002E009000E20F5000920032002E009000FF
:10F09000E20F500007003E002E0090000000E0004C
:10F0A0000B0032002E009000E10F50000D003200E6
:10F0B000BC0037002E009000E30F50009800320093
:10F0C0002E009000E40F5000AD003200B500370074
:10F0D00051032000205320005CC902000000000002
:10F0E000B40037008040EB0060002000E4B702006D
:10F0F00000000000E102200070562000E6C9020076
:10F100000000000020692200104078000004E000A8
:10F1100008003A00DAC2BF00644060000004E0006A
:10F1200010003200DAC2BF00624060000004E0005C
:10F130000C0032002069220010407800E14F50009E
:10F1400014003A00DBC2BF00624060000004E0002F
:10F1500010003A00DBC2BF00644060000004E00021
:10F160000C003A0091002000A02320005CC902009E
:10F170000000000051012000302420005CC9020082
:10F1800000000000E0992A00AC9E02000000000090
:10F19000880037000000EB00000F780046003700C1
:10F1A000403481000000E0000A003A00C4B50200CB
:10F1B000000000001E00780096B60200000000006B
:10F1C00038B70200000000000080FB001007980024
:10F1D00006003700800007001E007800DC000700F2
:10F1E000A10007000080FB00100798001E0090009F
:10F1F0000000E00028003A001E00780018C6020057
:10F200000000000080C2B30084A2020000000000E1
:10F210001E0078000080D10018C602000000000027
:10F220001E0078000000A200610060000004E00001
:10F2300004003200109A2A00809E020000000000A4
:10F240000F003700403481000000E00006003A0063
:10F25000EAB602000000000010C0B3005AB7020076
:10F260000000000003003700CE00070010C0B3000C
:10F2700090000700409A2A00809E020000000000D3
:10F28000F0992A00809E02000000000000C2B30036
:10F2900084A2020000000000403481000000E00071
:10F2A00003003A0004B6020000000000010037002D
:10F2B0005B0007001E0FE800F00F20009E0F1000FB
:10F2C000B7FF3400E0992A00AC9E02000000000065
:10F2D0003800370040348100E10F500001003A004F
:10F2E00007E2A9007100200050592000E6C9020081
:10F2F00000000000F100200010172100E6C9020004
:10F300000000000010C0B300D400070040348100AA
:10F31000E10F500027003A00BD000700250037002C
:10F32000709A2A00AC9E02000000000011C0B300D9
:10F3300020692200014878000742A9000782A9003D
:10F340000000EB00501088000000EB006010880007
:10F350000702A90080DD2100104078008080FB00BA
:10F360003069220000804000104078000080FB00DF
:10F370002010880007E2A80077E2A9000D003700FE
:10F380002069220010407800E14F500009003A0047
:10F39000F09C2A00AC9E020000000000DB62A90085
:10F3A0000400370041022000C0202000E6C902000E
:10F3B000000000000080FA00000006000000FA00D3
:10F3C000B100200070282100E6C902000000000002
:10F3D0000080FA00000006000000FA002069220008
:10F3E000104078000004E00006003A007602A80011
:10F3F00076C2BF00614060000004E000FCFF3A00FC
:10F40000050037000602A80006C2BF006140600088
:10F410000004E000FCFF3A000080FA000000060053
:10F420000000FA0020692200104078000004E0008B
:10F4300006003A007642A80076C2BF006440600031
:10F440000004E000FCFF3A00050037000642A80077
:10F4500006C2BF00644060000004E000FCFF3A0008
:10F460000080FA00000006000200FA002069220075
:10F47000104078000004E00006003A0079C2BF00A6
:10F480000080FB004700DE000080FB00000F7800DA
:10F490000500370009C2BF000080FB004700DE0006
:10F4A0000080FB00000F78001E0078000080FA004A
:10F4B000000006000200FA00004F780020692200D8
:10F4C000104078000004E00010003A009E407800F0
:10F4D00061C06000614060004501DD0061272000DF
:10F4E00091407800F0CDB30000C060000240700091
:10F4F00076E2B7007682A80076C2BF007040600056
:10F500000004E000FCFF3A000F0037009E40780046
:10F5100061C06000614060004501DD0061202000A5
:10F5200091407800F0CDB30000C060000240700050
:10F5300006E2B7000682A80006C2BF007040600065
:10F540000004E000FCFF3A000080FA000000060022
:10F550000200FA00004F7800206922001040780075
:10F560000004E00007003A001E80FB0090138800B2
:10F5700079C2BF000044B2000004E000FCFF3A0082
:10F58000060037001E80FB001010880009C2BF0073
:10F590000044B2000004E000FCFF3A000080FA00E2
:10F5A000000006000400FA002069220010407800E4
:10F5B0000004E0000A003A007662A80076C2BF00AC
:10F5C000684060000004E000FCFF3A008013800007
:10F5D000004F78001E80FB001007980009003700DC
:10F5E0000662A80006C2BF00684060000004E00098
:10F5F000FCFF3A0000108000004F78001E80FB00E6
:10F60000100798001E0090000080FA00000006001D
:10F610000000FA007742A9007782A9000000EB0001
:10F62000D01388000000EB00E01388007702A900E7
:10F6300080DD2100104078008080FB0030692200CE
:10F6400000804000104078000080FB00A01388007C
:10F6500077E2A8000080FA00000006000A00FA0025
:10F66000004F98000040EB00204798000040EB005E
:10F67000104798000040EB00004F78002AA30200DA
:10F6800000000000D822A800D842A800DA42A90051
:10F69000DA22A9006640A8006660A8008660A9007A
:10F6A000DAC2BF000080FB000000D10061406000B2
:10F6B000604798006E40900050479800DAC2BF0043
:10F6C0000080FB004200DE0061406000604798005F
:10F6D0006E409000304798000000370086C0BF00A1
:10F6E000684060000004E0000F003A0030A3020010
:10F6F0000000000004A30200000000000004E0007D
:10F70000F6FF320010A3020000000000004F780056
:10F710006640A9006660A9000E4890000004E00061
:10F7200063003A00650037008660A900DAC2BF00B6
:10F730000080FB000000D10061406000604798003D
:10F74000DAC2BF000080FB004200DE0061406000C2
:10F75000404798002E4090000004E0002E00320048
:10F760003E4090000004E0002B003A004E40900024
:10F770000004E000280032001E409000E74F5000D7
:10F780000B003E001E40780000404000004F780013
:10F790006E4090000004E000010032001E04A00052
:10F7A0001E4090000040E800104798003B003700E2
:10F7B0000E4890000004E000040032001E80FB00B0
:10F7C000A4A102000000000006003700C0C5B3007D
:10F7D000DEA20200000000001E407800DEA202004F
:10F7E000000000006E4090000004E00004003200C1
:10F7F000D0C2B300DEA20200000000000300370008
:10F80000B0C2B300DEA20200000000000040EB0026
:10F8100010479800210037003E4090000004E000AF
:10F820001E0032004E4090000004E0001B00320039
:10F830005E4090000004E0000B0032006E4090003B
:10F840000004E00008003A0010C0B3002047980010
:10F850000040EB0010479800B0C5B300DEA20200E4
:10F86000000000000D0037005E4090000004E00042
:10F870000A003A006E4090000004E00007003200E9
:10F880000040EB00204798000040EB001047980034
:10F89000D0C5B300DEA20200000000006E40900060
:10F8A000504798004E409000304798008BFF37003B
:10F8B000E0992A00AC9E0200000000000080FA00DF
:10F8C000000006000000FA00609F2A00809E0200EF
:10F8D000000000000080FA00000006000A00FA00A4
:10F8E000881F7800D822A800D842A800DA42A900D0
:10F8F000DA22A900D882A900A0DE210010407800F9
:10F900000040A000A1DE210080487800A0DE210098
:10F91000104078000030A100A1DE2100804878006E
:10F9200080C0EB0020C0B30036B50200000000002C
:10F93000E4FF07000000370010A3020000000000F1
:10F9400080407800606822000148780060682200EA
:10F95000104078000080FB004400DE00804078000A
:10F96000506822000148780050682200104078005A
:10F970000080FB00400798004E009000E10F50000F
:10F98000F40032004E009000E10F500004003C00F3
:10F990004E0090000000E000080032002F01370008
:10F9A0004E009000E40F5000240132004E00900001
:10F9B000E60F500012013200280137006068220073
:10F9C000104078000080FB00300798003E00900057
:10F9D000E40F5000330032003E009000E40F50006E
:10F9E00011003C003E009000E10F50001F0032006B
:10F9F0003E009000E10F500004003C003E009000EB
:10FA00000000E00019013200CE0037003E009000F7
:10FA1000E20F5000170032003E009000E30F50004C
:10FA20001A003200C70037003E009000E70F500078
:10FA3000280032003E009000E70F500004003C0018
:10FA40003E009000E60F50001B003200BD00370062
:10FA50003E009000E80F5000250032003E0090006C
:10FA6000EF0F5000B1003200B600370095FF0700DD
:10FA7000B1FF3700C4B502000000000010C0B300A1
:10FA800084A2020000000000ABFF370004B60200B1
:10FA90000000000010C0B30084A2020000000000BB
:10FAA000A5FF3700EAB602000000000084A20200B1
:10FAB00000000000A0FF37000040EB005AB7020032
:10FAC0000000000010C0B30084A20200000000008B
:10FAD00099FF370010C0B3005AB7020000000000C1
:10FAE00010C0B30084A202000000000092FF3700A3
:10FAF00004A30200000000000004E000FCFF32004C
:10FB000010A30200000000000080FB001007980016
:10FB10001E0090004800DD001007980004A30200BA
:10FB2000000000000004E000FCFF320010A302000F
:10FB3000000000008080FB001E00900001007000AB
:10FB40001007980004A30200000000000004E00079
:10FB5000FCFF320010A30200000000000080FB0048
:10FB6000000F78001E0078004800DD00000F7800CC
:10FB700004A30200000000000004E000FCFF3200CB
:10FB800010A30200000000000080FB001E0F7000A8
:10FB90009E00900000002100808F500003003E0076
:10FBA000000021009E0F1000040036000040EB0012
:10FBB00084A20200000000005FFF37000000EB009D
:10FBC000200798000D00370004A302000000000089
:10FBD0000004E000FCFF3200712781002E0090003D
:10FBE0000084400010A3020000000000004C7800D8
:10FBF0002E0090000000E80020079800AE00900062
:10FC00001E009000808F5000EFFF3900C4B5020045
:10FC1000000000000000EB00200798000E003700F5
:10FC2000712781002E009000008040001040780075
:10FC30000080FB0096B602000000000038B702000A
:10FC400000000000E14F5000D8FF32002E0090006D
:10FC50000000E80020079800AE0090001E00900011
:10FC6000808F5000EEFF39001E00E9001007980059
:10FC70000000EB0020079800140037007127810076
:10FC80002E00900000844000EAB602000000000050
:10FC9000004C7800AE0090001E009000808F500055
:10FCA000040031000040EB005AB7020000000000E1
:10FCB0000300370010C0B3005AB702000000000074
:10FCC0002E0090000000E800200798002E00900011
:10FCD0009E0F5000E9FF390004B60200000000004A
:10FCE00010C0B30084A20200000000000000EB007E
:10FCF0002007980009003700712781002E0090002E
:10FD0000008040001040780084A202000000000043
:10FD10002E0090000000E800200798002E009000C0
:10FD20009E0F5000F4FF390003FF37000040EB0046
:10FD30004AFE070010C0B30084A2020000000000C9
:10FD4000FDFE37000040EB0084A20200000000002E
:10FD5000F9FE37006068220090407800F0C0B300E0
:10FD600080C060006068220001487800606822005E
:10FD7000104078008040E800606822000148780068
:10FD800010C0B30084A20200000000008040EB001D
:10FD900040682200014878001200370004A30200E6
:10FDA000000000000004E000FCFF320010A302008D
:10FDB000000000000080FB0096B60200000000007A
:10FDC00038B702000000000084A20200000000001A
:10FDD00040682200104078008040E800406822001F
:10FDE0000148780040682200904078006068220056
:10FDF0001040780080CF5000E8FF3900CEFE370079
:10FE0000606822009040780030C0B30080C060007D
:10FE10006068220001487800606822009040780005
:10FE200020C0B30036B502000000000010C0B300CF
:10FE300084A2020000000000BFFE370060682200BC
:10FE400010407800DCCD02000000000010C0B300BC
:10FE500084A2020000000000B7FE37000040EB0063
:10FE600084A2020000000000B3FE37004F047800B7
:10FE70000080FA00000006000A00FA00100798004F
:10FE80002107980032079800430798001E00900051
:10FE9000202889002E009000302889003E00900024
:10FEA000402889004E009000502889000000EB0097
:10FEB000B02488009424A8009424A9009EC0A9001E
:10FEC0000000EB0060248800F00F20007024880000
:10FED000F00F2000502488000000EB00302588003F
:10FEE0000000EB004025880000E021004800DE0013
:10FEF000C024880000082000302488008804A8005E
:10FF00000000EB00602889000000EB0070288900E9
:10FF10000000EB00802889000000EB00000F780053
:10FF20000E0037001E0078004200DD008080E800EF
:10FF300020512200808040000000EB008008780003
:10FF40001E007800C200DD002051220080804000A9
:10FF50000000EB00800878001E0FE8001E0078000B
:10FF6000EF0F5000EFFF36008000EB000000EB00C9
:10FF7000E20307008000EB000000EB00EA0307004B
:10FF8000D0002000502588000000EB00902A890056
:10FF90008040EB0060552200014878000000EB0033
:10FFA000A02A89008040EB007055220001487800AB
:10FFB00081C0B30000E021000148780080E1210009
:10FFC00010F0880081C8B30010E0210001487800DB
:10FFD0008040EB0040E021000148780000E2210071
:10FFE00030F0880001C4B30050E0210001487800DF
:10FFF0000080FA00000006000000FA00010037004F
:020000040001F9
:100000009404A80094C4BF00614060000004E000B4
:10001000FBFF320011C0B300605522000148780098
:1000200094C4BF000044B2000004E000FCFF3A00AA
:1000300041C0B30060552200014878000080FA00FA
:10004000000006000000FA00020007000080FA002D
:10005000000006000000FA008AC4BF006140600092
:100060000004E0000300320023000700100020001D
:10007000502488008AC4BF00624060000004E00091
:1000800004003200F00F20007024880020002000BF
:10009000502488008AC4BF00684060000004E0006B
:1000A0000300320070000700800020005024880008
:1000B0008AC4BF00644060000004E0000700320012
:1000C000602881000000E00002003200602881000A
:1000D0000000010040002000502488000080FA0049
:1000E000000006000000FA00F00F200070248800D5
:1000F0000080FA00000006000200FA000000EB0099
:10010000902A890080002000502488000000EB0025
:10011000A02A890041C0B300605522000148780040
:100120008040EB0070552200014878008AC4BF006F
:10013000684060000004E000F2FF3A000000EB00BD
:10014000502588000000EB00602588000000EB00CF
:10015000702588000000EB00802588000000EB007F
:10016000902588000000EB00A02588000000EB002F
:10017000B02588000000EB00C02588000000EB00DF
:10018000D02588000000EB00E02588000000EB008F
:10019000F02588000000EB00002688000000EB003E
:1001A000102688000000EB00202688000000EB00ED
:1001B000302688000000EB00402688000000EB009D
:1001C000B0248800F00F200050248800F00F200099
:1001D000702488000000EB00000F78000800370052
:1001E0001E007800C200DD0000E021008080400099
:1001F0000040EB00904098001E007800640F400023
:100200001E007800E50F5000F5FF3600D0002000FA
:100210005025880081C0B30000E02100014878002B
:1002200080E1210010F0880081C8B30010E02100B7
:10023000014878008040EB0040E021000148780050
:1002400000E2210030F0880001C4B30050E021003A
:1002500001487800F00F20008024880094A4A900B1
:100260000080FA00000006000200FA0090248000DE
:1002700080407800E04F220001487800E04F2200E3
:10028000104078000080FB004300DE000080FB008F
:100290004200DD008000780000E021000080400086
:1002A00000288900E04F2200104078000034A000B0
:1002B0000080FB004300DE000080FB004200DD0008
:1002C0008000780000E021000080400010288900B4
:1002D00000288100104090008080FB00C0032000B7
:1002E00080806000010F7800400220009E007800AE
:1002F000808F50000C003200400320009E007800E8
:10030000808F5000040032001E007800E40F50007F
:100310000300320005003700060007000300370025
:10032000C802070001003700AC0207000080FA0095
:10033000000006000800FA001128810080C0B30008
:100340009040980094A4A90000288100100090001B
:10035000104078008080FB00000620008080600054
:100360003107980000022000BE009000808F5000EE
:100370002300320000042000BE009000808F500057
:10038000250032003E0090000000E0000100320035
:1003900027003700002881001000900010407800EE
:1003A0000080FB006300600020079800AE00900012
:1003B000E18F50000A0032002E009000E20F500042
:1003C0000A003200AE0090000100E000010032009F
:1003D00009003700002881003700070015003700AA
:1003E00000288100740107001200370000288100F6
:1003F000B50107000F003700060307000D003700A6
:10040000702881000000E0000A003200702881009E
:100410000000010007003700802881000000E00094
:100420000400320070288100000001000100370044
:10043000F80207000128810080C0B30080487800DE
:10044000002881001007980000288100100090000B
:10045000104078000004E0000F0035000028810003
:100460001000900066004000104078000004E0009A
:1004700006003A000028810010009000670040004C
:10048000104078000004E0000300320081CCB3008B
:10049000014F78000200370080C8B300004F780099
:1004A0001E4078009E0090009040980094A4A900FF
:1004B0000080FA00000006000A00FA0020079800F9
:1004C0002E00900090009000110798001E009000F0
:1004D0000000E800104078000080FB004007980012
:1004E0004E009000E50F500042003200CE00900018
:1004F000E58F50000A003C004E009000E10F5000D4
:100500001F003200CE009000E38F50002B0032001D
:100510004E0090000000E0000B0032002301370085
:10052000CE009000E88F5000FC0032004E0090009A
:10053000E90F500001013200CE009000E68F50001C
:10054000440032001901370010288100900090000B
:10055000902A8100804878001028810010009000C7
:100560008000E800902A81004800DE008048780082
:100570001028810021002000980207000C0137009C
:100580001E0090000080E80010407800E14F50000D
:1005900008003A00912A8100D0FF2F0000806000FF
:1005A000902A8900102881008000EB008B02070050
:1005B000FF00370097020700FD0037001E00900083
:1005C0000080E80010407800E14F500007003A003A
:1005D000902A81000010A000902A89001028810034
:1005E0008000EB007D020700F10037008902070060
:1005F000EF0037001E0090006300400010407800BC
:100600000004E00011003A001E0090000080E800A5
:10061000104078000004E0000C0035001E0090003F
:100620000080E80090407800705522000148780072
:10063000102881008000EB0068020700218228005A
:100640000000EB002D020700D900370071020700FF
:10065000D70037001E009000630040001040780073
:100660000080FB00300798003E009000E20F500031
:100670001F003200BE009000E38F50006F00320078
:100680003E009000E10F5000010032009D00370055
:1006900020288100C02A890020288100104078008D
:1006A0000080FB00D02A89001E00900067004000F7
:1006B000104078000004E00093003A001E00900013
:1006C0006600400090407800C02A81001040780009
:1006D00080CF50008C0031001E009000660040006A
:1006E000104078000080FB00D02A89008600370087
:1006F0001E0090000080E8009040780020288100D3
:10070000710040001040780080CF50000100390097
:100710004002070030288100C02A8900C02A8100D9
:100720000080E800104078008080FB00C02A810033
:1007300063004000104078000080FB004800DD00AE
:1007400000804000D02A89000000EB00000F7800F4
:1007500010003700C12A8100D02A810000804000AB
:10076000C02A8900C02A81000080E800104078007B
:100770008080FB00C02A81006300400010407800A8
:100780000080FB004800DD0000804000D02A890086
:100790001E0FE8001E0090000080E8001040780066
:1007A0000080FB009E0F5000EAFF3C001E009000FE
:1007B0006700400090407800C02A8100630040003C
:1007C0001040780080CF5000100039001E009000CB
:1007D0006700400090407800C02A8100630040001C
:1007E0001040780080CF500047003A001E00900073
:1007F0006600400090407800C02A81000080E80038
:100800001040780080CF50003F0031001E00900063
:1008100066004000104078008080FB001E009000C1
:1008200067004000104078000080FB004800DD00B9
:1008300000804000D02A8900330037001E0090005D
:100840000080E800104078008080FB005028810084
:10085000808F500001003500EE0107004028810024
:10086000C02A8900C02A8100104078000080FB0067
:10087000D02A89000000EB00000F78000900370043
:10088000C12A8100D02A810000804000C02A89004E
:10089000C02A8100104078000080FB00D02A890027
:1008A0001E0FE8001E0090000080E8001040780055
:1008B0000080FB009E0F5000F1FF3C001E009000E6
:1008C00067004000104078000004E0000E003A008D
:1008D0001E0090006600400090407800C02A810011
:1008E0001040780080CF5000070031001E009000BB
:1008F00066004000104078000080FB00D02A89008C
:1009000001003700C3010700E60107002185280028
:100910000000EB0079010700250037001028810056
:1009200090009000A02A8100804878001028810063
:1009300011002000A90107001D0037001E009000D3
:100940000080E80010407800E14F500015003E00A4
:100950001E0090000080E800104078000080FB003E
:10096000A02A8900A02A81000000E00006003200D1
:1009700001C2B3006055220001487800F4A30200D0
:10098000000000000300370001C1B30060552200E1
:1009900001487800102881008000EB008F010700DB
:1009A000030037009B010700010037009901070091
:1009B0000080FA00000006000600FA001007980008
:1009C0001E00900090009000010F78001E00E800CB
:1009D000104078000080FB00200798002E00900057
:1009E0000000E0000A003200AE0090000100E000CC
:1009F000320035002E009000EA0F50001100320046
:100A0000AE009000EB8F50001D0032002B0037002D
:100A100010288100900090000040EB008048780092
:100A200010288100100090008000E8000040EB00DA
:100A3000804878001028810021002000670107000D
:100A40001F0037009E00780064804000104078004E
:100A5000E14F500008003E001028810090009000F7
:100A60000040EB0080487800102881001100200031
:100A70005A01070012003700660107001000370016
:100A80009E0078006480400010407800E14F5000E4
:100A900008003E001E80E800104078000004E000DE
:100AA00004003A00102881008000EB004B01070091
:100AB0000300370057010700010037005501070008
:100AC0000080FA00000006000A00FA0030079800D3
:100AD0003E00900090009000210798002E009000AA
:100AE0000000E800104078000080FB0040079800FC
:100AF0004E009000E10F500038003200CE00900010
:100B0000E38F5000670032004E0090000000E000CC
:100B1000010032008300370010288100900090000F
:100B20000040EB0080487800102881001000900001
:100B30008000E8000040EB00804878002E00900024
:100B400064004000104078006F406000304798001B
:100B50002E00900064004000104078000080FB00F0
:100B60004700DE00204798003E4090000080FB00D8
:100B700000004000800078002E4090000080FB00C4
:100B8000008040004200DD008000780000E021008D
:100B9000008F40001E00780090409000B0CFB3005E
:100BA00080C060001E007800114098001E00780090
:100BB000104090000004E000040032001028810082
:100BC0009000900010C0B300804878001028810089
:100BD0002100200001010700530037002E00900083
:100BE00064004000104078006F406000304798007B
:100BF0002E00900064004000104078000080FB0050
:100C00004700DE00204798003E4090000080FB0037
:100C100000004000800078002E4090000080FB0023
:100C2000008040004200DD008000780000E02100EC
:100C3000008F40001E00780090409000B0CFB300BD
:100C400080C060001E007800114098002E40900087
:100C50000004E000060032001E0078009040900082
:100C600000C4B30080C070001E00780011409800DE
:100C70002E4090000004E00006003A001E007800BC
:100C800090409000F0CBB30080C060001E00780060
:100C900011409800102881008000EB00CF00070071
:100CA000210037002E0090006400400010407800C2
:100CB0006F406000304798002E00900064004000B4
:100CC000104078000080FB004700DE0020479800BD
:100CD0003E4090000080FB00000040008000780053
:100CE0002E4090000080FB00008040004200DD00AC
:100CF0008000780000E02100008F40001E00780096
:100D000010409000804078000124A0001E00780070
:100D100011409800102881008000EB00AF00070010
:100D200001003700BB0007000080FA000000060049
:100D30000200FA008AC4BF00614060000004E000C5
:100D400006003200ECFC0700100020005024880050
:100D5000F00F2000000F78001D0037008AC4BF008C
:100D6000684060000004E00017003200902480001A
:100D700080407800E04F220001487800E04F2200D8
:100D8000104078000080FB004400DE000080FB0083
:100D90006F0060000000E0000600320032FD070036
:100DA00080002000502488000000EB00000F780035
:100DB0000700370080002000502488000000EB006E
:100DC000000F7800020037000000EB00000F7800F1
:100DD0001E0078000080FA00000006000000FA0003
:100DE000E04F2200104078000080FB004400DE004D
:100DF0000080FB006F006000C200DD002051220077
:100E000000804000100078000000E0000B0032007D
:100E1000E04F2200104078000080FB004400DE001C
:100E20000080FB006F006000C200DD002051220046
:100E30000080400010007800000001000080FA00EF
:100E4000000006000000FA00E04F22001040780089
:100E50000080FB004400DE000080FB006F006000AB
:100E60004200DD008080E800205122000080400028
:100E7000100078000000E0000C003200E04F22007B
:100E8000104078000080FB004400DE000080FB0082
:100E90006F0060004200DD008080E80020512200E9
:100EA0000080400010007800000001000080FA007F
:100EB000000006000200FA00000F78001E00780013
:100EC000602889000080FA00000006000200FA0095
:100ED000000F78001E007800702889000080FA005A
:100EE000000006000200FA00000F78001E007800E3
:100EF000802889000080FA00000006000400FA0043
:100F0000000F7800110798001E007800C200DD0075
:100F100020512200008040009E00900001087800CF
:100F20000080FA00000006000400FA00000F7800BC
:100F3000110798001E0078004200DD008080E80064
:100F400020512200008040009E009000010878009F
:100F50000080FA00000006000200FA00000F78008E
:100F60001E0078009040900000C4B30000C06800EC
:100F700002C4B3008240600080C8B30000C07000AB
:100F8000804078001E007800114098000080FA0030
:100F9000000006000200FA00000F78009E007800B2
:100FA0000040EB00804878001E00780090409000E0
:100FB00000C4B30000C0680002C4B30082406000F7
:100FC00080C8B30000C07000804078001E00780028
:100FD000114098000080FA00000006000400FA00AA
:100FE000000F7800110798001E00900080407800E4
:100FF00000C0EB0080C060001E007800014878004F
:101000009E00780080CCB300904098000080FA00E9
:10101000000006000000FA0081C0B30000E02100DB
:101020000148780041C8B30050E021000148780031
:1010300041C8B30010E02100014878000080FA00A8
:10104000000006000000FA007055220010407800F1
:101050000004E00004003A0041C0B30060552200E3
:10106000014878000300370001C1B3006055220039
:101070000148780070552200104078000080FB0085
:10108000B024880080C0EB00705522000148780031
:101090008000EB000000EB0098FF07000080FA00E2
:1010A000000006000600FA00D02A81000000E000DF
:1010B0001C003200D02A8100200798002E009000EA
:1010C000E80F50000200360083002000230798003C
:1010D0002E009000000F78000000EB001007980031
:1010E0000C00370010288100900090001E00900036
:1010F00000814000C12A81001E0090000080400055
:1011000010407800004978001E0090000000E800C0
:10111000100798001E0090009E0F5000F1FF39004C
:10112000050037000000EB00000F78008000EB00A6
:101130000000EB0071FF0700112881001E007800FD
:10114000804878001228810010288100904090008B
:1011500000C4B30000C0680003C4B3008340600053
:1011600080C8B30000C0700010419800C12A8100FF
:101170001E00780000804000C02A8900D02A81002B
:101180001E005000D02A89000080FA0000000600EE
:101190000000FA0086C80200000000000080FB008A
:1011A0000080FA00000006000200FA00000F78003C
:1011B0001E007800EEC702000000000000102000B2
:1011C0000080FA00000006000000FA00ECC80200EF
:1011D000000000000080FB000080FA000000060014
:1011E0000000FA00A0422200104078004CC8020023
:1011F000000000000080FA00000006000000FA0075
:10120000A0422200104078000080FB000080FA001D
:10121000000006000000FA008040EB00A04222001F
:101220000148780041022000B0002000E6C9020019
:10123000000000000080FA00000006000000FA0034
:1012400011C0B300A04222000148780041022000F2
:10125000B0002000E6C90200000000000080FA0093
:10126000000006000000FA00A0DE21001040780017
:101270000040A000A1DE2100804878008040EB0003
:10128000C043220001487800D822A800DA22A90031
:10129000E1022000F0022000E6C902000000000088
:1012A0000080FA00000006000400FA00881F7800A1
:1012B000000F78001E00E0004400320020032000F0
:1012C0009E0F100041003E001E0FE900C0432200A7
:1012D000104078000080FB009E0F500005003E008B
:1012E00091022000D0052000E6C9020000000000A5
:1012F00063013700E1002000600820005CC90200A3
:10130000000000001E0078000040E80018A1020064
:101310000000000080A82A00809E0200000000005B
:101320008040EB0060432200014878001F00370036
:101330001E01780060432200104078008080FB008E
:101340004310DD0081004000D043220000804000B7
:10135000104078000080FB0018C60200000000006A
:1013600000C2B30084A20200000000001E01780049
:1013700060432200104078008080FB004310DD00B5
:1013800081004000D04322000080400010407800DF
:10139000EEC7020000000000604322001040780009
:1013A0008040E8006043220001487800604322004A
:1013B00010407800E74F5000DDFF3600B0A82A004B
:1013C000AC9E0200000000002D0137001E007800D6
:1013D00010079800500520009E009000808F50005C
:1013E00011013200500520009E009000808F5000B7
:1013F00008003E001E0090000000E00012003200D5
:10140000300320009E009000808F5000DD003200ED
:1014100017013700C00E20009E009000808F500002
:1014200063003200000F20009E009000808F50006B
:101430005F003200C00C20009E009000808F5000A2
:10144000020132000A013700D100200040092000CB
:10145000E6C902000000000071012000100A20000F
:10146000E6C9020000000000C043220010407800DE
:101470000004E00005003A0091022000D0052000A1
:10148000E6C9020000000000440037008040EB0085
:1014900070432200014878003A00370000C2B300D0
:1014A00084A2020000000000704322001040780077
:1014B0000040E80018A1020000000000C0A82A00B7
:1014C000809E0200000000008040EB00604322008C
:1014D0000148780016003700704322001040780061
:1014E0000081FB0060432200104078008080FB00F8
:1014F0004310DD0081004000D04322000080400006
:10150000104078000080FB0018C6020000000000B8
:1015100000C2B30084A20200000000006043220069
:10152000104078008040E8006043220001487800C5
:101530006043220010407800E74F5000E6FF36007D
:1015400061002000800B20005CC902000000000048
:1015500070432200104078000080FB00C300DD00D3
:10156000D04322000080400010407800F7000700C0
:1015700070432200104078008040E8007043220051
:1015800001487800C0432200904078007043220058
:101590001040780080CF5000C0FF3E00310D200089
:1015A000E00B2000E6C9020000000000B400370094
:1015B0001E00780080407800801A220001487800E0
:1015C000C00E20009E0F100005003A0031012000DF
:1015D00010192000E6C902000000000004003700D6
:1015E000D1002000401A2000E6C9020000000000DF
:1015F00071012000100A2000E6C90200000000006E
:101600008040EB0060432200014878000A01070097
:101610008040780070432200014878008040EB0051
:10162000C0432200014878004D00370000C2B300DB
:1016300084A20200000000006043220010407800F5
:101640000040E80018A1020000000000C0A82A0025
:10165000809E0200000000000000EB00A021890035
:101660000D003700A1218100D048220000804000F9
:10167000104078000080FB0018C602000000000047
:1016800000C2B30084A2020000000000A02181007B
:101690000000E800A0218900A0218100E70F500090
:1016A000F0FF360061002000800B20005CC90200C2
:1016B00000000000D048220010407800A30007007E
:1016C0006043220010407800E94F50001B003E00AC
:1016D0000000EB00A021890010003700C043220069
:1016E000104078008081FB00A4218100A1218100AD
:1016F000D048220000804000104178004318DD00EF
:1017000084004000D043220000804000024878005E
:10171000A02181000000E800A0218900A021810013
:10172000E70F5000EDFF3600C04322001040780064
:101730008040E800C0432200014878006043220056
:10174000104078008040E8006043220001487800A3
:10175000C7000700804078007043220001487800ED
:1017600070432200104078000004E000AFFF3A0010
:10177000B1022000101B2000E6C90200000000009A
:101780003F0037004800070011012000C01D200065
:101790005CC902000000000030C3B300EEC70200C5
:1017A000000000000000EB00A021890014003700B9
:1017B000A821810086C80200000000008040780057
:1017C000B04222000000440001487800A1218100BD
:1017D000B042220000804000104078000080FB00F2
:1017E00018C602000000000000C2B30084A202007C
:1017F00000000000A02181000000E800A021890075
:10180000A0218100E70F5000E9FF3600B0A82A00B0
:10181000AC9E020000000000B042220010407800A0
:101820004A000700160037001F00070001012000D2
:10183000D01E2000E6C902000000000050C5B30021
:10184000EEC70200000000000D0037001600070080
:10185000F1002000D01F2000E6C9020000000000B7
:10186000C0CCB300EEC70200000000000400370047
:1018700041022000C0202000E6C902000000000054
:101880004F0478000080FA00000006000000FA0013
:101890009100200030272100E6C90200000000006E
:1018A0000080FA00000006000200FA0068C702008B
:1018B00000000000004F7800A1002000002320005D
:1018C0005CC90200000000001E04E00005003A00B0
:1018D0003100200050BB2000E6C9020000000000DB
:1018E0001800370091002000A02320005CC90200EE
:1018F000000000001E80FB00610060000004E000AA
:101900000400320051012000302420005CC9020094
:10191000000000001E80FB000000D100610060009C
:101920000004E00004003200410120008025200076
:101930005CC9020000000000B0A82A00AC9E0200B2
:10194000000000000080FA00000006000400FA0019
:10195000004F78001E80FB00100798002002200036
:101960009E009000808F50001E0032002002200058
:101970009E009000808F500007003C001E009000E9
:10198000E40F50001C0032009E009000F08F5000C9
:101990000A00320022003700800220009E009000E2
:1019A000808F50000A003200D00220009E0090007C
:1019B000808F50001500320019003700B10120005F
:1019C000C0262000E6C90200000000001800370011
:1019D000A101200070282000E6C9020000000000DC
:1019E0001300370051012000102A2000E6C9020030
:1019F000000000000E00370081012000602B200055
:101A0000E6C90200000000000900370001012000C3
:101A1000E02C2000E6C902000000000004003700AE
:101A2000E1002000E02D20005CC902000000000061
:101A30000080FA00000006000000FA008040EB0081
:101A400050492200014878008040EB007049220094
:101A5000014878008040EB0060492200014878008E
:101A6000080007000080FB000080FA00000006006C
:101A70000000FA00030007000080FB000080FA006D
:101A8000000006000A00FA0010C0B300704798007A
:101A90000040EB00604798000040EB005047980082
:101AA00010C0B300104798000040EB00404798007A
:101AB0008040EB00804922000148780070492200F4
:101AC000104078000004E0009A003A0068C7020065
:101AD000000000000004E0000C0032008040EB0039
:101AE00050492200014878008040EB0070492200F4
:101AF000014878008040EB006049220001487800EE
:101B00000000EB00400798009F003700801A220079
:101B100010407800EEC7020000000000ECC8020090
:101B20000000000030479800ECC8020000000000F0
:101B3000204798003E409000E14F500003003A00DB
:101B40002E409000E14F500066003200BE409000F1
:101B50002E40900080CF500003003200BE40900025
:101B6000014F78002600370050492200904078004D
:101B70007E409000814F50000E0031005E4090008A
:101B80008080FB00D0482200008040009040780018
:101B90001E40900080C060000040EB00004F7800C5
:101BA0000104E0000C00320010C0B300004F7800C8
:101BB0000900370050492200904078000040EB00B7
:101BC000004F78007E409000814F500002003A00A4
:101BD00010C0B300004F78001E04E00008003A0077
:101BE0007E409000604798006E409000E84F5000A3
:101BF00003003E0060492200EE409000014878005A
:101C000010C0B3009E4F10000D003A005E409000DF
:101C10000081FB005E4090008080FB00D0482200E5
:101C200000804000904078001E40900080C070000E
:101C3000D048220000004100014878000F00370022
:101C40005E4090000081FB005E4090008080FB00C1
:101C5000D04822000080400010407800804078008A
:101C60001E40900000C0EA0000C060008040780084
:101C7000D048220000004100014878001E40780052
:101C80004CC80200000000007E4090000040E800C8
:101C9000704798001E409000004040001047980098
:101CA0001E4090000004E0000B003A005E409000EF
:101CB0008080FB00D0482200008040001040780067
:101CC000920007005E4090000040E80050479800F6
:101CD00010C0B300104798005E409000E74F5000DE
:101CE0008EFF3600FE40900000C4B30080CF50004D
:101CF0001000360080492200104078000004E00007
:101D00000C003A0050492200EE4090000148780053
:101D100050492200104078000004E00003003A001F
:101D200011C0B300704922000148780010C0B30010
:101D3000404798004E4090000004E000040032004C
:101D4000D0482200104078000004E0000B003A0068
:101D50008040EB0050492200014878008040EB00B1
:101D600070492200014878008040EB006049220061
:101D7000014878000040EB00404798004E4090003A
:101D80000080FB00400798004E0090000080FA00A1
:101D9000000006000E00FA000040EB0040479800EB
:101DA0000C0037004E4090000081FB004E40900038
:101DB0008080FB00D04822000080400090407800E6
:101DC00065004700017178004E4090000040E80037
:101DD000404798004E409000E74F5000F1FF36001A
:101DE0005049220090407800214798007049220015
:101DF000904078001147980060492200104F780009
:101E000001C4B30050492200014878008040EB0033
:101E100070492200014878001AFF07000004E00022
:101E20001A00320010C0B300304798000040EB00A9
:101E300040479800110037004E4090008080FB0022
:101E400065004700614178004E4090008080FB00B3
:101E5000D04822000080400010407800804F5100A0
:101E6000030032000040EB003047980009003700C3
:101E70004E4090000040E800404798004E409000DF
:101E8000E74F5000ECFF3600020037000040EB0047
:101E9000304798000040EB00404798000C003700A6
:101EA0004E4090000081FB004E4090008080FB007F
:101EB00065004700E1407800D04822000000410062
:101EC000014878004E4090000040E80040479800EC
:101ED0004E409000E74F5000F1FF3600504922007D
:101EE000AE40900001487800704922009E4090006A
:101EF00001487800604922001E4878003E4090006A
:101F00000080FB000080FA00000006000200FA00DA
:101F1000004F780080492200104078001E40680081
:101F20008080FB00901A22000080400090407800E2
:101F30008049220001487800804922001040780042
:101F40000080FB000080FA00000006000000FA009C
:101F5000E0A82A00809E0200000000000080FA0035
:101F6000000006000400FA00D822A800DA22A90026
:101F7000D882A900A0DE2100104078000040A00017
:101F8000A1DE210080487800A0DE2100104078000A
:101F90000030A100A1DE210080487800EBFF07009F
:101FA0000000370010A3020000000000804078000D
:101FB000B043220001487800B0432200104078006E
:101FC0000080FB004400DE0080407800A043220037
:101FD00001487800A0432200104078000080FB00F8
:101FE000100798001E009000E10F500078003200AA
:101FF0009E009000E48F50009A0032001E00900076
:102000000000E000010032009E003700B0432200D3
:10201000104078000080FB00000F78009E007800E0
:10202000E28F5000170032001E007800E20F5000CF
:1020300007003C009E0078000100E000950032009F
:102040001E007800E10F50000C0032005C003700E9
:102050009E007800E48F5000130032001E007800CC
:10206000E40F5000560035009E0078006880500054
:10207000E10F500052003E0010003700B3FF070090
:10208000C8FF370068C702000000000080407800E9
:10209000804322000148780010C0B30084A20200EF
:1020A00000000000BFFF370086C8020000000000EB
:1020B00084A2020000000000BAFF370010C0B30085
:1020C00084A2020000000000B0432200104078000B
:1020D000E94F500004003A00C1CEB300801A22003C
:1020E000014878000300370001CFB300801A2200B6
:1020F0000148780050FE07008040780080432200AD
:1021000001487800190037008040EB00904322001E
:10211000014878000D0037009043220010407800FD
:102120008080FB00D04822000080400010407800F2
:1021300084A20200000000009043220010407800BA
:102140008040E8009043220001487800904322003C
:1021500010407800E74F5000EFFF360044FE0700C4
:1021600080407800804322000148780080432200AC
:10217000104078000004E000E3FF3A008040EB00EC
:1021800090432200014878000800370000C0EB00AF
:1021900084A202000000000090432200104078005A
:1021A0008040E800904322000148780090432200DC
:1021B00010407800E74F5000F4FF360079FF3700F9
:1021C0000040EB0084A202000000000075FF370011
:1021D000B043220090407800F0C0B30080C060009F
:1021E000B043220001487800B0432200104078003C
:1021F0008040E800B04322000148780010C0B300DE
:1022000084A20200000000008040EB009043220006
:10221000014878000C00370010A302000000000005
:10222000EEC702000000000010C0B30084A202004C
:102230000000000090432200104078008040E80039
:10224000904322000148780090432200904078009B
:10225000B04322001040780080CF5000EEFF3900DC
:1022600050FF3700B043220010407800DCCD020060
:102270000000000010C0B30084A2020000000000B3
:1022800048FF37000040EB0084A20200000000007D
:1022900044FF37000080FA00000006000000FA004A
:1022A00020AB2A00809E0200000000000080FA009F
:1022B000000006000000FA000040EB005AB70200E0
:1022C000000000000040EB005AB7020000000000D0
:1022D0000040EB005AB70200000000000040EB0095
:1022E0005AB70200000000000000EB0096B60200A2
:1022F000000000000000EB0096B6020000000000A5
:102300000000EB0096B60200000000000080FA001A
:10231000000006000C00FA00881F7800A0DE2100F3
:10232000104078000040A000A1DE21008048780025
:10233000A0DE2100104078000030A100A1DE2100C5
:102340008048780011C0B30080DD2100014878008A
:1023500081C0B30090DD21000148780021C0B300A6
:10236000506722000148780080C0EB0020C0B30015
:1023700036B5020000000000D822A900D842A9000A
:10238000D862A80010C0B300C6B702000000000069
:10239000C2FF07000000370010A302000000000089
:1023A0008040780090672200014878009067220002
:1023B000104078000080FB004400DE008040780080
:1023C0008067220001487800806722001040780072
:1023D0000080FB00300798003E009000E30F5000A3
:1023E00014013200BE009000E38F50000A003C0050
:1023F0003E019000E10F5100A5003200BE019000A7
:10240000E18F5100F8003C003E0090000000E00029
:1024100012003200CE023700BE009000E68F50005E
:10242000770232003E019000E60F510004003C00AC
:10243000BE019000E48F510069023200C4023700EF
:102440003E009000E80F500084023200BE00900071
:10245000EA8F50002E013200BD0237009067220043
:10246000104078000080FB006101B900420798002D
:1024700053079800D0002000010020004E0190007A
:10248000DE019000800F5100818F59007C003E00DA
:102490004E009000DE00900000600100B0023700A6
:1024A0000C0037000D00370012003700170037000E
:1024B0001D00370023003700440037004800370074
:1024C0004C00370052003700580037005E003700DC
:1024D0006400370071FF0700AFFF3700C4B502008A
:1024E0000000000010C0B30084A202000000000041
:1024F000A9FF370004B602000000000010C0B300BE
:1025000084A2020000000000A3FF37000040EB009F
:10251000C6B702000000000010C0B30084A2020091
:10252000000000009CFF370010C0B300C6B70200D7
:102530000000000010C0B30084A2020000000000F0
:1025400095FF37005067220010407800E24F50009E
:1025500006003A00EAB60200000000008040780061
:10256000706722000148780006003700F00F200055
:1025700024B602000000000080407800706722004E
:1025800001487800A0DE210010407800684060001B
:102590000004E0000800320070672200104078005C
:1025A0000080FB0020C7020000000000804078008F
:1025B00070672200014878007067220010407800A0
:1025C00084A202000000000073FF370038B7020049
:1025D0000000000084A20200000000006EFF37002F
:1025E000D8B702000000000084A202000000000032
:1025F00069FF370010C0B3007CB702000000000084
:1026000010C0B30084A202000000000062FF370087
:102610000040EB00B4B702000000000010C0B3009F
:1026200084A20200000000005BFF370010C0B3006E
:10263000B4B702000000000010C0B30084A2020082
:102640000000000054FF37000040EB00A2B702007A
:102650000000000010C0B30084A2020000000000CF
:102660004DFF370010C0B300A2B702000000000009
:1026700010C0B30084A202000000000046FF370033
:102680000040EB0084A202000000000042FF37007F
:102690009067220090407800F0C0B30080C06000D6
:1026A000906722000148780090672200104078006F
:1026B0008040E800906722000148780010C0B30015
:1026C00084A20200000000008040EB00706722003E
:1026D000014878003D00370010A302000000000010
:1026E000804078006067220001487800A0DE210069
:1026F00010407800684060000004E00008003200EC
:1027000060672200104078000080FB0020C70200B4
:1027100000000000804078006067220001487800D7
:102720005067220010407800E24F500009003A0044
:1027300060672200104078000080FB0096B602001F
:102740000000000010C0B30084A2020000000000DE
:102750001900370060672200104078000080FB00FD
:1027600024B602000000000080407800606722006C
:1027700001487800A0DE2100104078006840600029
:102780000004E0000800320060672200104078007A
:102790000080FB0020C7020000000000804078009D
:1027A00060672200014878006067220010407800CE
:1027B00084A2020000000000706722001040780030
:1027C0008040E800706722000148780070672200AE
:1027D00090407800906722001040780080CF500031
:1027E000BDFF3900ECFE3700906722009040780072
:1027F000F0C0B30080C060009067220001487800FC
:1028000090672200104078008040E8009067220026
:102810000148780090672200104078007CB70200E1
:102820000000000010C0B30084A2020000000000FD
:10283000D9FE37009067220090407800F0C0B300C6
:1028400080C06000906722000148780090672200F5
:10285000104078008040E80090672200014878002E
:1028600010C0B30084A202000000000010A3020008
:102870000000000080407800806722000148780056
:102880008040EB0070672200014878001600370096
:1028900080672200104078000004E00004003D0042
:1028A00010C0B3005AB70200000000000300370058
:1028B0000040EB005AB702000000000080672200D1
:1028C000104078000040400080407800806722007F
:1028D0000148780070672200104078008040E800CE
:1028E00070672200014878007067220090407800ED
:1028F000906722001040780080CF5000E4FF39003C
:1029000010C0B30084A2020000000000A2FE370045
:1029100090672200104078000080FB00200798009C
:10292000400A2000AE009000808F5000120032005C
:10293000500A20002E019000800F5100B800320094
:10294000000A2000AE019000808F5100010032008B
:102950001F01370010A30200000000008040780033
:10296000406722000148780010C0B30084A2020032
:102970000000000088FE3700406722001040780009
:102980000080FB00100798001E009000E10F50002F
:10299000040032009E009000E28F500036003200AA
:1029A0009B00370010A30200000000000080FB0025
:1029B00090338900903381006300B900903389001F
:1029C0000000EB0080338900090037007127810087
:1029D000803381000084400010A30200000000004A
:1029E000004C7800803381000000E80080338900CB
:1029F0008133810090338100808F5000F3FF3900D4
:102A00000000EB008033890013003700712781003C
:102A100080338100008040000080E8001041780091
:102A20007127810080338100008040000000E800B1
:102A30009041780071278100803381000080400040
:102A400010407800834078004801070080338100FF
:102A5000630040008033890081338100903381001E
:102A6000808F5000E9FF390010C0B30084A202003B
:102A70000000000048FE370010A302000000000024
:102A80000080FB0090338900903381004200DD001C
:102A9000903389000000EB00803389000900370083
:102AA00071278100803381000084400010A3020060
:102AB00000000000004C7800803381000000E80036
:102AC000803389008133810090338100808F5000F2
:102AD000F3FF39000000EB00803389004400370029
:102AE0000040EB005AB70200000000000040EB007D
:102AF0005AB70200000000000040EB005AB7020085
:102B0000000000000040EB005AB702000000000087
:102B100071278100803381000080400010407800E0
:102B20000080FB0096B602000000000071278100C3
:102B300080338100008040000000E80010407800F1
:102B40000080FB0096B602000000000071278100A3
:102B500080338100008040000080E8001040780051
:102B60000080FB0096B60200000000007127810083
:102B700080338100008040006301400071278100A4
:102B800080338100008040006300400010407800E6
:102B90006F406000004978008040EB0070672200C1
:102BA0000148780006003700C2FD07007067220068
:102BB000104078008040E8007067220001487800EB
:102BC0007127810080338100008040006300400055
:102BD00090407800706722001040780080CF50004D
:102BE000F1FF3E00803381006400400080338900A3
:102BF0008133810090338100808F5000B8FF39000D
:102C000010C0B30084A2020000000000E2FD370003
:102C10000040EB0084A2020000000000DEFD37004F
:102C200040672200104078000080FB00000F780011
:102C30001E017800E10F5100040032009E0178006F
:102C4000E28F510040003200D3FD370010A3020094
:102C5000000000000080FB009033890010A30200F8
:102C60000000000080407800806722000148780062
:102C70000000EB00803389002E00370080672200BF
:102C80009040780060672200014878008040EB00A7
:102C90007067220001487800190037006067220041
:102CA000104078000080FB00610060000004E0003C
:102CB0000400320010C0B3005AB702000000000048
:102CC000030037000040EB005AB70200000000008C
:102CD00060672200104078000080FB000000D100F7
:102CE0008040780060672200014878007067220009
:102CF000104078008040E8007067220001487800AA
:102D00007067220010407800E34F5000E3FF360068
:102D1000EAB6020000000000EAB60200000000006F
:102D200084A2020000000000803381000000E8005F
:102D3000803389008133810090338100808F50007F
:102D4000CEFF390094FD370010A302000000000000
:102D50000080FB00903389000000EB008033890085
:102D60001600370022C0B30060B92000A10B20007C
:102D7000B8000700EB00070022C0B30060BB2D00C5
:102D8000A10B2000B300070022C0B300603D2D005E
:102D9000A10B2000AF000700E200070022C0B30033
:102DA00060BB2000A10B2000AA000700DD00070087
:102DB000803381000000E800803389008133810086
:102DC00090338100808F5000E6FF390072FD37009C
:102DD0000040EB0084A20200000000006EFD3700FE
:102DE0009067220010407800DCCD02000000000057
:102DF00010C0B30084A202000000000066FD37008E
:102E0000906722009040780030C0B30080C060001E
:102E10009067220001487800906722009040780077
:102E200080DD21000148780080DD2100904078009D
:102E3000506722001040780036B502000000000004
:102E400010C0B300C6B702000000000010C0B300FD
:102E500084A20200000000004FFD3700A0DE210028
:102E6000104078000040A100A1DE210080487800D9
:102E700090672200104078000080FB004300DE00D5
:102E80000000A200610060000004E00005003200C4
:102E9000A0DE2100104078000040A000A1DE21004B
:102EA0008048780021C0B3005067220001487800B4
:102EB00090672200104078000080FB004200DE0096
:102EC000610060000004E0000300320031C0B30084
:102ED0005067220001487800A0DE210010407800F1
:102EE0000030A100A1DE2100804878009067220018
:102EF000104078000080FB000000D10061006000FD
:102F00000004E00005003200A0DE2100104078003F
:102F10000030A000A1DE21008048780080DD210083
:102F200090407800506722001040780036B50200CB
:102F30000000000010C0B300C6B70200000000008F
:102F400010C0B30084A202000000000012FD370090
:102F50000040EB0084A20200000000000EFD3700DC
:102F60004F0478000080FA00000006000600FA0016
:102F70002047980031479800424798002E40900023
:102F80000080FB004600DE00004F78000040EB00B0
:102F900010479800220037001E409000E34F500079
:102FA0000C003A001E04E0000A00320010C0B3001A
:102FB000B4B70200000000001E80FB00BEC6020085
:102FC000000000000040EB00B4B702000000000069
:102FD000100037002E4090000080FB006100600070
:102FE0000004E0000400320010C0B3005AB7020031
:102FF00000000000030037000040EB005AB7020059
:10300000000000002E4090000080FB000000D10076
:10301000204798001E4090000040E80010479800AC
:103020001E409000E34F5000DBFF36003E40900012
:103030000080FB0096B60200000000004E409000A9
:103040000080FB0096B60200000000000080FA003D
:10305000000006000800FA001007980021079800F9
:10306000624798000040EB005AB7020000000000E1
:103070000040EB005AB70200000000000040EB00E7
:103080005AB70200000000000040EB005AB70200EF
:10309000000000001E00900020C702000000000099
:1030A00096B60200000000001E009000AE009000E6
:1030B0004809DD004800DE0000007100C808DE009D
:1030C00020C702000000000096B6020000000000C9
:1030D0001E009000AE0090004008DE0001002000BD
:1030E00020C702000000000096B6020000000000A9
:1030F0006E4090006F406000604798000040EB0019
:10310000004F7800020037006AFC07001E4FE800FD
:103110006E4090009E4F1000FBFF39000080FA00C7
:10312000000006000000FA0010C0B3005AB7020009
:10313000000000000040EB005AB702000000000051
:103140000040EB005AB70200000000000040EB0016
:103150005AB70200000000000000EB0096B6020023
:1031600000000000EAB602000000000084A2020095
:1031700000000000EAB602000000000084A2020085
:10318000000000004BFC07004AFC07000080FA002A
:10319000000006000600FA000000EB00800888002E
:1031A0000000EB00F00888000000EB00C00D880074
:1031B000103381000000E00008003A00416D20005B
:1031C0009140780000CCB30000C06000D4E6B700A6
:1031D0000000EB00A03289003D0037001033810071
:1031E000E30F500005003C00E0032000000F7800D2
:1031F00010A1A8001081A80015003700103381002D
:10320000FE0F500005003C00A00F2000000F7800CA
:1032100010A1A8001081A9000D0037001133810012
:10322000400F2000808F500005003C00007D2000F2
:10323000000F780010A1A9001081A8000400370039
:1032400000E82300000F780010A1A9001081A90058
:1032500010338100000178001E0078001100090081
:103260000280D8000000E900200798002E0090009E
:103270006008880020338100800078002E009000D4
